:020000040800F2
:100000000002002029050008C5040008810400083A
:10001000D5040008E5040008F5040008000000000D
:10002000000000000000000000000000450400087F
:100030000505000800000000290400081505000857
:100040008901000889010008890100088901000868
:100050008901000889010008D9160008D91600088E
:10006000D9160008D9160008D91600088901000819
:100070008901000889010008890100088901000838
:100080008901000889010008890100088901000828
:10009000890100088901000889010008D9160008B3
:1000A0008901000889010008890100088901000808
:1000B00099180008890100088901000889010008D1
:1000C00089010008890100088901000889010008E8
:1000D0008901000889010008491200084F12000830
:1000E000D916000889010008890100088901000863
:1000F00089010008890100088901000889010008B8
:1001000089010008890100089F180008890100087A
:100110008901000889010008890100088901000897
:100120008901000889010008890100088901000887
:100130008901000889010008890100088901000877
:100140008901000889010008890100088901000867
:100150008901000889010008890100088901000857
:100160008901000889010008890100088901000847
:1001700089010008890100088901000800000000C9
:10018000000000008901000800F0C4B900F004BBC1
:100190007047000070B50C46064600F061F9094B47
:1001A000094A1D682919914202D8084A914204D28D
:1001B0000C2333604FF0FF3500E0196000F058F970
:1001C000284670BD00020020000002202C600020A4
:1001D0001946104600F0ECBA1946104600F0F0BA85
:1001E000132303604FF0FF307047132303604FF079
:1001F000FF307047132303604FF0FF307047022930
:100200004FF0000303608CBF002001207047000006
:10021000114B70B500241C60104B114D18682E68EE
:1002200000F09CF80F4B53F820301B68A3F1080234
:1002300096420FD026B13179092904BF0A213171C4
:10024000092103F8041C33F9021C074B2A601980AA
:10025000012070BD204670BDF0020020C4030020C4
:10026000F802002000030020F4020020082930B525
:10027000037919D9082B32D842791A4B53F82250F6
:1002800000F108042DB12D68856053F822502C60D0
:1002900000E0846043F82240134C4279012303FAC2
:1002A00002F22368134319E0082B18D945790D4B46
:1002B00053F825203AB11468A2420BBF00222468EB
:1002C00043F825201460427953F822303BB9064C9C
:1002D000012303FA02F2236823EA02032360017177
:1002E00030BD00BF00030020C403002008B50A4B46
:1002F0001B681A79082A02D95B7983420AD900F06F
:10030000BAF818B1054B01221A6008BDBDE80840D3
:1003100000F082B808BD00BFF8020020F002002003
:1003200008B500F09DF8094B094A1B88094D1BB21E
:10033000002442F82340084A286813682146013BFC
:100340001360FFF793FF2C6000F062F8F4020020C6
:1003500040030020F8020020FC0200200023C20716
:1003600002D440080133FAE718467047134423F0DB
:10037000030310B54FF077321C1F43F8042C6207BB
:1003800042BF4FF0883243F8082CA3F108044FF025
:10039000807304E909000F4B44F80C3C002344F837
:1003A000103C032344F8143C2246022344F8183C32
:1003B000012344F81C3C42F8201D0B2342F8043D65
:1003C000013B032BFAD120466FF0020340F8443D75
:1003D00010BD00BF21030008064B0749074A1868F3
:1003E000884203D1934201D20433F8E70348C01A8C
:1003F000704700BF00000020FEE7FEE7000200207B
:10040000EFF30880704700000048704700000020AC
:1004100000F02AF801DFFEE7024A536843F08053F8
:100420005360704700ED00E0EFF3098020E9F00F22
:1004300040F804ED02490968086000F003F8000084
:10044000F8020020FFF7E4FE04480068016801C9D3
:10045000B1E8F00F81F3098800470000F80200209E
:10046000EFF3108072B6704762B6EFF310807047FA
:1004700080F310887047EFF30580C0B2704700002A
:100480000D490E4A0E4B6846904203D8984201D956
:10049000002102E009468D460121042072460242F5
:1004A00002D1EFF3088001E0EFF309802DE9F00FAE
:1004B0006B4600F06FF800BF000200200000022031
:1004C0006005002008B50249042000F08DFB00BF44
:1004D000C40F010808B50249062000F085FB00BFE3
:1004E000D00F010808B50249072000F07DFB00BFCE
:1004F000E30F010808B50249082000F075FB00BFB2
:10050000F50F010808B50249092000F06DFB00BF96
:100510000910010808B502490A2000F065FB00BF78
:100520001B1001087047704708B5FFF7FBFF6A46CC
:10053000114B1249934202D243F8041BFAE7104AC6
:10054000104B11498B4204D252F8040F43F8040BAC
:10055000F8E70E4B0E4A0021934202D243F8041BE7
:10056000FAE7FFF7E0FF00F01FFB0EF0FBFDBDE830
:10057000084000F073BB00BF00000020FEE7FEE76C
:100580005844010800020020F0020020F002002080
:100590002C6000202DE9F04F9A46494B8FB09346CE
:1005A0009A6B03925A6B04929F6ADA6A05921A6BED
:1005B000DB6B0793434B06921A68434B9A420446FF
:1005C000884602D041480FF063F8B8F1000F05D01B
:1005D0003F4800250FF05CF82E4626E094E80E0018
:1005E000E068D4F81C9008902069099060690A902E
:1005F00019F4007F3748A6690D930CBF04F120055C
:1006000004F124050C920B910FF042F8089B009323
:100610000BA90EC930480EF0B1FFCDF8009033465B
:100620000A9A09992D480EF0A9FF2D480FF030F8CD
:1006300039462C480EF0A2FF05992B480EF09EFF7C
:1006400006992A480EF09AFF079929480EF096FF5E
:100650003A0403D5039927480EF090FF3B0603D5D3
:10066000049925480EF08AFF24480FF011F85946E6
:1006700023480EF083FFB8F1000F1BD121480FF083
:1006800007F8314620480EF079FF69461F4BC91A1A
:1006900003D549421E480EF071FF20468268C368A8
:1006A00001698C4641698E46AD46514691E8F00F8E
:1006B0004168006801BE1749052000F095FA00BFA7
:1006C00000ED00E000000020FEE7FEE72910010831
:1006D0003F1001086E10010889100108C6100108BA
:1006E000041101080D1101081D1101082D11010847
:1006F0003D1101084D1101085D1101086D1101083E
:100700007211010884110108B51101085801002077
:10071000DD1101080A12010810B568B1012815D1D0
:10072000174A136823F003031360136843F400733C
:1007300043F0010313601BE0114B1A6842F00E02F4
:100740001A605A6842F480725A6011E00D4A1369C7
:1007500023F0040313610024FFF782FEBFF34F8FE1
:1007600030BFFFF785FE54B1BDE8104000F010BC6B
:10077000044A136943F0040313610124ECE710BD3C
:100780000070004000ED00E008B5FFF769FE0020B2
:10079000BDE80840FFF7C0BF034B044A4FF4E13106
:1007A000002000F0C7BC00BF04020020270E000894
:1007B0000A460146014800F041BB00BF0402002088
:1007C00010B50A460C460146002000F019FD2046EF
:1007D00010BD002001F00AB8034B1968024611B998
:1007E000084600F0CFBF70470C04002010B5094A3E
:1007F00013685BB19C6881688C4202D21A461B6800
:10080000F7E703D15C6841688C42F7D90360106058
:1008100010BD00BF18040020F0B51F4E1F4D3368F7
:100820001F4C013333601F4B00201A6818602B687F
:10083000226019460746B64641B1DEF800C08E6810
:10084000664503D80F4601200968F5E700B1296025
:1008500007B9F0BD00213960E2B133B15168586881
:10086000814294BF1146194600E0114608461268BD
:100870001B680AB903600BE00BB9026008E0556819
:100880005E68B54294BF15461D4605602846EEE7F2
:100890002160F0BD2360F0BD10040020180400208A
:1008A00014040020080400202DE9F0412E4F2F4CA5
:1008B00001233B6023683BB9FFF7AEFFFFF789FFD9
:1008C0000130FBD0002502E0FFF783FF05464FF023
:1008D0000008236823B9FFF77CFF854214D91AE08A
:1008E0005E68FFF776FF854208D923685E68FFF7E8
:1008F00070FFA8422CD3B042F7D329E08642F4D946
:10090000361A132EE7D8F0E7236843B9FFF761FFE3
:10091000854206460BD9FFF77FFF0025D9E75E68C1
:10092000FFF757FF063E14308642D2D309E010F19C
:10093000140F04D3FFF74DFF8642FBD9EBE74FF0CE
:10094000FF3600233B603046BDE8F041FFF744BF6F
:1009500023681A682260C3F80480C3F80880DA6844
:1009600018699047B5E700BF0C040020140400206C
:10097000144B1A6882420AD112681A6012B1506888
:10098000063801E04FF0FF30FFF726BF13461A6824
:1009900022B19042FAD102681A6070470A4A13687D
:1009A0001BB1984203D01A46F9E7084A05E00368EC
:1009B000136070479842FAD01A461368002BF9D199
:1009C000704700BF14040020080400201804002011
:1009D00008B500231846054A054900F019FF4FF0F5
:1009E000FF30BDE80840FFF7F7BE00BFA9080008C8
:1009F00040420F0070B5084EFFF7EBFE3468054625
:100A0000FFF7E7FE8542F7D800222346141843F18A
:100A100000052046294670BD10040020F8B50446A4
:100A20000D46FFF7D6FE002385420646236010D30D
:100A3000A5F10A0383420CD20A35FFF7CAFE8542AC
:100A4000FBD3FFF7C6FE8542FBD8E36820699847D1
:100A50003EE0FFF705FD63680746002B34D1A3682D
:100A6000002B31D11B4B65601A681B68B54238BF3B
:100A70000132A260A2689A4203D92046FFF7B6FE6F
:100A80001EE0B54202D9144B19460EE0134A136812
:100A900023B159688D4201D31A46F8E723601460E8
:100AA0000EE05068854203D313461A68002AF8D135
:100AB00022601C600B689C4202D1A81FFFF78CFECD
:100AC0003846FFF7D5FC03E02046FFF751FFC9E7A2
:100AD0000020F8BD100400201404002008040020A9
:100AE00038B50446FFF7BCFC6368054633B9A36814
:100AF00023B92846BDE83840FFF7BABC2046FFF7C7
:100B000037FFF6E7C36870B504460D46C3B1FFF77B
:100B1000E7FF092D0CD8FFF75CFE0646FFF759FEEC
:100B2000801B8542FAD8E3682069BDE87040184709
:100B3000FFF74FFE29182046BDE87040FFF76EBF53
:100B400070BD00002DE9F04704460E4690461AB9E4
:100B5000BDE8F047FFF7D6BFFFF782FC63680746A2
:100B6000E3B9A368D3B9DFF83CA0FFF732FEDAF8A7
:100B700000508146FFF72DFE8145F6D8304408EB42
:100B80000502864288BF01326060A2602046FFF7FE
:100B90002DFE3846BDE8F047FFF76ABC2046FFF758
:100BA000E7FEE0E71004002008B50121094800F045
:100BB0009BFC0121084800F097FC0121074800F048
:100BC00093FC0121064800F08FFCBDE8084000F0CE
:100BD00021B900BF0D0C02400C0C02400E0C02406B
:100BE0000F0C02407047000008B50F4B1A680C4606
:100BF0009AB9012203281A6003D171460B480EF0FE
:100C0000BDFC21460A480EF0B9FC00F04FF9094836
:100C10000EF0B4FC08480EF0B1FCFFF721FCFFF722
:100C2000E1FFFFF7B1FD00BF1C0400202F120108F7
:100C3000331201085B1201084F12010808B501F0D8
:100C4000B5F903480EF09AFC01F0D8F8002008BD71
:100C50005D12010808B500F00BF9FCE71FB5FFF7BE
:100C6000FFFB0E4B0E481B68029300240D4B0093B4
:100C70000F220C234FF48071019400F055F80A4BB9
:100C80000A481B6802930A4B009307220C234FF477
:100C9000C061019400F048F8FFF7BAFB1802002089
:100CA00020040020550C00081C0200202005002014
:100CB0003D0C000808B5FFF7D3FB094B1B681A79F8
:100CC000082A07D95A79074B53F8221011B109683D
:100CD00043F82210FFF7CCFBBDE80840FFF79CBBB0
:100CE000F80200200003002038B50B79082B03D947
:100CF00008490320FFF778FF4C7901F108020368E7
:100D00002BB113F8035CAC4201D31846F7E78B60B4
:100D1000026038BD1D120108031F53F8042F9A42C8
:100D2000FBD0181A704700000F2A2DE9F74F05462F
:100D30008B4691469A462AD810F003031BBFC3F195
:100D40000403ED180B46CB1A303B23F003031AF0D3
:100D5000080F05EB030405D02A46A24203D2126015
:100D60000432FAE72D600193FFF77AFB2749019BD4
:100D70008046012251F8227016B25FB10132212A59
:100D8000F8D14046FFF774FB6FF08A003BE06FF04C
:100D9000150038E01D490C9841F822402A46E680AB
:100DA0000D99FFF7E3FA0E9B194AA3624FF0FF3348
:100DB000E3611368206001331AF0010F6562C4F823
:100DC0002CB084F805902771A760E7602761676100
:100DD000A7612762136004D001212046FFF746FA7D
:100DE0000DE00A212046FFF741FA1AF0040F06D160
:100DF0004046FFF73DFB4846FFF778FA02E04046E1
:100E0000FFF736FB304603B0BDE8F08F400300200B
:100E1000FC02002008B501F039FB00F0B9F8BDE88C
:100E2000084000F01CB838B50446043000F04FFD0F
:100E30000546204601F02AF9284638BDF8B5044693
:100E40000E461746051D3A463146284600F02AFD53
:100E500020B90121204601F0E9F8F4E7F8BD08B512
:100E6000002000F01BFA0120BDE8084000F016BA8F
:100E7000F8B50D4B1E68C6F307221D4622B9F4B221
:100E8000003418BF012400E00224FFF7E9FA2B68C0
:100E90009E42074602D12046FFF73EFC3846BDE899
:100EA000F840FFF7E5BA00BF200200202DE9F04F1F
:100EB0002C4B2D4A1B882D492D482E4EDFF8CCB0E7
:100EC0008BB00DF1280906F1800A29F8043D0EF0D7
:100ED00055FBFFF781FA0546FFF796FA0446FFF740
:100EE0008FFA2A46009023464FF4007122480EF0F4
:100EF00045FB25EAE5754FF4007856F8044B14B32A
:100F00002779E26A5BF82730606A0793904406927B
:100F1000FFF702FF069AB4F90610079B101A226821
:100F20000592626A04920390E26A029262790192E7
:100F3000082FD4BF4F4609F1010700970544A26A64
:100F40000E480EF01BFBB245D7D10D4B02958DE834
:100F500008010C4A0C4819460EF010FB0BB0BDE816
:100F6000F08F00BFB5120108E4120108EA1201086F
:100F7000EF12010844030020371301088113010810
:100F8000BD130108BF130108C3130108B8120108FB
:100F900038B5FFF765FA1B4C0023E360054600F007
:100FA00037F84FF41443A360A268164B12F00C0FED
:100FB000FAD1154A40F20571116081221A601A684F
:100FC00042F480321A601A6812F4003F0D4AFAD0D7
:100FD0000E4B5360136843F0807313601168094B24
:100FE0008901FBD59A6842F002029A609A6802F081
:100FF0000C02082AFAD100F017F82846BDE838405C
:10100000FFF736BA00380240003C0240042A40078D
:10101000044B1A6842F001021A601A689207FCD564
:10102000704700BF00380240044B9A6812F00C0F62
:101030001EBF1A6822F001021A6070470038024091
:10104000034B044A00280CBF10461846704700BFE7
:1010500000BD010580DE800204281CD8DFE800F016
:1010600003080D1217000D4B1A6C1143196412E09E
:101070000A4A536C194351640DE0084A136B194333
:10108000116308E0054A536B1943516303E0034AB7
:10109000936B19439163BFF34F8F70470038024041
:1010A000042821D8DFE800F003090F151B000F4AC0
:1010B000136C23EA0101116470470C4A536C23EA54
:1010C000010151647047094A136B23EA010111635E
:1010D0007047064A536B23EA010151637047034A84
:1010E000936B23EA01019163704700BF003802400F
:1010F00038B514230C4A4343D4582568AA0608D5AA
:101100000A4B616803EBC002C9B253F83030506833
:1011100098472B0748BF6368054B1B681BB1BDE8A8
:101120003840FFF7C7BD38BD3C140108200B002034
:10113000F002002001282DE9F04780460D461746B1
:1011400003D92B490320FFF74FFDDFF8B090294A60
:10115000142404FB009442F83070E66802EBC002ED
:1011600001215360304600F0BFF9304600F092FA9A
:101170003046617C00F054FA4E464FB1D4F80890E6
:101180000021484600F0B0F9217C484600F048FABA
:10119000142303FB08F806EB080999F812A0D9F804
:1011A00004105046FFF758FF56F808400023E3604C
:1011B000504623616361FFF743FFB0FBF5F080B257
:1011C000A06077B199F8133001215AB203F01F03E0
:1011D00001FA03F35209084941F8223042F22C0384
:1011E00001E042F20803E3600020BDE8F08700BFA1
:1011F0001D120108200B002000E100E03C14010852
:10120000012838B505D80E4C14230A4403FB0043CB
:1012100009E00C490320FFF7E7FC25682D06FCD503
:1012200011F8015B65608A4201D01C68F5E7142360
:101230005843034B1A5813685B06FCD538BD00BFF2
:101240003C1401081D1201080020FFF751BF0120C6
:10125000FFF74EBFF8B5104C04EB4014012167684E
:10126000384600F041F9A6680021304600F03CF90C
:10127000E5680121284600F037F9247D38462146EB
:1012800000F0CEF92146304600F0CAF92146284642
:10129000BDE8F84000F0C4B97014010801282DE938
:1012A000F041044603D910490320FFF79DFC0F4B82
:1012B000DFF83C80002543F820506401FFF7CAFFA7
:1012C00008EB04031E7F9F6930463946FFF7C4FED2
:1012D00058F8043039461D603046DD615D60BDE878
:1012E000F041FFF7DDBE00BF1D120108300B0020EA
:1012F00070140108012870B50C4621D84A1C22D070
:1013000021F0FF0313F5807F11D114F0FF041AD1EF
:101310000E4B03EB40152E69731C14D0012130468F
:1013200000F0E2F8297D304600F07AF906E001216C
:10133000204600F0D9F8204600F0ACF9002070BD3E
:101340004FF0FF3070BD6FF0010070BD70140108E8
:10135000042B2DE9F84304460E461546984603D95A
:1013600017490320FFF740FC1648DFF8609067013B
:10137000012100EB840000F059FE09EB07031C7FFC
:1013800099692046FFF768FE0F4B59F8071004EBE8
:1013900084041C4416F5807F14F8082045EAC20531
:1013A00045F004050D6015BF0B684B6843F44073AE
:1013B00043F0040314BF0B604B600020BDE8F883CA
:1013C0001D120108300B002064140108701401087C
:1013D0000B4A430110B50446D018D3588169007FE9
:1013E00000221A605A6822F004025A60FFF758FE81
:1013F000044800EB8400BDE8104000F047BE00BF89
:1014000070140108300B00202DE9F843089E099F55
:10141000884691461D4623B91EB931490320FFF77E
:10142000E3FB304B400118F5807F1C58236843F0E4
:101430004003236005D0B8F1FF3F02D0404600F0E2
:1014400032F9A6B92F44AF4206D0A3689E07FCD557
:1014500015F8013B2373F6E7A3689807FCD5A3684A
:101460001906FCD4A368DA0720D5E368FAE70DB1C2
:10147000002319E030463744B84217D0A3689B07D1
:10148000FCD52573A368DE07FCD5237B00F8013B60
:10149000F2E7A2689007FCD5EA5C2273A268D10744
:1014A000FCD5227BF2540133BB42F2D1A3689A07E8
:1014B000FCD5A3681B06FCD4B9F1000F0ED1B8F11E
:1014C000FF3F0BD0236818F5807F23F04003236093
:1014D00004D04046BDE8F84300F0DCB8BDE8F8832E
:1014E0001D12010870140108F8B50D460126C0F35D
:1014F000832120F00F0400F00F0706FA01F102200B
:10150000FFF7AAFD07FA06F00323216883406FEA7C
:10151000030C01EA0C012160216805F0030E0EFAAC
:1015200000FE4EEA01012160E2680CEA0202E2607C
:10153000E168C5F3810282400A43E2606268BE400E
:1015400022EA060666606268C5F30015BD401543D1
:101550006560A2681343A3600020F8BD2DE9F04147
:1015600000F00F0415462B4A42F8343002EBC40257
:10157000069B536006468846C0F383274FF480419C
:101580000120FFF769FD41463046FFF7ADFF042C0F
:10159000214B03DCA11D01228A4003E0092C03DC5E
:1015A0004FF400021A6002E04FF480725A601B4B45
:1015B0000120996800FA04F2D243114099609968B9
:1015C00005EA000E0EFA04FE4EEA01019960D968A0
:1015D0000A40DA60C540DA68A54004F00C0404F162
:1015E000804404F59C341543DD6006F00302A568D1
:1015F00092000F21914025EA0101A160A168974066
:10160000B0400F43A76058611A681043186000206B
:10161000BDE8F081380B002000E100E0003C014013
:1016200020F00F0300F00F02F0B51E6857000325ED
:10163000BD4026EA05051D601D680224072A04FA3C
:1016400007F444EA050494BF002201221C6003EB66
:10165000820300F007001C6A80000F22824024EA07
:1016600002021A621A6A814041EA02001862F0BD61
:1016700020F00F0300F00F00196810B5032244009A
:10168000A2400A4214BF5B691B69012202FA00F002
:10169000184010BD20F00F02012300F00F0003FAE4
:1016A00000F09061704720F00F0200F00F00103042
:1016B000012303FA00F09061704710B50446FFF76C
:1016C000D7FF20B12046BDE81040FFF7ECBF204611
:1016D000BDE81040FFF7DEBF104B2DE9F0415E6919
:1016E0001A680F4F164000244FF001081D4608FAF3
:1016F00004F31E4206D06B6107EBC40357F8342095
:10170000586890470134102CF1D1064B1B681BB16F
:10171000BDE8F041FFF7CEBABDE8F081003C0140E2
:10172000380B0020F00200202DE9F843124ADFF8C0
:10173000508003010746D5582E69EB6800241E40EF
:1017400008EBC0090223A3401E4209D0EA68D9F879
:10175000040022EA0303EB60214658F8373098472B
:101760000134042CEED1054B1B681BB1BDE8F843D6
:10177000FFF7A0BABDE8F883B0140108F00200201A
:10178000B80B0020032910B516D80D4B00011C180A
:101790001B586068024001F10C0003EB80004260BE
:1017A0001869022202FA01F120EA01021A61DA68DC
:1017B0001143D960002010BD4FF0FF3010BD00BFB5
:1017C000B014010803290BD8074B00010222185856
:1017D000C36802FA01F123EA0101C16000207047E9
:1017E0004FF0FF30704700BFB01401080001024BFA
:1017F0001B58586A704700BFB0140108034B000122
:101800001A58136843F0010313607047B0140108BD
:1018100001282DE9F8430546884630D81A4E1B4961
:101820000401371941F8302097F80C9001EBC00102
:1018300048464B60B968FFF70FFC36597B680024B7
:10184000346048467460F362FFF7FAFB104B7A7B12
:1018500013F809305843B0FBF8F3013BB36251B2BF
:10186000012302F01F02736149099340094A284687
:1018700042F82130FFF7C2FF2046BDE8F8834FF061
:10188000FF30BDE8F88300BFB0140108B80B00209A
:10189000D014010800E100E00020FFF745BF01205F
:1018A000FFF742BF70B513467BB18568C468A54297
:1018B0000BD084680668651C85604568013D2C4036
:1018C000013B345D01F8014BEEE7D01A70BDC368EF
:1018D000426830B584681B1B934208D0C368046813
:1018E000013A5D1C1340C560E154002030BD4FF04B
:1018F000FF3030BD002208B5104601210AF042FB3E
:101900000121084600220AF03DFB0B4A0B48002348
:1019100013600B4A13600B4B01221A60FFF7C3FEE2
:101920000948FFF7C0FE0948FFF7B4FE0848BDE8C4
:1019300008400DF0ADBE00BFE01200200D0C0240CB
:10194000680C00209C0C00200C0C02400E0C024085
:10195000E01401082DE9F0479E4C90B040F2D243CC
:101960001822002104A8E3820DF000FD0423049353
:1019700099497B2305A8ADF8263007F0DFFC00234A
:101980001A462146954806F0BFFF0028C0F21A818A
:101990004FF000084446052708220AAE0096904BF7
:1019A0008E480DEB020107F013F80028C0F2848086
:1019B000DFF874920020FFF719FFD9F80030029D7C
:1019C0005D1B0544294687480DF0D8FDBDF80C2065
:1019D00046F667739A42DFD1B8F1000F13D1804900
:1019E00004A80AF0E3F9002803DA7F480DF050FE5E
:1019F000F5E70AF03FFA89E8030001467B480DF05D
:101A0000BDFD4FF00108012C13D179480DF040FEC7
:101A1000734904A80AF0CAF9002801DA7248F5E708
:101A20000AF028FA89E80300014670480DF0A6FD87
:101A3000002447F22F539D42DFF8F09166DD052F19
:101A400040F0AD80D9F8003053B9334602226949DD
:101A5000624807F02BF8002802DA67480DF018FEFC
:101A6000664B1F68012F0BD140F2DB323946002054
:101A70000AF088FA4FF47072394638460AF082FA52
:101A80005F4FD7F800A0BAF1000F40F088805D48A2
:101A90000DF0FEFD5C48FFF706FE5C48FFF703FE15
:101AA0005B48FFF7F7FD46F270225146012007F030
:101AB000BFFC01233B6072E056480DF0E9FD504B3E
:101AC0001A683AB934B9012046F2702221461860EA
:101AD00007F0AEFC494B1C68012C15D1214640F2A1
:101AE000DB3200200AF04EFA4FF470722146204695
:101AF0000AF048FA4448FFF7D6FD4448FFF7D3FD03
:101B00004348FFF7C7FD47E7012445E7052F57D1B5
:101B10004FF47872012100200AF034FA012140F2DA
:101B2000922208460AF02EFA344B01201860002554
:101B3000334B29461D60FFF745FE334602223649E6
:101B4000264806F0B3FFA84202DA2B480DF0A0FDAC
:101B50002E48C9F80050FFF7A6FD2D48FFF7A3FD5A
:101B60002948FFF797FD39462C480DF007FD08225C
:101B700000210DEB02000DF0F9FBD9F80030012B2C
:101B80007FF40AAF334602222549144806F08EFF3F
:101B90000028BFF601AF18480DF07AFDFCE6334689
:101BA000022214490D4806F081FF002802DA12488B
:101BB0000DF06EFD47F230539D424FF00007D2D139
:101BC0000137D0E717480DF063FD002010B0BDE8E5
:101BD000F08700BF3C020020F0140108C80B002071
:101BE000404B4C0018150108321501086815010812
:101BF00075150108C2160108B2150108E01200208F
:101C0000680C0020C61501080C0C02400E0C0240A6
:101C10000D0C0240E1150108A5240108D2150108A8
:101C20009A29010800150108E81200209C0C0020E8
:101C3000F0B51C491C487B23CB82002389B01A468F
:101C400006F062FE002827DB184C04F1180702AEEC
:101C500000964FF0FF3330221449134806F0B8FEC7
:101C60000028F4DB0020FFF7C1FD114D00BA2B68FE
:101C7000206200203B60FFF7B9FD00BAA062334646
:101C80003022A5F12801084806F010FF0028DEDA0E
:101C900008480DF0FDFCDAE707480DF0F9FC0020DC
:101CA00009B0F0BD24020020F41E00206C0C0020BE
:101CB000940C0020B21501080015010830B58DB054
:101CC000672318228DF8143000216F230DEB0200DA
:101CD0008DF815300DF04AFB0423069340F2D243F1
:101CE000ADF82E30BA238DF81C30AD238DF81D30A1
:101CF000A5238DF81E3055238DF81F3017238DF83E
:101D00002A3036238DF82B30022400250020FFF7DF
:101D10006DFD0CA906AB41F8200D08221D4806F008
:101D2000C5FE002802DA1C480DF0B2FC00954CF20A
:101D30005033032203A9174806F04AFE002807DAA9
:101D400074301AD015480DF0A3FC022C0AD014E010
:101D50009DF80C306E2B05D0612B0ED11048FFF78B
:101D600099FC0AE00F48FFF79EFC0D48FFF79BFC2B
:101D70000D48FFF7A2FC022406E00B48FFF793FC96
:101D80000848FFF79AFC01240848002160430AF044
:101D90002BFABBE7C80B0020EE150108041601085A
:101DA0000E0C02400D0C02400C0C024040420F0091
:101DB00084B030B58BB00FAC84E80E0000231A4617
:101DC0002146054603F04EFC58B9282221466846B4
:101DD00007F0FEF92A46014606480DF0CFFB012028
:101DE00003E005480DF0CAFB00200BB0BDE8304011
:101DF00004B070471C1601084E16010810B50821E2
:101E0000ACB0564800F02EFB08AC55480DF040FC35
:101E10001022002120460DF0A9FA102200210CA862
:101E20000DF0A4FA05A802F00BFFBA238DF82030BC
:101E3000AD238DF82130A5238DF8223055238DF860
:101E4000233008230093002206AB0221BDF91400C1
:101E500002F0E2FC0028A4BF9DF818308DF82E3067
:101E60004FF08002A4BF9DF819308DF82F30214625
:101E70000CA80DF0E1F9002340222146BDF9140021
:101E800001F07AF89DF82E30172B5BD19DF82F309A
:101E9000022B23D10B9B009394E80E000120FFF747
:101EA00087FF304B029300242F4B009308220C2312
:101EB0004FF4C06101942D48FEF736FF2C4B18807B
:101EC0002C4B02932C4B00930194082306224FF4D1
:101ED000C0612A48FEF728FF294B31E0362B31D16B
:101EE0000023284A28490120FFF792FC4FF47A7317
:101EF00000211A46084609F0D1FF002210460121B0
:101F00000AF040F84FF47A731A460021012009F0D4
:101F1000C5FF0121002208460AF034F800211B48C1
:101F20000AF062F91A4B029300230193194B0093B4
:101F3000062208234FF4C0611748FEF7F5FE174B41
:101F4000188002E016480DF0A3FB16480DF0A0FB28
:101F500080220CA9144807F0D3FA00BFA012002079
:101F60007216010899160108BD1C0008F212002023
:101F7000E4120020AC160108311C0008F218002001
:101F8000640C0020F518000800BD010580841E00C7
:101F9000C416010855190008A00C0020F0120020FA
:101FA000D7160108E2160108D414010808B500206C
:101FB00007F04CFAFEF70CFD03F06EF804F04EFE4D
:101FC00000F03EFC06F018FF00F006F801F05AF9A8
:101FD000BDE8084003F0A2B913B50E4C0E490F48F6
:101FE0000AF06EF90D49204602F06AFD002806DA73
:101FF0000B48002102B0BDE810400DF0BFBA0094BC
:10200000084B094802224FF4806102F0EFFD02B054
:1020100010BD00BFE8230020001701089023002016
:102020001817010852170108901F002070B50546C7
:102030000C46FEF715FA2B6806462BB94FF0FF3316
:102040002B60FEF715FA18E0CCB10F4B1C6802218B
:102050002046FEF70BF92B68013305D104F1080384
:102060002B600023A36003E021462846FEF73CFED8
:102070003046FEF7FDF9FEF7CFF9012070BDFEF7FF
:10208000F7F9204670BD00BFF802002070B5044685
:10209000FEF7E6F9256806461DB16B1C05D1002345
:1020A0002360BDE87040FEF7E3B928460A2150F8E6
:1020B00008392360FEF7DAF8236813B94FF0FF33CD
:1020C000236015F8034C3046FEF7D2F92046BDE8F0
:1020D0007040FEF70BB90000F8B505460E46FEF756
:1020E000BFF9364B364A1B881BB2074652F82320ED
:1020F000D2F820E0BEF1000F1AD054699369A342D0
:1021000016D9631C5361D3691C4046B9136933B9AE
:10211000631C04D13846FEF7ABF92046F8BD002C0D
:102120000ADB0EEBC40393E8030085E8030004E038
:102130004FF0FF34002EE9D0D560166976B33368CE
:102140001361002C0CDB95695169D369691A8B42C4
:10215000A9BF691C4FF0FF351D4091610EEBC5050D
:10216000736893E8030085E8030016F8043C052B28
:1021700009D0002373600A21A6F10800FEF776F863
:1021800016F8034C00E00F243846FEF771F90E2CC8
:1021900002D82046FEF7AAF80120F8BD002C09DA83
:1021A00010460321FEF762F83846FEF761F9FEF7A4
:1021B00033F9F1E73846FEF75BF9EDE7F40200206A
:1021C0004003002010B583694469C2691C1BA24208
:1021D00001DA002010BD5C1C13408461F9D4026A4E
:1021E00003C902EBC30383E80300012010BD000014
:1021F0002DE9F8431E46264B53F82150254B1B88EA
:102200000380074691462DB93046FEF731F94FF06D
:10221000FF3439E02B79032B28D01F4B0146284689
:10222000D3F80080FFF7CEFF044638B13046FEF702
:102230001FF998F80430052B25D122E0B9F1000FE1
:1022400003D13046FEF714F91EE098F80430C8F8C0
:102250000C70052B0CBF052104214046FEF706F843
:10226000414605F11000FEF73FFD07E003C8EB68AB
:1022700083E803000A212846FDF7F8FF3046FEF701
:10228000F7F8FEF7C9F801242046BDE8F88300BF3F
:1022900040030020F4020020F802002038B5044674
:1022A000FEF7DEF8074B1B882380074B21460546C7
:1022B0001868FFF787FF04462846FEF7D9F820463E
:1022C00038BD00BFF4020020F802002008B50F4B13
:1022D00053F82130B3B1212202801A79032A0BD19D
:1022E00003C8DA6882E8030018460A21FDF7BEFF3A
:1022F000074B0120186008BD01461846BDE808409C
:10230000FFF760BF4FF0FF3008BD00BF4003002063
:10231000F002002070B504460D46FEF7ACF828B177
:1023200029462046BDE87040FFF7D0BF094B1B8807
:102330001BB29D4204D12046BDE87040FFF7AEBFFE
:10234000FEF78EF82946034601222046BDE870407C
:10235000FFF74EBFF402002070B504460D46FEF7AD
:102360008AF8064628B129462046BDE87040FFF7A6
:10237000ADBF0A4B1B881BB29D4204D12046BDE86D
:102380007040FFF78BBFFEF76BF8324603462946D5
:102390002046BDE87040FFF72BBF00BFF4020020CD
:1023A0002DE9F041124F3B881BB2934206460C4682
:1023B000154603D10F490320FEF716FCFEF750F82F
:1023C0003A880D4B12B2804653F8227005213846E8
:1023D000FDF74CFF96E80300FC60434684E80300E9
:1023E000012229462046BDE8F041FFF701BF00BFAA
:1023F000F40200201D1201084003002070B50446BD
:102400000D46FEF72DF8B4F90020114B53F8224089
:1024100006461CB90F490320FEF7E6FB2379052B7E
:1024200004D0FEF725F84FF0FF3070BD95E80300AB
:10243000E36883E803000A212046FDF717FF64796B
:102440003046FEF715F82046FDF750FF012070BD1D
:10245000400300201D1201080021FFF73DBE0121AD
:10246000FFF73ABE08B5074B4A1E1B6811401862B9
:1024700003D005490320FEF7B7FB59619961DA6182
:1024800008BD00BFF80200201D1201080F4BD3F851
:10249000882042F47002C3F888200D4A9A60102206
:1024A00083F822200021DA7701F1604000F56140D5
:1024B0000131522980F80023F6D11A6942F0100246
:1024C0001A615A6942F400725A61704700ED00E0E7
:1024D00000000008034600201BB1DA685B68104466
:1024E000FAE7704710B50822094904460CF072FE5D
:1024F00048B12378FF2B08D1607800F00F00831ECD
:102500005842584110BD012010BD002010BD00BF31
:10251000B4170108002102F0CDBE38B5CBB20021BE
:1025200014460246084602F0A1FB054618B92046AB
:10253000FFF7F0FF0FE094F9103001330AD1A368E0
:1025400082681B7903F03F0321462046137102F095
:1025500071FC04466C60284638BD00002DE9F04748
:102560008C680746104688461546FFF7B3FFA379E7
:1025700040BAFF2BA0800AD12B7C023BDBB2022B9E
:1025800003D8214AD35CFF2B00D13B23A371E3790D
:1025900043B90FB9402304E0384600F0CFFC90F86F
:1025A000CA31E37104F108061022184930460CF0D4
:1025B00011FE8246D0B904F1180915491022484687
:1025C0000CF008FE014630B9102230460CF0CEFE69
:1025D0000123E3750AE049465246384600F088FD7B
:1025E000014618B1102230460CF026FE414628461E
:1025F00002F0DAFB002804DA831C08BF0020BDE8E3
:10260000F0870020BDE8F08761170108C4170108B2
:10261000141801088B6870B558800C46054600F008
:102620008DFC014618B919490320FEF7DDFA6668EA
:102630003046FFF74FFFB1F8C831984204D9204621
:10264000BDE87040FFF766BFD1F81C320133C1F816
:102650001C323046FFF73EFFD1F824321844B1F85F
:10266000C631C1F82402DB0708D5234640F2022216
:102670000749012002F07CF830B9E0E721462846FE
:1026800002F0AFF80028DADD70BD00BF1D120108AE
:102690000000FFFF2DE9F04F85B090F910300133B5
:1026A00000AF044689460AD18368B3F9026002F09C
:1026B0000FFE00286AD043680446984601E0804631
:1026C0000026404602F004FE054600285ED0444540
:1026D000836818BF60601A461B7ED0F8048008BF6C
:1026E0000446FF2B2BD186B907F1080002F0A8FAA7
:1026F00000284BD0002122460846B7F90860FFF7B2
:102700000CFF0446002800F09380B9F1000F06D0BA
:10271000424629463046FFF721FF002836DBA268F3
:10272000137943F040031371304600F05FFE4368B5
:102730000133436021463046FFF76CFF78E01346D3
:10274000183310223C4918469B460CF043FD40B11B
:102750005946002E39D1381D00F06EFC064600287F
:1027600038D0B9F1000F06D0424629463046FFF76F
:10277000F5FE00280ADB2846FFF7ACFE00210246E2
:102780000223084602F0A4FC064608B9204619E0D8
:1027900083689846EA68A96840460CF04DFDEB68EE
:1027A0006D6842461A449046002DF3D12046FFF74B
:1027B000B1FE224B3146B3F9000002F01FF80028A9
:1027C00036DC3046FFF7A6FE32E0304600F00CFC67
:1027D0000028C6D107F11001082301F80D3D32464B
:1027E0005B4607F1080005F0E1FCEA46064640B109
:1027F000B9F1000F09D042462946FFF7AFFE002885
:1028000003DA2046FFF786FE11E02246F97807F149
:102810000800FFF782FE044648B1304600F0E6FDAE
:1028200003680133036021463046FFF7F3FED546C7
:102830001437BD46BDE8F08F141801082C24002081
:102840001FB50F4CB4F9003063B90E4A01930E4B1B
:1028500002920093042208234FF480610B48FEF794
:1028600063FA20800A480B4B036001230371142391
:1028700083600AF052FFB4F9000004B010BD00BF3D
:102880002C2400205C170108392B00082E2400207E
:10289000F823002030280020292B2DE9F843814619
:1028A0000F4614461D4606D03A2B06D0112B0CBFFE
:1028B0000423002302E0022300E00323292D3B74BC
:1028C00001D03A2D03D1A74259D1012605E0A742F4
:1028D00002D063689F4252D100267B6893F91000B2
:1028E000022805D016B30121204602F0D1FC1DE0DC
:1028F000294602F03DFA18B986F0010836B101E028
:102900004FF000080121204602F0C2FC234640F2AD
:1029100001221E4997F9100001F02AFF10B9204644
:10292000FFF7F8FDB8F1000FDCD00AE0234640F2D3
:1029300001222946022001F01BFF10B92046FFF7B3
:10294000E9FD06B3292D07D03A2D18D12146484676
:10295000BDE8F8430BF048B800232374616839B12F
:1029600091F91030022B03D1204602F063FAF5E70B
:10297000022323742046BDE8F84300F00BB8044955
:102980000320FEF731F9BDE8F88300BF0000FFFF28
:102990001D1201082DE9F047044618B964490320C7
:1029A000FEF722F94FF0FF3102F00FFA0546A0B111
:1029B0008368B3F90260002EF0D0304600F016FDB7
:1029C00043690133014643612046FFF783FDEA680E
:1029D0008B699B1A1844886100E006462746254605
:1029E00095F91030022B08D1EB68282B05D1AB6884
:1029F0001B7803F0F003602B08D0D5F804802F4635
:102A0000B8F1000F6ED04546EAE73C46D5F808809D
:102A1000E368B8F8041049BA89B2994203D2204653
:102A200002F0DEFB0FE022460023D068034492F957
:102A30001000022803D1283B994204D95DE0526876
:102A4000002AF2D1F7E708F118091022394948465F
:102A50000CF0C0FB002855D04846FFF743FD49461F
:102A600000B136B9002000F0E7FA002E08BF064694
:102A700002E0304600F0B8FAB0FA80F040090028D1
:102A800040D008F10800FFF72DFDB0BB4846FFF726
:102A900029FD90BB98F80730013BDBB288F807307E
:102AA0005BB3284602F014FC38B34FF0FF312046E8
:102AB00002F08BF9014610B1204602F0BBF9214625
:102AC0000025084602F004FC18B92846FFF722FD4D
:102AD00013E04168456005460029F2D1BDE8F047A2
:102AE000FFF7D8BDA3681B7803F0F003602B04D177
:102AF000204602F0EDFB074668B92046BDE8F047E6
:102B0000FFF708BD98F80630224639463046BDE842
:102B1000F047FFF7C1BE0222282102F0F3FA87F83E
:102B20001080054600287FF470AF3846E6E700BF06
:102B30001D1201081418010810B5102298B00DEBF1
:102B4000020000210CF012FC504B0593504B082161
:102B50001B88ADF81C3008A8FFF784FC04A90220EC
:102B600002F0BAF840F20523ADF80A3000246846B6
:102B7000FFF775FCBDF802306FF400721344222B8E
:102B8000F5D801A252F823F0152C00081D2C0008DE
:102B9000272C0008272C00086F2B00086F2B00083B
:102BA0006F2B00086F2B00086F2B00086F2B00089D
:102BB0006F2B00086F2B00086F2B00086F2B00088D
:102BC0006F2B0008372C00086F2B0008432C0008DF
:102BD0006F2B00086F2B00087B2C00086F2B000860
:102BE0004B2C00086F2B00086F2B00086F2B000880
:102BF0006F2B00086F2B00086F2B00086F2B00084D
:102C00006F2B0008532C00085B2C0008632C000875
:102C1000732C00080198FFF7BDFEA8E70121019879
:102C2000FFF738FDA3E76FF0850302A96846039319
:102C3000FFF7E4FB9BE7019A537E23F008035376EA
:102C400095E7019800F044FF91E7019800F0CEFF6E
:102C50008DE7019805F024FA89E7019805F076FAE6
:102C600085E7019B587C00F00F0004F063F80474C2
:102C70007DE7019805F0D0FC79E7019A0023194619
:102C8000B2F91A0001F012FB71E700BF0000FFFF6C
:102C9000F40200200121FFF7C9B92DE9F84300F53E
:102CA000E075074628468846FFF7F4FF00244FF0FA
:102CB000380909FB04764146304606F022FA38B15D
:102CC0001022002130460CF051FB0023337402E047
:102CD0000134082CEDD12846BDE8F843FFF7D6B9FA
:102CE00008B5102203490CF075FAB0FA80F04009DB
:102CF00008BD00BFC417010810B5082209490446E1
:102D00000CF068FA48B12378FF2B08D1607800F006
:102D10000F00831E5842584110BD012010BD0020F5
:102D200010BD00BFB41701082DE9FF470026054676
:102D30008846924699463446AF194146384606F0D1
:102D4000E0F900287FD13846FFF7CAFF10B1002C08
:102D500008BF3C463836B6F5E07FEDD12746002C5B
:102D600071D01022414620460CF066FA237884F890
:102D700011A0FF2B84F8109016D0B5F8C631DA07F1
:102D800012D501F0E1F8814670B105F5E0763046E4
:102D9000FFF77CF9B5F9C4014B464A46214601F0DC
:102DA00083F93046FFF776FF98F80030FF2B04D107
:102DB000237C43F00103237441E04046FFF79CFF6E
:102DC0008146C8B9B5F8C62102F00602062A17D115
:102DD00005F5E0763046FFF759F9B5F8C631DB075F
:102DE00006D54B464A464946B5F9C40101F05EFA9C
:102DF0003046FFF74FFF03E0237C63F07F0323742B
:102E0000B5F8C63103F00303012B18D040F2FF22BE
:102E10000023CDE900234FF080730293FF238DF848
:102E20000C3098F80D308DF80D30B8F80E30ADF844
:102E30000E308022002369462846FFF775FF40F2D6
:102E4000112363866463384604B0BDE8F0870388C5
:102E50005BBA23F03F031B041B0C4FF6C062934286
:102E600009D00378FF2B08D1407800F00F00052827
:102E700018BF0E207047052070470E2070472DE9BF
:102E8000F0470025804691461F460C462E464FF0DF
:102E9000010A3FB13A780AFA05F31A421AD0237CA4
:102EA000DB0717D42046FFF71BFF98B94946204699
:102EB00006F03CF937B999F80030FF2B02D0637C5B
:102EC000834207D8B04205D9B8F1000F01D0C8F845
:102ED000004006460135082D04F13804D9D13046AA
:102EE000BDE8F08770B5134CB4F9C451A84206464A
:102EF0001ED0EDB904F5E070FFF7CCFE4FF4A063EF
:102F0000A4F8C831402384F8CA31A4F8C4612B4620
:102F1000A4F8C651802208492046FFF705FF04F5B2
:102F2000E070FFF7B3F82046BDE8704000F06CBEDB
:102F300070BD00BFB02A0020E4170108034BB3F9AD
:102F4000C42182420CBF184600207047B02A0020DE
:102F5000B0F8C631DA0707D511B143F0020301E03A
:102F600023F00203A0F8C6317047B0F8C631DB0782
:102F700001D505F011BB70472DE9F0410D4617460C
:102F80009846FFF7DBFF044610B90020BDE8F0814A
:102F90000029FAD00846FFF7A3FE0028F5D1802FBC
:102FA000F3DC04F5E0763046FFF774FE43463A461C
:102FB00029462046FFF7B8FE04463046FFF766F87C
:102FC0002046BDE8F081000010B520B90548B0F9F1
:102FD000C43133B101E0FFF7B1FFBDE81040FFF7A6
:102FE0005CBE10BDB02A00202DE9F8438946FFF7EA
:102FF000A5FF0446E8B100F5E0763046FFF74AFE4B
:10300000002504EB05084946404606F07AF80746D5
:1030100028B13046FFF73AF84046BDE8F883383526
:10302000B5F5E07FEDD13046FFF730F83846BDE822
:10303000F883BDE8F883000038B5084C0546B4F9BC
:10304000C4011DB9FFF7D0FF20B938BDFFF7CCFF91
:10305000286008B1B4F9C40138BD00BFB02A00200F
:103060002DE9F34102AD00260E4C45F8046D88466B
:10307000074604F5E070FFF70DFE33464246214651
:103080002846FFF7FCFE20B1019B3B60B4F9C44128
:1030900000E004460448FEF7F9FF204602B0BDE810
:1030A000F08100BFB02A0020702C00202DE9F341F0
:1030B00002AC0027884644F8047DFFF73FFF00F587
:1030C000E07506462846FFF7E5FD20463B464246AA
:1030D0003146FFF7D4FE044628461CB1FEF7D6FF62
:1030E000019802E0FEF7D2FF204602B0BDE8F08171
:1030F0002DE9F04F87B00F461546FFF71FFF00F58B
:10310000E073804618460193FFF7C4FD01220021B9
:1031100002A80CF02BF94646C3464FF0FF3A0024B4
:103120004FF001099BF80020FF2A12D05846FFF704
:10313000D7FD70B945B99DF8081009FA04F20A43A1
:103140008DF80820A24604E05846FFF7D5FD002878
:10315000F1D10134082C0BF1380BE3D1BAF1FF3F68
:1031600000F0878004AD2246002128460CF0FEF8CE
:103170003B78FF2B04D197F8019009F00F0309E089
:103180003846FFF7B9FD20B93846FFF760FE0090DA
:1031900001E0022300934FF000094C469DF808100F
:1031A000012303FA04F2114232D039463046B346C5
:1031B00005F0A7FF002855D13046FFF79DFD18B94F
:1031C0003046FFF744FE00E00220009B834208D116
:1031D0002A5D0432D2B22A554A4588BF4FF004090D
:1031E0000AE009D92A5D0232D2B24A4513462A556D
:1031F00038BF4B465FFA83F9B2694AB12A5D0132A2
:10320000D2B24A4513462A5538BF4B465FFA83F976
:103210000134082C06F13806C0D10122002102A891
:103220000CF0A4F800209DF80820014601246E5CF3
:103230004E4504BF04FA01F0024301F1010104BF4D
:10324000D2B201200829F2D108B18DF8082006A8D1
:10325000002340F80C3D3A4602AB4146FFF70FFE13
:10326000DDF80CB0BBF1000F05D1382202FB0A8B50
:1032700001E04FF0000B0198FEF708FF584607B039
:10328000BDE8F08F2DE9F04F8DB005A801F0D8FC16
:103290000026544F03900DF11205B146039B9E4248
:1032A00000F09D8035F9020FFFF748FE0446002824
:1032B00000F0918000F5E07A5046FFF7EBFC012327
:1032C000B5F90000009300220DF1130317218DF8CA
:1032D000139001F0A1FA86302CD09DF91330012B08
:1032E00028D108230DF13008ADF818304FF6FF73E0
:1032F00028F8103DB7F8C631B5F9000043F00303D4
:103300004FF0020BA7F8C631002206AB0521CDF81D
:1033100000B001F0A7FAB5F90000CDF800B0112116
:103320004346002201F078FABDF82010B5F90000FC
:1033300005F0BEFA4FF00808B5F90000CDF800809E
:1033400006AB0022414601F067FA00280FDB424637
:1033500006A90AA80BF070FF4246234908A80BF003
:103360006BFF0023402208A92046FFF7DDFC022363
:10337000B5F90000009300220DF11603112101F0B0
:103380004BFA002806DBBDF81630B3F5A06F28BF56
:10339000A4F8C83100231A462421B5F90000CDF85D
:1033A000009001F039FAB4F8C6310028CCBF43F0E0
:1033B000800323F08003A4F8C6315046FEF766FE72
:1033C00001212046FFF7C4FDB4F8C631DB0702D562
:1033D000204604F02DFE013607F50C775EE70DB0B0
:1033E000BDE8F08FB02A0020B417010808B5FFF738
:1033F000A5FD00F5057008BD2DE9F3410746884697
:1034000016461C460AF0B4FC054640B90323009357
:103410003246A3B2414638460AF03CFC20E0437EE7
:1034200003F00703012B01D103210DE0027EA3B2BB
:103430009A4200F110070CD031462C7622463846CD
:103440000BF0FAFE0321284602B0BDE8F04100F07F
:103450008FBE2246394630460BF0BCFE0028EBD129
:1034600002B0BDE8F08100002DE9F04F1D46D37990
:1034700091B0FF2B8046069116461A9F40F0B4800B
:103480006B78002B40F0B080172F40F2AD802B7A84
:10349000FF2B00F0A98002F1080955491022484687
:1034A0000BF098FE70B105F108014046FFF79CFD56
:1034B0000590002800F098800023183F1C4619460C
:1034C0009A461BE00D224B4906F118000BF082FED4
:1034D000002800F08980E6E70AF1180205EB020BEC
:1034E000AA5C012A0DD0212A08BF5C469BF8012066
:1034F0000AEBC20A1FFA8AFAA7EBC207002FEBDC1D
:103500000BE008AB2A780698009331465B4601F041
:103510000DF8031E68DB5946E8E74046079306911D
:10352000FFF70CFD0699079B18B933490320FDF7F7
:103530005BFB08AA002942D0002C40D0B0F8C6118D
:1035400001F0030103293AD12978029301924B46F5
:103550000A4600943146404604F018FF002304F167
:1035600008020F21074604F0F7FE054617B910229E
:10357000494620E0237A83F002038DF82830637AED
:103580008DF82930A37A8DF82A30E37A8DF82B3024
:10359000237B8DF82C30637B8DF82D30A37B8DF849
:1035A0002E300822E37B8DF82F300AA90EA80BF0ED
:1035B00043FE124908220CA80BF03EFE09E04946E2
:1035C0004046FFF719FF102249460CA80BF034FEC5
:1035D0000025337E0095A3F1FF0253425341059924
:1035E0000CAA404600F0D4FC11B0BDE8F08F00BF3B
:1035F000C4170108F41701081D120108B4170108C7
:103600002DE9F04F89B003F108099246059149462A
:103610001D468046129E0AF0ABFB9AF80730FF2B3E
:1036200040F0B5806C78002C40F0B180172E40F24D
:10363000AE802B7AFF2B00F0AA80002800F0A78034
:10364000183E2746002E27DD07F1180305EB030B74
:10365000EB5C022B0DD0212B16D10023029301939A
:103660002A78CDF800B04B465146404604F08EFE15
:103670000AE006AB00932A7805985B46514600F0B5
:103680009CFF041EC0F283809BF8013007EBC30748
:10369000BFB2A6EBC306D5E74FF0FF31059801F0A6
:1036A00094FB08B1876800E00746494640460AF0A7
:1036B0005FFB064600286AD0437E03F00703022B17
:1036C00012D127B13B7813B17B78002B31D106A9F9
:1036D000A6F81A803476224606F110000BF0ACFDF5
:1036E0002B79590616D512E01FB13B780BB17B78C8
:1036F00013BB002C49D1377E003718BF01272B7927
:103700009A062AD44FB3A4BB2B795B0601D50721B7
:1037100001E01FB10321304600F02AFD95F9043085
:10372000002B737EB4BF43F0080323F008037376C5
:103730002DE0002CCBD12AE02CB3337E9C4209D063
:10374000224606A906F110000BF044FDB0FA80F005
:10375000400900E000200746D1E7002CD4D0A6F8AD
:103760001A803476224606A906F110000BF064FD9B
:10377000CAE7737E03F00703072B08D10321304605
:1037800000F0F6FC03E02746B9E70027B7E709B0E9
:10379000BDE8F08F2DE9F04F87B015469846814679
:1037A0000291109FFFF7CAFBB0F8C6319A07064690
:1037B00069D5EB79FF2B66D198F80140002C62D1D6
:1037C000072F60D905F10803083F0DF1100A039394
:1037D000002F1FDD04F1080308EB030B18F803307A
:1037E000012B0FD198F800200298CDF800A05B467D
:1037F000294600F09BFE031E45DB524603994846CE
:10380000FFF7FAFD9BF8013004EBC304A4B2A7EB69
:10381000C307DDE7B6F8C63113F0040F05F108055C
:1038200028D013F0010F194B194C18BF1C4605F096
:1038300013FE06F5FC7780463846FDF751F9B6F8D9
:10384000C631DB0716D5294648460AF091FA88B1F9
:10385000B8FBF4F140F21523A6F80E320D4BC6F872
:103860001002B3F9003006F5037204FB11813846EB
:1038700008F0E4FC294648460AF07AFA18B1437E7B
:1038800023F00803437607B0BDE8F08F80841E0064
:1038900020A107002C2400202DE9F04F89B092468A
:1038A000059181461E46FFF749FB0AF1080B0546C4
:1038B0000822844958460BF08DFC002840F0FF8018
:1038C0009AF80830FF2B00F0FA809AF80730FF2BA7
:1038D00040F0F5807378002B40F0F180129B0F2BA5
:1038E00040F2ED80594648460AF042FA074650B980
:1038F0000B23009302460346594648460AF0CAF98C
:10390000074668B9DBE0437E190706D5F28852BA4C
:1039100092B212B923F0080301E043F008037B766A
:10392000F3889CB264B15CBA674B68491B88A4B247
:103930001BB207F13002614307F11C0008F07EFC66
:1039400033790BB185F8CA31B5F8C631C3F30D022E
:10395000A5F8C62173791B0203F440431343A5F86D
:10396000C631B068A8B1D5F8D03190FA80F8984542
:103970000FD005F071FD0A22B0FBF2F303FB120039
:10398000053008FB00F0C5F8D081B0FBF2F0C5F8B7
:10399000D401F36813B11BBAC5F8D83105F5E0704E
:1039A000FEF774FB129B103B0393002302930493D6
:1039B000039B002B58DD029B103306EB0308F35CDE
:1039C000052B1CD004D8012B0DD0032B1ED03FE0BB
:1039D000222B2AD0232B3BD14346129A314648460C
:1039E00004F052FE34E006AB00933278059843466B
:1039F000514600F09BFD031E049329DA5FE0424626
:103A00003178484600F013FE10BB58E0424631784A
:103A1000484600F029FE002851D0D8F804301BBADF
:103A2000B3B19C4228BF1C4612E04146307804F0F6
:103A30007FFD002843D0B8F806305BBA9BB23BB19B
:103A40003C22B4FBF2F2934202D23C2202FB03F48A
:103A500098F80130029A02EBC30292B20292039AE2
:103A6000A2EBC3030393A3E7049B06AA5946484667
:103A7000FFF7C2FC05F5EE70FDF732F8B5F8C63178
:103A8000DA071CD504EB4404042C88BFA1084FF0CE
:103A9000000498BF0121384685F8CB4104F030FC82
:103AA0003B463A462146B7F91A0000F0FDFAB5F850
:103AB000C6319B0703D501212846FFF756FA09B006
:103AC000BDE8F08FB4170108F402002040420F0057
:103AD0002DE9F041437E03F00703022B86B0044634
:103AE00001D0052B7BD194F89420B4F91A50012A07
:103AF00071D9022B11D14FF080730493FF238DF8FD
:103B00001430637B8DF8153040F2FF200021E389EB
:103B1000ADF81630CDE902010BE094E8030002ABEA
:103B200083E8030004F1080393E8030006AB03E90C
:103B30000300013A84F894201DBB01AE304601F029
:103B40007FF80746BD4208D036F9150002AB224681
:103B5000002100F0A9FA0135F4E7224B04F1380501
:103B6000B3F900602846FCF7BBFF40F21223A4F82B
:103B70004E3004F14C0233461B49284608F05EFBE8
:103B80002DE02846FFF7DAF90646224602AB06F595
:103B9000E075B4F91A00002100F086FA01212846E8
:103BA000FEF744FA0F4BD6F8D871B3F9008004F150
:103BB00038063046FCF794FF40F21223A4F84E304A
:103BC0003046434604F14C02394608F037FB28469C
:103BD000FEF75CFA03E0214628460AF0F1F806B049
:103BE000BDE8F0812C24002040420F00437E03F00A
:103BF0000703042B03D0072B04D1032100E0052188
:103C000000F0B6BA7047000038B500F5E07504461C
:103C100001212846FEF70AFA05F01EFC0A210A4B8C
:103C2000B0FBF1F202FB11000530C4F8D031434380
:103C3000B3FBF1F3C4F8D431044BC4F8D8312846AF
:103C4000BDE83840FEF722BA80C3C90140420F00E8
:103C500010B5044608462378FF2B14D00022182301
:103C6000872109F02BFF002270B183681A715A7105
:103C70009A71DA7121686268DA609960A168E26815
:103C80005A61196110BD002010BD38B50B78FF2BAB
:103C900005460C46104616D000221823882109F04C
:103CA0000DFF002280B1836825F01F051D71DA71B8
:103CB0009A715A7121686268DA609960A168E26855
:103CC0005A61196138BD002038BD08B500220823AB
:103CD000852109F0F3FE28B1836800221A715A7118
:103CE0009A71DA7108BD10B5002304461046CA1D4A
:103CF00002F0F802194601F0EBF920B18268147065
:103D0000C368DB08537010BDF8B516460F461A4657
:103D1000B11CFFF7E8FF044660B18568C268023550
:103D2000023A002128460BF021FB3246394628464C
:103D30000BF082FA2046F8BD13460A4601460120E0
:103D4000FFF7E2BF13460A4601460220FFF7DCBF39
:103D50002DE9F04180460F4616461D4600221023ED
:103D60008621079809F0AAFE60B1069B846827F0B7
:103D70003F0776BA2DBA1BBA84F804806771E680D3
:103D8000A560E360BDE8F0812DE9F0410746884673
:103D900016462021079A03201C46FFF7A4FF05467C
:103DA000C8B1806824BA0021846028F03F0800F17F
:103DB000100436BA017341738173C173877080F840
:103DC00003804660102220460BF0D0FA3A4606994E
:103DD000204605F0D1F92846BDE8F08110B50A4625
:103DE000044608210520FFF77EFF28B183680022E2
:103DF00024BA9A70DA705C6010BD000008B5102219
:103E000003490BF0E7F9B0FA80F0400908BD00BFA4
:103E1000C417010810B50822094904460BF0DAF965
:103E200048B12378FF2B08D1607800F00F00831E83
:103E30005842584110BD012010BD002010BD00BFE8
:103E4000B417010870B506460846194609F0C0FEC9
:103E50000446A0B18368FF22DA7100231A4619468E
:103E6000184600F003FF054620B92146204600F021
:103E7000E1FF02E083685E804460284670BD70BD4B
:103E8000002101F017BA0000F7B51F46537C802BC4
:103E900005460E46144603D911490320FCF7A4FE3B
:103EA0001046FFF7ABFF08B1002017E02046FFF7F0
:103EB000B1FF0028F8D1217CCB07F5D43388607C92
:103EC000626913F0010F14BF002680268DE8900070
:103ED000A3693143FFF758FF2860012003B0F0BD0C
:103EE0001D12010830B585B0022300930D460DF177
:103EF0000E0300220521044600F08EFC002803DB9F
:103F0000BDF80E30062B10D80823009300222B4654
:103F10000221204600F080FC002802DBADF80E00F4
:103F20000EE00023ADF80E300AE0082300930022D3
:103F30002B460321204600F06FFC0628E4DDEDE768
:103F4000BDF80E0005B030BD38B5002009F05AFFAD
:103F5000044658B1637E03F00703013B012B03D9EC
:103F60000A4B00221A600EE02046EFE7074D286852
:103F700009F048FF034618B909F044FF034610B1A1
:103F80002B60184638BD204638BD00BFE02C00200D
:103F90002DE9F7430A9C0F46994680461646FEF7E0
:103FA000CDFFB0F8C631990701D4002507E040469F
:103FB000FEF7C4FFB0F8C6315A07F6D58025304663
:103FC000FFF71CFF38B11022334930460BF034F9AB
:103FD0000223737001E045F04005B9F1000F0BD0EA
:103FE00069464046FFF77EFF30B1C1B222466846BF
:103FF000FFF7A8FE68B1044624B13B7CDB0758BF3D
:1040000045F02005224639462846FFF73EFE814608
:1040100008B920463BE00146002332464046FFF700
:1040200011FF054608B9484631E03B7CDFF8749043
:1040300013F0010F23D005F00FFA184BB0FBF3F784
:10404000314607FB1307404609F092FE044618B9B3
:1040500013490320FCF7C8FD00F154063046FCF775
:104060003FFD40F20223A4F86A30E566B9F900305A
:1040700004F168023946304608F0E0F809E00146EC
:10408000B9F9000000F0ADFB002802DC2846FFF77C
:10409000F7FE03B0BDE8F083D417010840420F00DB
:1040A0001D1201082C2400202DE9FF4707460D466C
:1040B00090469946FEF742FF824618B92A490320E6
:1040C000FCF792FD35B92A4641463846FFF710F80D
:1040D000054668B102A93846FFF704FF064650B10D
:1040E000C1B2002202A8FFF727FE044620B935E03E
:1040F0000646044600E00446BAF8C631DB0714D58C
:10410000082E0AD00823009300226B44032138466E
:1041100000F082FB80B208281FD1234602AA0F219B
:10412000002004F019F9C0B1044621464046FFF7CB
:104130008FFD064688B101462B464A463846FFF7B2
:1041400081FE044608B9304608E0084B0146B3F941
:10415000000000F046FB002802DC2046FFF790FE3E
:1041600004B0BDE8F08700BF1D1201082C24002018
:104170002DE9F041437E23F007030B430529044654
:10418000437620D0072903D004294BD1264E05E0E1
:10419000B0F91A00FEF7D2FED0F8D461234B04F137
:1041A0003805B3F900702846FCF79AFC40F2172353
:1041B000A4F84E3004F14C023B4631462846BDE897
:1041C000F04108F03BB8B0F91A00FEF7B7FE032340
:1041D0000646224606F5E07584F89430B4F91A00D4
:1041E00023460021FFF760FF01212846FDF71EFF4F
:1041F0000E4BD6F8D871B3F9008004F1380630467A
:10420000FCF76EFC40F21223A4F84E3030464346D1
:1042100004F14C02394608F011F82846BDE8F04197
:10422000FDF734BFBDE8F081404B4C002C2400204A
:104230002DE9F3411B4D002918BF0D4600222946E8
:104240008046FEF755FF074670B169464046FFF7C6
:1042500049FE38B1C1B200226846FFF76DFD044641
:1042600018B91AE0044600E004462046FFF72DFD89
:10427000064688B101463B462A464046FFF7E2FD26
:10428000044608B9304608E0074B0146B3F9000080
:1042900000F0A7FA002802DC2046FFF7F1FD02B08B
:1042A000BDE8F081041801082C2400202DE9F04F0E
:1042B0008BB0002791468A46039302900797FEF73A
:1042C0003DFE964B064600F5E07801214046B94593
:1042D00008BF9946FDF7AAFEB6F8C65115F00105CC
:1042E0001BD1344606F5E377B3465C4500F0ED801C
:1042F000627C9BF811309A4240F0E4805946204697
:1043000004F014FF637C834200F2DC8000E01D4671
:104310003834A045E8D1079D4FE004F06DF905461B
:1043200000284AD0846906F5E37BECB163689E42BD
:1043300018D1AB699C4200F0D780A268996892F8C6
:1043400011E0487C864540F0E380104605930492D6
:1043500004F0ECFE049A059B527C824200F2D88065
:1043600000E01F462468E0E74FF0010B05EBD403A3
:104370009A7D04F007030BFA03F31A420CD0E0B263
:1043800002F0D8FC428A417C0346007C009704F08E
:104390004DFA079060B107460134102CE6D12A4649
:1043A000A98A28693B4604F067FA0546079020B9B8
:1043B0004046FDF76BFE384681E0B6F8C6311B0774
:1043C00007D52946B6F8C801FFF708FD0790F8B1F0
:1043D0000546BAF1000F0FD14046FDF757FE49469A
:1043E00001220298FEF784FE012182464046FDF735
:1043F0001DFEBAF1000F10D008A90298FFF772FD58
:1044000058B1C1B22A4608A8FFF796FC079018B920
:104410004046FDF73BFE3DE00546B6F8C62102F0FA
:104420001004A4B20CB196F8CA4102F020039BB26A
:104430004BB1D6F8D4313A498B4206D84FF47A7B47
:10444000B3FBFBFB03E09B4601E0DFF8DCB002F0CE
:104450004007BFB22FB1D6F8D8714FF47A73B7FBCB
:10446000F3F7039B13B9B6F8CC2100E000224046D5
:104470000392FDF70BFEB6F8C611039A01950912D7
:10448000204600975B4601F0C001FFF761FC04463F
:10449000079008B9284612E0014653464A4602985A
:1044A000FFF7D0FC0146079008B9204607E01D4BF6
:1044B000B3F9000000F095F900282BDC0798FFF70E
:1044C000DFFC27E00BF1380B0FE72B46224639467D
:1044D00007A8FFF7D9FC00283FF41AAF079B002B71
:1044E0007FF415AF28460DE03B46A268594607A861
:1044F000FFF7CAFC00283FF435AF079B002B7FF481
:1045000030AF3846FFF7BCFC4046FDF7BFFD01E089
:104510001B680FE70BB0BDE8F08F00BFE417010880
:1045200000A493D62C24002080EE3600F8B51E4659
:104530009F1C5B780446154613B96FF01500F8BD53
:1045400001F10800FFF75AFC0028F6D17CB394F97A
:104550001030013304D1A3681C78022C04D001E090
:104560006468F3E7082C06D17378012B14D0022B72
:10457000E3D1082411E0853D022D1BD884B972785F
:1045800008236FF0010413FB024402FB036616F8D4
:10459000013D2BB9013CFAE70224853D022D09D8E3
:1045A0002246394606980AF047FE2046F8BD853D6A
:1045B000022DE4D96FF08500F8BD70B51D465B781B
:1045C0000446164613B96FF0150070BD01F10800DE
:1045D000FFF714FC0028F6D1882E27D1A91CA4B11E
:1045E00094F91030013304D1A3681C78022C04D054
:1045F00001E06468F3E7082C06D16B78012B0ED03C
:10460000022BE0D108240BE054B96C78E408023C9A
:10461000E4B20B1913F8013C13B9013CF8E702248A
:10462000224604980AF008FE204670BD70BDF8B519
:1046300017460D46FEF782FC7C78012C06460FD10A
:10464000862D0FD100F5E07521462846FDF7EEFCDA
:104650007B681BBAA6F8C8312846FDF717FD01E0B4
:104660000020F8BD2046F8BD2DE9F0415378042B19
:1046700086B00746154671D186294ED102F1100841
:104680004046FFF7C7FB0646002846D13846FEF7EE
:1046900055FCB0F8C631DA0703D595F90330002B85
:1046A0003BDB41463846FEF79FFC044618B1427C8E
:1046B000AB789A422AD06B6843B31022002102A83B
:1046C0000AF054FEEB785B0616D4AA78414602A89D
:1046D00004F052FDEB78AA7803F0C00302A9384633
:1046E000FEF74AFC0446002839D03846FEF726FC7F
:1046F000012103F051FF09E00821009104AB0022E1
:10470000384600F089F80028DFDA28E06B6833B912
:104710001CB121463846FEF757FC01261FE01BBAA4
:104720006361AA68013312BAA2610CD00E4B6968AA
:104730000E481B8809BA41431BB204F1300204F150
:104740001C0007F07BFD237C23F07F03DBB2237486
:10475000EA7822F03F0213432374DEE70026304656
:1047600006B0BDE8F08100BFF402002040420F0017
:104770002DE9F3410446884617461D4600F0F8FA35
:10478000064650B34146204600F0E0FA711E04464A
:10479000284600F07DFD04B3237A53B1012B17D1D5
:1047A000E068ADF8027000226946019508F062FCED
:1047B00007E0B4F90C10ADF8027068460195FDF7FA
:1047C000CBFD002804DD204600F0E6FA0446E2E7CF
:1047D0000021284600F06EFDF5E7304602B0BDE846
:1047E000F08107B540F20223019101466846ADF819
:1047F0000230FDF7B1FD03B05DF804FB07B540F2F0
:104800000123019101466846ADF80230FDF7A4FD91
:1048100003B05DF804FB000000B589B006930A9B65
:10482000ADF81C304FF401738DF81410ADF816205C
:10483000ADF80630024605AB03A901A80293FDF7C7
:10484000AFFDBDF80E2040F205239A4203D0044983
:104850000320FCF7C9F9049809B05DF804FB00BF18
:104860001D12010800B589B006930A9BADF81C30F3
:1048700040F203238DF81410ADF81620ADF8063081
:10488000024605AB03A901A80293FDF789FDBDF817
:104890000E2040F205239A4203D004490320FCF77E
:1048A000A3F9049809B05DF804FB00BF1D120108CC
:1048B0002DE9F04384680746208F638D8FB000F0A8
:1048C000280EADF818304EF0010E0E4611B96FF0FB
:1048D00015005DE091F91030013354D18D682B79CA
:1048E0002A7813F0C00F03BF02F108035B1995F893
:1048F00001C0294B18BF4FF0020C12B105F108019D
:1049000007E0420747BF04F12E01082204F12C0101
:10491000022294F8360000F1010884F836800490F1
:104920000DF12008BDF81800ADF80800ADF804003E
:10493000CDF80CE0CDF800C0404604F07BFA81468B
:104940000028C4D0304607A900F048FA0646E8B16E
:10495000816881E800032B7913F0C00FBB6815BF95
:104960001A69DA680132013214BF1A61DA60236809
:10497000079A1B682046984700210446304600F0FD
:1049800099FC204604E06FF04C0001E06FF06800F5
:104990000FB0BDE8F08300BFB21701082DE9F04366
:1049A00087683B685C68002387B01A46194638461A
:1049B000A047041E15DD002322461946184600F0C4
:1049C00087FB054668B13B6881685E6822466B4696
:1049D0003846B047B0F1000805DC0021284600F059
:1049E00069FC002466E03E8F06F00206B6B2002E97
:1049F0005BD1A86804F0B2FA044608B9014637E072
:104A00000146C0EB08083246284600F07BFB814691
:104A100008B90146E2E7866801AA04A9304604F015
:104A200013FB01AA044602A9304604F0BBFA002C8D
:104A300001DA00241BE00028FBDBC1B2E3B204AAC8
:104A400002A800F013F906460028F2D0022C0CD17F
:104A50009DF81030FF2B08D19DF81130FF2B01BFBE
:104A60008268137963F07F031371344626B90021FD
:104A7000284600F01FFC1DE0B3689DF801209A71E4
:104A80009DF800205A710D4A12885A8097F82830F4
:104A90002B744946284600F0CDF9002373602B465D
:104AA0005A680AB11346FBE75E604146284600F0AB
:104AB00097FB2C46204607B0BDE8F083F4020020A7
:104AC000034B0360034B436081600020704700BFCD
:104AD000B14800089D490008F0B5254E8468338828
:104AE000838195B00821054604A8FDF7BBFC3088FA
:104AF000204B6360A56000B200F090F82368204668
:104B00009B68984740F2032741F234266846FDF738
:104B1000A6FCBDF80230BB4213D0B3F5017F08D22A
:104B200040F202229342F1D12B680199284698471E
:104B3000EAE70AD0B342E9D123682046DB68984708
:104B4000E2E7236801995E6902E0236801991E6922
:104B50000B894A6809782046B04740F20523039044
:104B600002A96846ADF80A30FDF748FCCCE700BF63
:104B7000F4020020794B000813B50346806879B928
:104B800041F234230190B0F90C10ADF802306846C0
:104B9000FDF7C0FB002822DC12480AF079FD1EE078
:104BA000042919D0072913D0022918D1436898473E
:104BB0000446A0B103460C4990F9100040F20122CE
:104BC000FFF7D6FD014650B9204600F073FB06E022
:104BD0009A6901329A6102E05A6901325A6102B05F
:104BE00010BD00BF641701080000FFFF30B585B09D
:104BF000089C6CB1A5685DB10293074B00930194CA
:104C00000823FCF791F80028D8BF6FF0150001E0E9
:104C10006FF0120005B030BDD94A0008074B10B53F
:104C2000B3F90040A04201D1002010BD14B16FF0D3
:104C30000B0010BD1880FEF755F9F5E7E42C0020B5
:104C4000044BB3F9003013B10380012070471846BC
:104C5000704700BFE42C0020034BB3F900301B1A4F
:104C600058425841704700BFE42C00202DE9F04124
:104C7000174603F108020A440E46002180461D46ED
:104C800008464FF0FF3300F023FA00220446F8B143
:104C900083681E705D705A805A719A711A71B8F1EA
:104CA000000F08D03EB180680278B24203D141467D
:104CB00008300AF0C1FA5FB155B1A0684378AB4241
:104CC00006D1037808332A46394618440AF0B4FA64
:104CD0002046BDE8F081000008B50B7A53B9B1F960
:104CE0000C200B4B53F822301B6A1BB909490320D7
:104CF000FBF77AFFC3B2042B9FBF074B53F820206A
:104D00000A6043F8201094BF00206FF0150008BD22
:104D1000400300201D120108E82C0020C3B2042B20
:104D200011D8094A52F820308B4206D11B6842F84C
:104D300020307047914204D013461A68002AF9D1F6
:104D400001E00A681A607047E82C0020C3B2042B07
:104D500009D8064B53F8200020B143688B4203D09A
:104D60000068F9E770470020704700BFE82C00207A
:104D7000C3B2042B0BD8074B53F8203000202BB1C3
:104D80005A681B688A4208BF0130F8E77047002064
:104D9000704700BFE82C002028B14368006810B1BC
:104DA00042689342FAD1704749B190F91030032B11
:104DB00003D0042B06D103F0F3BF08F08FBE6FF0D1
:104DC000150070476FF00100704728B190F910305E
:104DD0008B4201D04068F8E77047000070B5044688
:104DE0000E4619B912490320FBF7FEFE10B9002048
:104DF000306070BD01460025496801350029FBD1AE
:104E00006FF00103EA00204600F062F90028EED0BE
:104E10008368002BE6D00833A26843F8082CE268C8
:104E2000646843F8042C0833002CF5D1356070BD5C
:104E30001D12010810B504468C42084601D1646871
:104E400008E023465A682AB1904201D01346F9E798
:104E500042685A600021416000F02CFA204610BDE3
:104E600070B5556804460846EDB129464B680BB14C
:104E70001946FBE71CB91A490320FBF7B5FE0028C9
:104E8000F9D0002AF7D043685360844206D0234605
:104E90005E6826B1B04219D03346F9E7144653682C
:104EA0004B60556015E0002CE5D00029E3D0002AC6
:104EB000E1D04B6853608C4206D02346596841B11B
:104EC000884205D00B46F9E7144602E05A60E6E74F
:104ED0005A600021416000F0EDF9204670BD00BF2E
:104EE0001D12010870B503461A4A072B88BF033309
:104EF00010688CBF23F003030823002140B34468EB
:104F0000A34202D901460068F8E7E41A072C0344DB
:104F1000114E05D8046809B9146011E00C600FE067
:104F2000C6F108051D44B5F5C05F02D90021116026
:104F300003E009B9136000E00B60026883E8140025
:104F4000064A9B1B11889BB2994201D2138070BD07
:104F500070BD00BF002D0020042D0020FC2C00207F
:104F600001210148FDF762B804450020204A38B508
:104F7000831AB3F5C05F39D21E4D2C68002324B1CB
:104F8000844202D223462468F9E707298ABF033105
:104F9000082121F003010460141AC1F5C052224413
:104FA000072A98BF891841600BB9286011E05A6838
:104FB00018601A44821A072A0BD818B90E49032020
:104FC000FBF712FE026841681A60C21A0A445A606E
:104FD0001846036853B1426802449A1A072A05D852
:104FE0001A6802601A1A5B681344436038BD00BF38
:104FF000042D0020002D00201D1201082DE9F8438A
:10500000814614200F4616469846FFF76BFF04466C
:10501000D8B15EB13046FFF765FF054638B9204686
:105020001421FFF7A3FF2846BDE8F8833546012386
:10503000C4F80490A560E66084F81080236027B16E
:105040003246394628460AF0F7F82046BDE8F8838C
:10505000F8B50F4D04460026CCB1631BB3F5C05F15
:1050600003D30C490320FBF7BFFD94E88800012B14
:1050700009D1E168A0682660FFF778FF1421204677
:10508000FFF774FF01E0013B23603C46E4E7F8BD15
:10509000042D00201D12010808B5FFF761FF094A21
:1050A000094B1360182100221A705A709A70DA7036
:1050B0001A7159719A71DA710448BDE80840FCF719
:1050C000E5BF00BF002D0020042D00200445002076
:1050D000B2F5C05FF8B505460E4614461F460DD81A
:1050E000FFF73EFF22463B4631462846FFF786FF44
:1050F00004460348FCF7CAFF2046F8BD0020F8BD6F
:105100000445002007292DE9F84388BFCF1C0D4630
:105110008CBF27F00307082704469146FFF720FFBE
:105120002DB124B1E3689D4201D8A3682BB92B4867
:10513000FCF7ACFF0020BDE8F8831420FFF7D2FE97
:1051400006460028F3D0E3689D422ED0AF4202D835
:105150005A1B072A29D82846FFF7C4FE074610B96C
:10516000142130460BE0E068401BFFF7BBFE804691
:1051700040B914213046FFF7F9FE29463846FFF7BB
:10518000F5FED4E72A46A16838460AF055F8E268E9
:10519000A168521B294440460AF04EF8E168A06815
:1051A000FFF7E4FEC4F8088005E0A7689D4214BF3D
:1051B0007B190023A360E36808485B1BE360636816
:1051C00073600123B760F56086F810903360666005
:1051D000FCF75CFF3046BDE8F88300BF04450020C3
:1051E000072970B588BFCE1C04468CBF26F0030685
:1051F00008260D46FFF7B4FE1CB922490320FBF731
:10520000F3FCE368A06813B90028F6D106E0002893
:10521000F3D01D4A821AB2F5C05FEED29D422CD067
:105220002DB930B11946FFF7A1FEA56024E09D42DB
:1052300002D8991B072917D82846FFF753FE0646C0
:1052400020B91248FCF722FF0C2070BDA16829B1DB
:10525000E268AA4228BF2A4609F0EEFFE168A0688A
:10526000FFF784FEA66007E0033323F003039E42AA
:1052700002D23044FFF77AFEE5600448FCF706FFEF
:10528000002070BD1D120108042D002004450020DF
:1052900038B504460D46FFF763FE24B123682B445E
:1052A00023606468F9E70248BDE83840FCF7EEBEC9
:1052B0000445002010B50446FFF752FE2046FFF7D4
:1052C000C7FE0248BDE81040FCF7E0BE04450020E0
:1052D00038B50446FFF744FE0CB1E26822B90E4827
:1052E000FCF7D4FE002038BD2368012B0FD994F9B8
:1052F0001030A1686068FFF781FE054610B1236891
:10530000013B23600448FCF7C1FE284638BD024833
:10531000FCF7BCFE204638BD0445002007B501A8B7
:10532000FFF78EFCBDF9040000F020F903B05DF832
:1053300004FB00002DE9F043082187B08248834C2C
:10534000834FFDF78FF840F20523ADF81230264663
:1053500002A8FDF784F8BDF80A30B3F5017F0AD83A
:1053600040F20322934280F0E68040F20122934211
:1053700000F08780ECE7B3F5106F04D040F601121F
:10538000934273D0E4E7734D05F16C0815F8013CC6
:10539000D3B1D5F81730022B0DD9042B05D8D5F889
:1053A00013302946986900F0F9FAD5F81730023B16
:1053B000C5F8173008E0D5F81390681F01F0ECF835
:1053C0000021484601F076F924354545DED1637861
:1053D000002B43D0238E013B9BB24FF6FD729342CC
:1053E0005D4B02D84FF4004201E04FF000429A6159
:1053F00096F98C30002B20DC96F83730022B18D829
:1054000094F8351051BB94F83430032B07D93C2362
:1054100084F8373084F8341084F835101EE00133F6
:1054200094F82920206A84F8343000F0C3FD032367
:1054300000E0023B84F8373010E0E269002ADBD15B
:10544000218E4FF6FF729142D6D1023B5BB2002B08
:1054500084F88C30D0DC3D4801F0F9F8B7F9003021
:105460003E4A3F493F4806F0E9FE71E703980028AD
:105470003FF46EAF4369002B3FF46AAF06F044FE81
:1054800066E7DDF80C80B8F1000F03D13649032040
:10549000FBF7AAFB02214046FFF797FC4FF0FF31D4
:1054A00005464046FFF791FC002DEFD018B1836808
:1054B000B3F9021000E00146AA68D8F808506B78EA
:1054C000032B33D8DFE803F0020D1D2893885BBA65
:1054D0009BB20093281D02F11803083200F0A0FAD5
:1054E00024E08368587928779B796B7793885BBA37
:1054F0009BB20093281D02F11803083200F0ACFBA8
:1055000014E093885BBA9BB20093281D02F1180344
:10551000083200F0B9FE09E093885BBA9BB20093B1
:10552000281D02F11803083200F008FF0021404650
:10553000FFF7C0FE0CE76FF0850304A902A80593EE
:10554000FCF75CFF04E700BF0C450020E8490020A1
:105550000845002061450020000C02405402002054
:1055600080841E00D04500201D1201087FB51C4C10
:10557000B4F90050064625BB1A4B1B481D701B4B47
:1055800002931B4B00930195082305224FF4806181
:10559000FBF7CAFB208000B316499B2288810320B9
:1055A0004A60FFF799FB00F011FF134A13491448B2
:1055B000B4F9003006F042FE80222946114809F075
:1055C000D5FE0023802210493046FDF7D5FC00208F
:1055D0000D4900F0E3F9B4F9000004B070BD00BF5C
:1055E00008450020C8450020E44500209A1701081E
:1055F000355300084C4500205402002080841E00D2
:10560000D0450020784A00208A170108012380F83D
:105610002F30002380F82C3080F82D3070473C2349
:1056200080F82F30002380F82C3080F82D30704720
:1056300010B5012104460948FCF7F8FC084B18781E
:10564000421C1A7014B140F0800401E000F07F04A5
:105650000248FCF71BFD204610BD00BFCC450020D2
:10566000C845002013B50C4612B11846FFF7E0FFFD
:105670002146022201F0EEF8044678B3002203210D
:1056800080F8252080F82710012314220A2180F8B1
:10569000243080F8262080F8281084F82F3084F8F1
:1056A00032304FF48073238694F83630052043F06F
:1056B000030384F8290084F836303C20094B6085C8
:1056C000F02084F82E00B3F9000001910092082325
:1056D00040F6011204F1380106F03CFD204602B00C
:1056E00010BD00BF084500200021FFF7E3BD10F00A
:1056F000800F4BB202D0002B11DA01E0002B10DB3F
:10570000884204D2C1F1800303440F2B09DD884293
:1057100005D9401A0F28CCBF002001207047002077
:105720007047012070470000F8B5074615461E4631
:105730000C4639B920461949FDF77EFC044608B9E4
:10574000384625E035B916492046FDF7AFFC054639
:105750000028F5D0114A2946002E18BF3246384697
:1057600008F036FA06460028EAD000231A46194601
:105770001846FFF77BFA83680A495C800546466055
:10578000034640F202220220FEF7F2FF20B928462B
:10579000BDE8F840FFF7A8BFF8BD00BF8A170108B1
:1057A000B41701080000FFFF002370B510220C465B
:1057B00019460646FFF78CFC054618B93046FFF738
:1057C00093FF24E0836804221A7000210E225A708D
:1057D0009970A27FDA70E27F1A7194F820205A71D2
:1057E000A269B2F88A2052BADA80A269B2F8882097
:1057F00052BA1A81A269D2F884201288197352BA57
:105800005A8194F821205A73628C52BADA81284660
:1058100070BD002370B520220E4619460446FFF7DE
:1058200057FC054618B92046FFF75EFF1EE080686A
:10583000082303701E2343704023C37033695A69E1
:1058400042609A6982605B7C8370002100F11004E1
:10585000017341738173C1731022204609F086FDE4
:10586000336931465A7C204603F086FC284670BDD9
:105870002DE9F3410F460446002800F0898090F896
:10588000363003F0020300F1080603F0FF0533B1E0
:1058900031460020FFF7BDFF0546002878D094F878
:1058A0003630DB070CD528463146FFF77DFF05462D
:1058B00000286DD094F8363023F0010384F8363098
:1058C00000231A2219462846FFF702FC804608B931
:1058D000284637E0836822781A7094F82E205A7090
:1058E00094F83220022A04D14FF0FF329A70DA7015
:1058F00002E0228E52BA5A8094F8802094F82F1039
:10590000D20042EAC11294F825100A431A7194F8A1
:1059100024205A7100229A71DA713546083304F155
:10592000180E2A4603CA724518605960154603F1DD
:105930000803F6D1042301229B21404608F0BEF85B
:1059400028B9404602B0BDE8F041FFF7CDBE03469E
:105950000022D9685B680A44002BFAD10E4B17B1BC
:105960003978FF290DD1996901319961D9690A44C2
:10597000DA61B4F92C1000963B460022FFF7D4FE02
:1059800006E019690131196159690A445A61F0E761
:1059900002B0BDE8F08100BF784A0020F0B51E4B90
:1059A00085B000220546186803900F460A239B2104
:1059B000104608F083F8064658B380680024047146
:1059C0004471042203A9063009F036FC324623460E
:1059D000D16852680B44002AFAD1104A17B13978BD
:1059E000FF290FD1916B01319163D16B0B44D363CC
:1059F00005B10835002200953B4611463046FFF7B9
:105A000093FE06E0116B01311163516B0B4453633C
:105A1000EEE705B0F0BD00BF9E170108784A0020F0
:105A200030B41948BDF808505BB11978FF2908D087
:105A3000046A01340462446A2C444462052D07D888
:105A400020E0846A01348462C46A2C44C462F5E7AD
:105A50001B780E48FF2B09D143789BB190F8323068
:105A6000022B0FD0383030BC06F05EBB43784BB110
:105A700090F8363043F0010380F83630114630BCE0
:105A8000FFF7F6BE30BC7047784A0020E849002096
:105A90002DE9F04F8BB00026159F07933E600C4612
:105AA000154600F054FF8246002800F0CF80B04633
:105AB0004FF47A7B079B434540F2C8802B78082B34
:105AC00000F2BD80DFE803F0050FBBBB147698BB86
:105AD0004C003B6808F1010843F001033B601FFAEA
:105AE00088F80135E6E73B6843F002033B60A6E037
:105AF0003B6843F010033B6094F8363043F00103F9
:105B000084F83630688940BA80B200F067FC10B182
:105B1000C4F8840003E000F061FCC4F88400E87875
:105B200084F8260095F804E084F827E0697984F881
:105B30002810EB885BBAA4F88A302B895BBAA4F8EA
:105B400088306B7B84F82930EA8984F83900012396
:105B500052BA03FA0EF36285E36384F838106EE0FC
:105B60003B68B4F92C0043F480733B6094F8363002
:105B7000082143F0020384F83630009108AB00227C
:105B8000FEF74AFE002802DAEB785B0657D50822BA
:105B900008A905F1100905F1180009F04DFB0023D3
:105BA000AA78B4F92C004946FDF7E6F9002846D05A
:105BB000A06144E03B68B4F92C1043F020033B6043
:105BC00094F82900638DEA7843430BFB03F3002E1E
:105BD00008BF2E460493802A4FF0010394BF12069B
:105BE00000221498039310230190009202932A1D1F
:105BF000184807F01DFC22E03B6843F040033B607F
:105C00000EB900261BE04FF010096A79638DCDF8BC
:105C1000009053430BFB03F3029395F902300D48B8
:105C2000DB43DB0F0193311D149B102207F088FC2E
:105C3000737802331E443378052BE6D0E1E76B78A6
:105C4000023398441FFA88F81D4433E750460BB0DE
:105C5000BDE8F08FF82300202DE9F04786B0174605
:105C60000022039204460D46BDF83860AD4A5BB190
:105C70001B78FF2B08D0136801331360536833443B
:105C800053601D2E07D849E1936801339360D368B0
:105C90003344D360F5E71E3E03A92078B6B200F086
:105CA000B7FB002800F08F8063885BBA9BB24FF689
:105CB000FF72934200F02F812379DDF80C80C3F34B
:105CC000C20388F88030002000F088FBC8F8840008
:105CD0004DB928469449FDF7AFF9054618B99349DF
:105CE0000320FAF781FF2A46002304F108010398F4
:105CF00000F0BEFB039D06AA05F10808002342F848
:105D0000083D3946404600F0F3FB18B9049B002BD0
:105D100000F00181637885F82E3023790399DB093F
:105D200085F82F30237903F0070385F82530049B8D
:105D3000227E83F82020627E83F82120628852BA76
:105D4000DA8206AB002243F8042D0120019300976C
:105D5000334604F11A02FFF79BFE002800F0DB80B7
:105D6000059810F0100407D1039800F070FC394634
:105D70002046FFF713FED1E0AB6943B94146B5F9C0
:105D80002C00FDF793F9002800F0C580A86140467B
:105D9000FFF73CFC664A95F82730B2F9000095F809
:105DA0002820019295F826200092012202FA03F39E
:105DB00005F1380140F6011206F0CCF9049940468D
:105DC00000F078FCAAE0039D002D00F0A78005F10B
:105DD0000808102204F10801404609F0FBF9814649
:105DE000002840F09B80039A237992F88020C3F327
:105DF000C2039A4240F09280627895F82EA0104635
:105E00005146FFF774FCC8B195F83230012B0FD121
:105E1000130601D5FF2A00E07F2A1ABF0132D2B251
:105E20004A4685F82E2005F1380006F07DF90BE092
:105E300085F82E20404600F01BFC05E01146504638
:105E4000FFF755FC00283DD195F83230012B0BD1DE
:105E500063885BBA9BB24FF6FF72934205F138003C
:105E600032D006F0AAF959E006AA002342F8083D0C
:105E70003946404600F03CFB049B08B9002B4DD04E
:105E80001BB105F1380006F098F9049900293FF498
:105E900026AF237E81F82030637E81F8213063882D
:105EA0005BBACB82404600F005FC049B1A7972B9BC
:105EB00063885BBA9BB24FF6FF7293422ED12A8E53
:105EC0009A422BD005F1380006F02EF926E0EA6957
:105ED000934223D15A7D63799A4202D04046FFF71C
:105EE00095FB049B62795A7523790399DB0985F840
:105EF0002F30237903F0070385F8253006AB002205
:105F000043F8042D012001930097334604F11A024F
:105F1000FFF7BEFD10B9039800F099FB06B0BDE88D
:105F2000F08700BF784A00208A1701081D12010877
:105F300008450020F8B500230C46164619461422E1
:105F40000746FFF7C5F8054618B93846FFF7CCFBFA
:105F500011E0836805221A7012225A7000229A708A
:105F6000DE702146043304F1100251F8040B43F8AB
:105F7000040B9142F9D12846F8BDF8B500230E462E
:105F80001546194606220746FFF7A2F8044618B937
:105F90003846FFF7A9FB0AE0836806221A7004223C
:105FA0005A70ED0100229D70DA701A715E71204600
:105FB000F8BD00002DE9F04F8DB00E460692054663
:105FC000002800F0FD8090F83230012B00F0F880BE
:105FD00021B9C669002E00F0F38005360CA805F142
:105FE00008030024194640F8044D059309940A94C7
:105FF000FDF736F80B9B002B00F0E2800121724880
:10600000DFF8D8B1FCF712F8A04604940394DBF84B
:1060100008309C4268D2DBF8007007EB4417D7E9E0
:10602000022313435ED0BB69DA070CD4039BD3B9B8
:10603000012206991846FFF7A0FF0A9088B9624826
:10604000FCF724F8BCE0049B83B91A46069918466D
:10605000FFF793FF804609900028F0D001230493B6
:1060600004E0012303930DF1280901E00DF1240957
:106070007B699A78FF2A03F1020A07D1D87800F0E9
:106080000F00A0F10E035842584120E008224F496A
:106090000793504609F09EF8079B08B9002016E0C8
:1060A0009A78FF2A04D1DB7803F00F03022BF5D096
:1060B00010224749504609F08DF80028EED01022F2
:1060C0004449504609F086F8003018BF012048B115
:1060D000FA7CD9F800005146FFF72CFFC9F8000000
:1060E0000028ACD0013492E73748FBF7CFFF0A9B7A
:1060F000B8F1000F02D0C8F8043000E00993802204
:106100000B990998FFF716FF04460990002857D00D
:1061100095F90070002F07DA002310220599FEF789
:10612000D7FF0A9030B30990DDF8248000230422C1
:1061300019464046FEF7CCFF04460A9008B940468F
:1061400019E083682A781A70002FB4BF4022002219
:106150005A705A78099062F07F025A7095F833208D
:10616000DA7000279F70022204239B2107F0A6FC0F
:106170000A9018B92046FFF7B7FA21E009900246C5
:106180003B46D16852680B44002AFAD13278FF2A84
:10619000114A0ED0116D01311165516D0B445365DB
:1061A000059BB5F92C10009300223346FFF7BCFA8B
:1061B00006E0916D01319165D16D0B44D365EFE738
:1061C0000DB0BDE8F08F00BF04240020B417010813
:1061D000C417010814180108784A0020F823002089
:1061E0002DE9F7430E4691460446002846D090F923
:1061F0000080B8F1000FACBF0823182303229B21B5
:10620000002007F05BFC0546002837D0876823781C
:106210003B71B8F1000F09DA80237B71102204F181
:10622000080107F1080009F007F801E000237B717D
:10623000002387F80690FB712A46D16852680B4408
:10624000002AFAD10F4A16B13178FF290FD1916F88
:1062500001319167D16F0B44D367B4F92C10083426
:106260000094334600222846FFF75EFA06E0116FDD
:1062700001311167516F0B445367EEE703B0BDE87E
:10628000F08300BF784A00202DE9FF4117460546FC
:10629000BDF82840284A8BB11B78FF2B0ED0136C19
:1062A00001331364536C234453646B7813F0400F31
:1062B0000CBF082318239C423AD306E0936C0133A9
:1062C0009364D36C2344D364EFE7287800F0C2F8DA
:1062D000064668B36B785B0605F1040106F1080811
:1062E00001D4083C07E01022404608F073FFF8B9DB
:1062F00005F11401183C96F83220022AA3B217D0F7
:1063000004AA002042F8040D0097019202200A46D8
:106310003146FFF7BDFB58B195F90130002B04DA87
:10632000EA7839463046FFF75BFF4046FFF76EF9E3
:1063300004B0BDE8F08100BF784A002070B5224A61
:106340000446BDF81000A3B11978FF2911D0116ED1
:1063500001311166516E014451661B78FF2B32D01A
:1063600094F90130002BACBF0823182398422AD19E
:1063700006E0916E01319166D16E0144D166ECE781
:10638000207800F067F80546E8B194F90130002B59
:1063900005F1080602DBE37843B90CE01022211D69
:1063A000304608F017FF0028F5D070BDA27895F8A8
:1063B00033309A4207D1012385F835303046BDE8A5
:1063C0007040FFF72CB970BD784A002008B500F086
:1063D0002DFB014B186008BDF84A0020054B1B68D7
:1063E0000BB900F023BB1A8882420CBF184600206C
:1063F000704700BFF84A002090F83220022A02D1EC
:10640000383005F0D7BE0149FFF732BA8A170108C4
:1064100010B500230E4A0B6054780CB90A6004E0F2
:106420001478844201D10A600FE00B686BB11870D8
:106430000B68012058700B6800224FF48071A3F89C
:106440008A20A3F88810DA6110BD184610BD00BF7D
:10645000E8490020054A53782BB1137883420CBFDA
:106460001046002070471846704700BFE8490020DA
:10647000F8B5044608B1407818B91B490320FAF76B
:10648000B3FB0D4604F1080701F1100E2868696896
:106490003E4603C6083575453746F7D14FF6FF71BE
:1064A00021861249E164142184F82610032184F81E
:1064B00027100A2184F82810052184F829103C218E
:1064C0006185F020002184F8330084F8321084F8CC
:1064D000241084F83410246584F835102462A285D1
:1064E000A3610120F8BD00BF1D120108F963000877
:1064F0002DE9F8430026264F166080460D461446C7
:106500004FF0010917F8013C33B9B9F1000F14D06D
:106510007A1F2260994610E0D7F8133043450CD11A
:106520002946384602F0EDFD38B11A4A242303FB10
:10653000062626600020BDE8F8830136032E07F109
:106540002407DFD1206800B3C0F818802368002238
:106550001A60D8F8143033B11A680AB11346FBE751
:1065600022681A6002E02368C8F814302368012208
:106570001A7123682946053305F1100251F8040BFE
:1065800043F8040B9142F9D10120BDE8F88300BF24
:10659000614500205C45002030B5044687B018B93D
:1065A00020490320FAF720FB85696B6998422AD1BC
:1065B00010221D491D4807F00CF82368D3B10020B4
:1065C000FBF714F922681A4BB0FBF3F0D369B5F965
:1065D0002410181A4FF47A73584305320123039399
:1065E0000192102300220490009202930E4A0F4859
:1065F00006F01EFF6B699C4205D123686B6108E0C1
:10660000944204D013461A68002AF9D101E02268A6
:106610001A6024220021204608F0A8FE012007B0BD
:1066200030BD00BF1D120108C4170108F823002067
:1066300040420F0038B50446406920B10568FFF7B5
:10664000ABFF2846F9E74FF6FF73238538BD10B539
:1066500004460830FFF7EEFF04F1380005F0AAFD0C
:1066600090220021204608F081FE012010BD00008C
:1066700010B5037F013303774369044633B1FFF755
:10668000D9FF102209490A4806F0A3FF228D4FF6D0
:10669000FF739A4208D0238504F1300005F044FDD1
:1066A000A369052283F88C2010BD00BFC417010820
:1066B000F82300202DE9F04F0A4689B00446E1B1E5
:1066C000438C90F821105943D16141698A4214D119
:1066D000B0F9241090F8210043434FF47A704343FB
:1066E00005320493012303930192102300220092A8
:1066F0000293564A564806F09BFE6369228D069225
:10670000002B00F099804FF0010B00226669626156
:1067100092469146002E36D00AF1010A35460027EE
:106720002D6801370DB9D84610E05F45F8D1FAE77A
:10673000B8F1000F0DD12A4635463668013FB9F150
:10674000000F1CD0C9F80050A9461546002FEFDCF9
:1067500001E02DB9EFE7B8F1000F12DD8DB157B1AF
:10676000A2690793D2F884202946D2683046904720
:106770000028079BDFDD2A6808F1FF38DFE7656145
:10678000E2E72E46C6E7B9F1000F01D0C9F8006074
:10679000BAF1010F4FEA4B0BB7DC6269D08A4FF6B2
:1067A000FF71884248D0934223D0A06990F880209E
:1067B000023A012A06D80022591DFFF7FBFB2046AA
:1067C000FEF724FF638C94F82120B4F924102048AC
:1067D0005A434FF47A735343626904930532012399
:1067E000039301921023002200920293174A06F0AD
:1067F0001FFEA3696069D3F8843000215B68984765
:10680000069B2085834203D004F1300005F08CFC08
:10681000606978B1A369228DB3F88810C38AB2FB8E
:10682000F1F2B3FBF1F39A42056801D8FFF7B4FE29
:106830002846EEE763692BB9204609B0BDE8F04F62
:10684000FFF716BF09B0BDE8F08F00BFC4170108FD
:10685000F8230020334BB3F900302DE9F34106460D
:106860000C4615460BB9002058E0002301930B7825
:10687000FF2B0BD14B7803F00F030E2BF3D12146E6
:106880006846FCF7D9FB074608BBECE70822264917
:10689000204608F09FFCA0B12378FF2B04D1637839
:1068A00003F00F03022B0CD010222049204608F0E1
:1068B00091FC30B110221E49204608F08BFC0028C4
:1068C000DDD123780433DBB2012BD8D9CBE7DDF857
:1068D0000080B8F1000FC6D001A93046FFF798FD3F
:1068E0000028C0D00020019EFFF778FDC6F8840084
:1068F00001984FF48073A0F888300023A0F88A3004
:10690000214680F8805043463A46FFF7B1FD0446E1
:10691000019814B9FFF79BFEA5E7006202B0BDE83D
:10692000F08100BF08450020B4170108C417010812
:1069300014180108022380F82A3000218069FEF72C
:1069400097BF002380F82A30303005F0EDBB70B5DA
:1069500000249C422ED21578082D25D8DFE805F0BA
:1069600005242424091319240E000134A4B2013291
:10697000EFE7012822D155780E2D14E001281DD112
:1069800055781E2D0FE0022818D15578122D0BD9FD
:1069900014E0022812D191F880505678012D14BFCE
:1069A00004251425AE4209D1557802352C44A4B2F1
:1069B0002A44CEE70CBF0120002070BD002070BD2E
:1069C000704721B910B94FF6FF707047C18A90F82F
:1069D000202090F8213013446FF0090293FBF2F36A
:1069E000826903F5807392699BB20028A2F888300F
:1069F00008BF4FF4807358188142E4DC80B27047BE
:106A0000C28ACB8A9A4203D38CBF012000207047F0
:106A10004FF0FF30704738B50446FFF7F1FF00280C
:106A2000CCBF0846204638BD70470000004870477C
:106A30005C0200200021FEF73DBC00002DE9F04182
:106A40009EB0102200210AA808F090FC804B0B9306
:106A5000804B08211B88ADF834300EA8FBF702FDEF
:106A60000AA90120FEF738F940F20523ADF81A30E3
:106A700040F2032440F2012504A8FBF7F0FCBDF826
:106A80001230B3F5017F09D8A34280F0D880AB4221
:106A90000CD040F2022293426ED0EDE740F2252264
:106AA0009342E9D1059800F0EDF9E1E7059D28460C
:106AB000FEF70EFC044600287ED00121FEF785F982
:106AC000054608B1C3681BB92046FFF7B3FFCFE7FF
:106AD00083681B78412B11D1FEF7FAFB054600288D
:106AE000F2D001221146FEF70DFB01460028EBD043
:106AF0002046FEF79FF90223044631E003F0D80256
:106B0000C02A03D1204600F0B1FAB1E703F0E00358
:106B1000602BD9D10021022328220846FEF7D8FA9B
:106B2000089010B9089890B9CEE703AB0093002302
:106B300021461A4608A800F0DFFC01460028F1D0E3
:106B400001222046FEF7DEFA014618B90898FFF741
:106B500071FFB9E72046089AFEF782F90023044640
:106B60002B7440F20122234639490220FDF700FE32
:106B700000287FF47DAFA7E7059DEDB1EB68072BFB
:106B80001AD96B68C3B193F91030022B14D128467F
:106B9000FEF79EFB044678B18768B7F9020001F062
:106BA00095FE61688046002619B1CB6849681E448D
:106BB000FAE7B8F1000F01D1284686E798F80430CB
:106BC00023B1204600F086FF70B97DE701231A4605
:106BD0000846FEF77DFA00283FF476AF636843600D
:106BE0006060836841221A70626800231AB1D1681C
:106BF00052680B44FAE7B8F80210994208D32146CC
:106C0000B7F90200FDF7EDFD00283FF731AF5BE774
:106C1000114B596800297FF457AFB6F5006FBFF4E8
:106C200053AF79889A8108A840F2252219805C60C8
:106C30009E60ADF822200993FBF730FB18E76FF058
:106C4000850306A904A80793FBF7D8FB10E700BF4C
:106C50000000FFFFF4020020FC4A00201FB50A4C90
:106C6000B4F9000000280DDC084B029300230193C7
:106C7000074B0093032208234FF480610548FAF77D
:106C800053F8208004B010BD0C4F0020A21701085B
:106C90003D6A00080C4B002038B50E4B142404FB51
:106CA00000340546638A63B10020FAF79FFD0A4B62
:106CB000B0FBF3F0094B53F82530834206D800238C
:106CC0006382637C23F01003637438BD1B1A6382F4
:106CD00038BD00BF0E4F00200087930350500020A6
:106CE0002DE9F041012180461048114DFBF79EF936
:106CF000002426462746E0B2FFF7CEFF2B7C53B197
:106D00004146284602F012FA2B7C834203D8B8424F
:106D100084BF2E4607460134102C05F11405EAD134
:106D20000248FBF7B3F93046BDE8F08190500020EF
:106D30000E4F00200F2838B5044615D801210B4806
:106D4000FBF774F92046FFF7A7FF094B142000FB5F
:106D5000043506482C7C1CB1FBF798F9284638BD51
:106D6000FBF794F9204638BD002038BD9050002034
:106D70000E4F00202DE9F8430F2806468846154699
:106D80001F469DF820903FD8002A40D0012121487D
:106D9000214CFBF74BF9002F4FF0140303FB064384
:106DA00008BF4FF00009802D88BF80225F828CBF12
:106DB0001A741D74B9F1000F02D046F0100300E000
:106DC0003346142000FB064441466374204602F01B
:106DD00098F9014640B91022204608F0C7FA227CF3
:106DE0004146204602F0C8F90020FAF7FFFC0B4BA1
:106DF000B0FBF3F00A4B0744064843F82670FBF754
:106E000045F92046BDE8F8830020BDE8F883104628
:106E1000BDE8F883905000200E4F002000879303B8
:106E2000505000200021FEF745BAF8B50E46017813
:106E30004378174601F10802024405460830FDF781
:106E400015FF0446E0B18368B5F902205A802A791B
:106E50001A716A795A71AA799A71B7424FF0000192
:106E60003A464FF0010328BF32460846FEF730F994
:106E7000054620B92046FFF7D5FF2846F8BD6060DB
:106E80002046F8BD2DE9F04F054685B0B0F9000069
:106E900001F01CFDD5F80480D8F8044083464FF07B
:106EA000000A1CB1E36864689A44FAE7BBF1000F7A
:106EB00005D14046FFF7B6FFC5F804B0D0E0B5F8FD
:106EC0000C90B9F1000F42D1674FAE683B88D8F8FB
:106ED000080001333B80CAEB06039AB2BBF80230CC
:106EE000043B134403F0F8039B1A1FFA83F909F1DA
:106EF00004025146FFF799FF034600283AD0426842
:106F0000D2F808A076BAAAF800609AF8002062F0D9
:106F10003F028AF800203A8852BAAAF80220D8F82C
:106F20000470002F7CD0FA68B9680093C4EB09069E
:106F3000964228BF1646201D344432465044A4B21F
:106F400008F07AF9A145009B6AD97F68E9E7D14545
:106F500080F08280BBF80260D8F80800AF68053E78
:106F600006F0F806C9F10501721D5144FFF75DFFF7
:106F7000034628B96868FFF755FF00236B606FE090
:106F800042689268511D009179BA1180117861F0C0
:106F90001F01117034494F440988CAEB070A49BAE6
:106FA0004FEADA0A518082F804A0D8F80470FFB1E1
:106FB000A1451BD0FA68A11889B2894513D2C4EB48
:106FC00009041FFA84F9C9EB0204B442B9680098B5
:106FD000019328BF34462246494408F02DF9A4B253
:106FE0007F68019B05E07F680C46E0E7002400E035
:106FF0003C46A64214D99FB1FA680193C4EB060837
:107000009045009BB96828BF9046181944444246F1
:10701000A4B208F011F9A642019B01D07F68EAE70B
:107020001946BBF900000093FDF7DBFB0028009B2D
:1070300002DC1846FFF7F6FE002C9BD0AB890395C7
:107040001C44AC8140F2252302A8ADF80A30FBF7BE
:1070500025F9F9F72FFE03E04046FFF7E3FE6C60E9
:1070600005B0BDE8F08F00BF9450002010B58268D5
:10707000137803F0F803C02B044606D0E02B0DD1A3
:107080001379C268DB00053A02E0C2680023043AC3
:1070900060682146806800F013F82046BDE8104083
:1070A000FFF7C0BE002203682BB119689A80DA800E
:1070B0001A600160F7E7436070470021FEF7FAB8F5
:1070C0002DE9F04F8FB081460020924604911F4673
:1070D0008E68AA4DFAF78AFBA94A834605F1900803
:1070E0002C46606858B1A368C3EB0B03934206D9E2
:1070F0000292FFF7E2FF2046FFF7D4FF029A243402
:107100004445EED199F800B009F1080307930BF15B
:1071100008034B44069399F80130029333885BBA15
:10712000C3F30A03059373885BBAADF826300020D9
:107130009BB20A93FAF75AFB002308901C4603936C
:107140006A68A846002A00F02581D2680599914214
:1071500023D1EA8B0A998A421FD12A7F93451CD1F9
:107160006A7F0299914218D15A4607990B9305F10B
:107170000C0008F02FF80B9B78B9029A069905F1DC
:10718000140008F027F80B9B38B97C4C039A242391
:1071900003FB0244089BA3604EE014B96A6802B97D
:1071A0002C463BB1A9689A68521A76498A4294BF24
:1071B000A8469846039B0133042B039305F124054D
:1071C00001D04346BCE784B9B8F1000F03D16E4942
:1071D0000320F9F709FDD8F804000028F7D0FFF7DD
:1071E0006CFF4046FFF75EFF444600210223059AEC
:1071F0000846FDF76DFF6060002800F0DD808368C1
:1072000000210020C3E90001089BA3605A460799AA
:1072100004F10C0008F010F8029A069904F1140029
:1072200008F00AF89DF808306377BDF82630E3834C
:10723000002384F81CB0238425680FBB3379412BCD
:1072400003D105360AF1FF331FE003F0E003602BA2
:1072500006F1040618D10EAB204643F8047D50F821
:10726000042F0093D2680499042300F045F9002804
:107270007CD00D9A28320AEB020306441B1A05E063
:1072800005365346002201E053463A466068C1681D
:1072900003EB070E8E456AD81FFA87FE0EF1FF3109
:1072A000194489B26DB1B5F804804145C0F08280BF
:1072B000B5F806C0E6457DD8C6456FD161456DD1AC
:1072C00078E01FFA83F80EF1FF314144DFF8C0A0E7
:1072D00089B2AC460AEBCC05B5F806B0BBF1000F9D
:1072E00011D1ADB1E98021682960A5F804E0218CB5
:1072F000256080684144174421849A1A31463844F5
:1073000007F09AFF04E00CF1010CBCF1340FE1D15D
:107310006368228CDB689A424ED1637F217F04F13F
:10732000140204F10C00FDF7A1FCF8B18368B9F96F
:1073300002205A8099F804201A7199F806209A714F
:1073400099F805205A710023436063682BB15A688D
:107350000AB11346FBE7586000E0606063680B49C0
:1073600040F201220220FDF703FA10B96068FFF72E
:10737000A4FE2046FFF796FE1EE000BF98500020B6
:10738000C0C62D00FEFFFF7F1D1201080000FFFF99
:1073900028510020002C7FF404AF01E7FFF78DFE99
:1073A0002046FFF77FFE3B46524604994846FFF7CA
:1073B00087FE01E02D6875E70FB0BDE8F08F00BFD4
:1073C000037823F00F0343EA11130370437803F0AB
:1073D0000F0343EA01114170704700000822014980
:1073E00007F02ABFB41701081022002107F0BEBF22
:1073F00010B508220949044607F0ECFE48B123788D
:10740000FF2B08D1607800F00F00831E58425841CE
:1074100010BD012010BD002010BD00BFB417010831
:1074200073B51546194A04460E46106851686B46F6
:1074300003C32CB3637CDB0624D4227C802A1DD0BA
:10744000402A1FD9D208D11F501C2944C2F10F0273
:10745000304407F0BFFEA8B9237CD9080D44725C04
:1074600015F8080C03F0070302A90B44424013F877
:10747000083C1A420CBF0120002004E0012002E079
:10748000204600E0002002B070BD00BFA617010832
:107490000023042A10B54370037016D0082A02D0C6
:1074A000022A26D118E00B7883F0020303704B7890
:1074B00043708B788370CB78C3700B7903714B79F1
:1074C00043718B798371CB7911E00B7883F00203E0
:1074D00003704B7843700223FF240022C470FE2403
:1074E000827004714271CA5C82710B445B78C37113
:1074F00010BD184610BD00002DE9F74F1E464B6821
:1075000000920F46D3F808A0D1F808B0019018B93E
:10751000C0490320F9F768FB019B1B68002BF7D0DB
:10752000DA68272AF4D90BEB06089D6898F9013030
:10753000002B2B7803F00F0343F060032B701BF834
:10754000063003F01803ACBF02240324082B27D015
:1075500017D8002B52D118F804102846FFF730FF37
:1075600008EB04014B7803F00F026B7813436B7048
:107570008978AA78E31C0A43AA7018F80320043417
:1075800029E0102B2AD0182B38D100212846FFF7EC
:1075900017FF6B7823F00F036B700023AB702CE0A8
:1075A00018F804309B099B0043F060032B706B7844
:1075B00003F00F01697018F8043003F00F0308EBB3
:1075C00004020B436B705178AA78A31C0A43AA707B
:1075D00018F803200334EB7813430EE018F8041076
:1075E0002846621CFFF7ECFE6B7823F00F036B70EC
:1075F0000023AB70EB70144600E0EB701BF8063014
:107600005B075CBF18F80430AB711BF8063003F061
:10761000030358BF0134022B08D0032B08D0012BE1
:1076200007D018F80430EB71013403E0402300E088
:10763000FF23EB7198F8013003F0400202F0FF09DC
:1076400072B118064ABF98F802000020000913F032
:10765000300905D0FFF76EFB8146002800F031822B
:1076600098F8013003F07003302B42D00FD8102B64
:107670001CD0202B26D0002B40F08C8008EB04017E
:10768000102205F1080007F0D7FD103482E0502BDE
:107690003BD006D8402B7DD105F10800FFF7A4FEB2
:1076A00078E0602B45D0702B62D073E005F10800C4
:1076B000FFF794FE082208EB040105F1100007F023
:1076C000BBFD34E005F10800FFF788FE4FF0FF3204
:1076D0000023EA746FF001022A752B746B74AB748B
:1076E0006B75022208EB040105F1160007F0A4FDFA
:1076F0003CE0514605F1100011F8082BFFF7C8FED9
:1077000005F10800FFF76AFE44E0B9F1000F3FF40D
:10771000FFAE082208EB040105F1100007F08CFD14
:1077200099F81020494605F1080001F025FD0834BC
:1077300030E0B9F1000F3FF4EBAE4FF0FF32002321
:10774000EA746FF001022A7508EB040102222B741F
:107750006B74AB746B7505F1160007F06DFD99F84D
:107760001020494605F1080001F006FD023411E041
:10777000B9F1000F3FF4CCAE514605F1100011F8FD
:10778000082BFFF785FE99F81020494605F10800FF
:1077900001F0F2FC98F8013059070FD51A064ABFDC
:1077A00098F80200002000F00F0013F00B0F05D036
:1077B000FFF7C0FA8146002800F0838198F8013075
:1077C00003F00F030C2B00F27C81DFE813F00D00B7
:1077D0001600250042007A015100610082000D0070
:1077E0009400A600B800C60008EB0401102205F1C1
:1077F000180007F021FD1034D9E005F11800FFF75B
:10780000EDFD082208EB040105F1200007F014FD4E
:107810003CE000BF1D12010805F11800FFF7DEFD76
:107820004FF0FF32002385F823206FF0010285F826
:10783000242085F8203085F8213085F8223085F81D
:107840002530022208EB040105F1260007F0F4FCC4
:107850003DE09AF800109AF801200831514405F1F2
:107860002000FFF715FE05F11800FFF7B7FD9EE0B9
:10787000082208EB040105F1200007F0DDFC99F86F
:107880001020494605F1180001F076FC08348EE01E
:107890004FF0FF32002385F823206FF0010285F8B6
:1078A000242008EB0401022285F8203085F82130DD
:1078B00085F8223085F8253005F1260007F0BCFC5C
:1078C00099F81020494605F1180001F055FC0234E2
:1078D0006DE09AF800109AF801200831514405F142
:1078E0002000FFF7D5FD99F81020494605F1180052
:1078F00001F042FC5BE005F11800FFF775FDFF2386
:107900002B7618F804306B76611C0522414405F192
:10791000230007F091FC063449E005F11800FFF759
:1079200063FDFF232B7618F804306B76611C03226D
:10793000414405F1250007F07FFC043437E005F1F0
:107940001800FFF751FDFF232B7602236B7618F802
:10795000043085F82730013429E005F1180099F842
:1079600010A0FFF741FD99F81030402B84BF402351
:1079700089F81030FF232B7618F804306B7608EB6B
:10798000040349465B78AB7699F81030EB7699F8AA
:10799000102005F1580001F0EFFB211D04224144A5
:1079A00005F1240007F048FC063489F810A0009B7C
:1079B00013B9FB681B1B01E0009B283B5BBAAB8043
:1079C0001BF806305B077ED518F8043003F0F80387
:1079D000F02B78D1019BBD68D3F800A0009BDAF8AA
:1079E0000890344404F1010815F804B04BB900992B
:1079F000042308220846FDF76BFB002865D0826847
:107A000002E009F1280200200BF00303022B14D03E
:107A1000032B1FD015F808101170012B05EB040380
:107A20009978517004D0D978917005341B790FE0A2
:107A3000DB780434A3F5805318E015F80830A3F57B
:107A400080535BBA13802B19043499789170DB78DA
:107A5000D3700DE015F808301909A1F5756149BA20
:107A600003F00F0302341180A3F575635BBA5380F2
:107A70001BF0040F03D00021FDF71CFC25E02B5D5B
:107A80009371A31C2C446178D17118B1F968083145
:107A9000C91A01E00099283949BA9180112189F861
:107AA00006109288A9F8042018B1019AC0F804A021
:107AB000106053B19C1B0C9B0C9A1B68083313601D
:107AC00001E0002003E0204601E00024F3E703B0DA
:107AD000BDE8F08F2DE9F04F4268D0F80890966825
:107AE000D268002189B0824601230846FDF7F0FAEA
:107AF000029038B38568AB4960232B7006F1080B00
:107B000000236B701022584607F064FB38B15846CA
:107B1000FFF7E6F8804610B1437CD90601D44FF058
:107B20000008337EFF2B00F0628206F11800FFF799
:107B3000D7F80746002800F05A82437CDA0640F165
:107B4000568201E0029858E2B8F1000F04D098F88C
:107B500011301B0703D15FB17B7C1C0708D06B7809
:107B600063F07F036B700023AB70032401E0474692
:107B7000022431683378727821F4704121F0FF01DA
:107B80001B01A9B943EA121313F0FF0F2B7803D19D
:107B900043F018032B7036E043F010032B7073781A
:107BA00031781B09621C43EA01132B5594B22AE079
:107BB0005BB203F030011209114304F101010ED14F
:107BC0002B7843F008032B7032688BB2317812BAED
:107BD0008910C2F3034242EA81122A5509E0134395
:107BE0002B55326889B212BAC2F30342A31C6A54FD
:107BF0009BB2326812BA120AEA549C1C01339BB23F
:107C00000022EA54A4B2B379112B6DD1DAF8043012
:107C1000586883681A88B3F802E052BA92B222F028
:107C20000F0C1FFA8CFC4FF2B0018C451AD19EFA52
:107C30009EF121F00F010904090C614512D10322C4
:107C4000B271598849BA1FFA81FE198849BA89B2B6
:107C50000EEB011101F5AA61197099795970D97962
:107C6000997026E09EFA9EFE0EF47F4EBEF5704F90
:107C700004D10122B2715A8852BA0CE002F47F4258
:107C8000B2F5704F0ED10222B2711A8852BA1A7030
:107C90009A785A70DA789A709A79DA70DA791A7171
:107CA000052206E00022B2719A791A71DA795A71C6
:107CB0000622B17961F00F01C2F1080EB1711A44C8
:107CC000C168C3EB020CCEEB01018C4504D212F863
:107CD0000E1002F8011BF3E7FDF782FA2B7843F050
:107CE00004032B70012303E0621C2B5594B2002384
:107CF0000393F379402B07D0FF2B0AD0012B0CD133
:107D00002B7843F0010302E02B7843F002032B7041
:107D100006E02B7843F00303F9E7621C2B5594B27D
:107D200010222049584607F055FA18B96B7843F0ED
:107D3000400335E0B8F1000F0CD06B7843F04003FE
:107D40006B7098F8112010070AD0AB7843EA021341
:107D5000AB7005E05846FFF74BFB002800F0408170
:107D600008AB0020002163E9040199F80020082AEB
:107D700000F224814FF48A71D140C90740F11E817D
:107D800009F108011846FFF783FBDDE90423716957
:107D90003069994208BF904206D16B7843F03003B6
:107DA0006B7021E0C417010804AA59464046FFF74A
:107DB00037FB0028F1D13369B3F17F4F05EB0400A5
:107DC0006B7840F00381B28A52BA92B2B2F57E4F1C
:107DD00040F0FC8043F020036B70022206F1160194
:107DE00007F02AFA0234A4B2337EFF2B72D16B78EB
:107DF00043F008026A70728BCABBF269BABB328C5C
:107E0000AABB727E022A0FD1326A6AB9B28C5AB901
:107E100096F8262042B943F00B036B7096F82720A2
:107E20002A55631C9CB2B4E0728C8AB996F824205F
:107E300072B943F00A036B70737E2B55601C0322EA
:107E400006F1250115FA80F007F0F6F904349FE0F9
:107E500096F82220002A40F0948043F009036B70CA
:107E6000737E2B55601C052206F123012CE0B38B99
:107E7000ADF81030F38BADF81230338CADF8143010
:107E8000738CADF8163004A8FEF72AFF002878D0CE
:107E9000437CDB0675D5027CF37E9A4271D16B7808
:107EA00043F004036B70437C13F00F031EBFAA78EA
:107EB0001343AB70737E2B55631C9BB2B27EEA54A6
:107EC000A01C042206F1240115FA80F007F0B4F991
:107ED00006345DE01FB199F801303BB951E006F17D
:107EE0001800FFF785FA0028F5D14AE057B16B7802
:107EF00043F004036B707B7C13F00F031EBFAA7862
:107F00001343AB7099F8001099F8012008314944E7
:107F100004A8FFF7BDFADDE90423716A306A9942CB
:107F200008BF904204D16B7843F003036B7030E0DC
:107F300004AA06F118013846FFF772FA0028F2D1B8
:107F4000336AB3F17F4F05EB04006B780FD1B28C2D
:107F500052BA92B2B2F57E4F09D143F002036B7070
:107F6000022206F1260107F067F9023410E043F01F
:107F700001036B70082206F1200107F05DF9083457
:107F800006E02819102206F1180107F055F91034FF
:107F9000A4B2039B1BB1631CB2792A559CB2214643
:107FA0000298FDF71DF9DAF804105046FCF742FF7D
:107FB000029A43685360426001201EE00821B9F92B
:107FC000020000910022FCF727FCDEE643F01003DC
:107FD0006B70082206F1100107F02EF9083402E751
:107FE00028191022594607F027F91034FBE6B8F19A
:107FF000000F3FF4BCAD0027A9E509B0BDE8F08F44
:1080000010B508220949044607F0E4F848B123787E
:10801000FF2B08D1607800F00F00831E58425841B2
:1080200010BD012010BD002010BD00BFB417010815
:10803000F8B5B0F8C631DB07044603D41549032070
:10804000F8F7D2FD00F5E0760121002504F5EE7782
:108050003046F9F7EBFF384684F8CB51F8F740FD8E
:108060004FF40873A4F8F2310B4B0C49B3F900300C
:10807000C4F8F44104F5F872384604F0DFF83046ED
:10808000FAF704F82946B4F9C401BDE8F840FCF752
:10809000CFB800BF1D1201082C2400208096980044
:1080A000F8B5B0F8C631DB07044603D424490320F1
:1080B000F8F79AFD00F5E07601213046F9F7B6FFB2
:1080C00094F8CB31022B03D8013384F8CB3116E07E
:1080D000DD1E01F0C1F90123AB403B2BB0FBF3F5F2
:1080E00005FB13009EBF94F8CB31013384F8CB31EC
:1080F000092804D93C2828BF3C20054600E00A2571
:1081000004F5EE773846F8F7EBFC4FF40873A4F863
:10811000F2310C490C4BC4F8F4416943B3F9003017
:1081200004F5F872384604F089F83046F9F7AEFFE6
:10813000B4F9C4010021BDE8F840FCF779B800BFEC
:108140001D12010840420F002C24002010B50446E7
:10815000B0F91A00FAF7F2FEB0F8C631DA0703D424
:1081600010490320F8F740FD637E1B070BD4002065
:1081700005F048FEA8B9B4F91A00FAF7DFFEBDE829
:108180001040FFF755BF10220749204607F022F89C
:108190000028ECD02146B4F91A00BDE81040FCF7E5
:1081A00047B810BD1D120108C41701082DE9F0439E
:1081B00080468DB01846894614461F46FFF720FFBB
:1081C0000546B8B910230693029308AE07AB079093
:1081D00003900093019706AB32460DF11601474814
:1081E00005F031FA002806DB069B102B0CBF354644
:1081F000002500E000253946204605F0B9FD064679
:10820000002D74D030B93946BDF9160005F0B0FD27
:108210000646E0B1B6F91A00FAF790FE18B1B0F8C8
:10822000C631DA0706D5737E03F03003302B08BF62
:108230003D4600E03D4645B93846FFF7E1FE0028DF
:1082400051D03D46002D3CD00EB1AF4204D029465E
:10825000204605F08DFD06462846FFF7D1FE58B3AF
:1082600026B1737E03F03003202B25D107AE3046B4
:10827000FCF7E6FC0822074689F80020A9184046CA
:1082800006F0DAFF98F8003083F0020388F8003037
:10829000CCB9BC4215D036F91400FAF74FFE48B1FC
:1082A000B0F8C631DB0705D50CAB03EB440434F959
:1082B000140C1FE00134ECE7737E03F03002202A37
:1082C00003D1002016E0204614E003F00703032B3F
:1082D00003D104213046FBF74BFF32464946404666
:1082E00005F0C6FD06E0FBF72FFE0546AAE70028CD
:1082F000A2D08FE70DB0BDE8F08300BFF8230020C7
:1083000070B50E4618B911490320F8F76DFC002925
:10831000F9D0B0F91A00FAF711FE00F5EE7504462F
:108320002846F8F7DDFB4FF40873A4F8F23108494A
:10833000084BC4F8F44104F5F87271432846B3F9C8
:108340000030BDE8704003F079BF00BF1D12010886
:1083500040420F002C240020F8B507460D46164673
:1083600010211A462120FBF7BEFC044660B180684C
:1083700000236DBA0822877043710371C370C580F2
:108380003146104406F058FF2046F8BD2DE9F04F65
:1083900085B080460E9E7578022D0F4692461C468B
:1083A00040F0B8800823009300226B440321FCF7BF
:1083B00033FA0028C0F2AE804046FAF7BFFD2146EE
:1083C0008146404605F0D4FCBAF1870F04464ED0F2
:1083D000BAF1880F40F09E80B9F8C631D90740F154
:1083E0009980DDE90223D6F80CB0D6F808A05B45E9
:1083F00008BF524540F08E80002800F08B80B57891
:10840000012D2ED00BD3022D40F08480404607F181
:10841000080105F0D5FC4846FFF70AFE7AE009F5A9
:10842000E07901214846F9F701FEF6883D4B04F159
:108430003807384676BAB3F90080B6B2F8F750FB81
:10844000394940F21223013EA4F84E3038464346E3
:1084500004F14C02714303F0F1FE4846F9F716FEB1
:108460005BE007F118014046FAF7AEFD52E0B9F8BB
:10847000C6319A074ED0B378002B4BD10837102263
:108480002A49384606F0A6FE002843D0D4B1637EC0
:108490009B060CD5D4F88C20D4F8903052EA030116
:1084A00005D0F168B0688B4208BF824234D1B6F87B
:1084B0000690B9F1000F05D13946404605F080FC21
:1084C0004D462AE0F3882BB384B9032300930F9A17
:1084D000109B3946404605F0DDFB0446E8B13246C4
:1084E00000F18C0352F8080F516803C3637E0E48F5
:1084F00023F0300343F030036376F188094B49BA27
:1085000089B24143B3F9003004F1840204F17000F0
:1085100003F094FE002500E00125284605B0BDE8E3
:10852000F08F00BF2C24002000879303C41701089C
:1085300013B58A784B78402A01D8022B00E0032B30
:108540000ED186280ED1C878CB88C0F300145BBA50
:1085500000949BB2083100F00F00FEF70BFC01E025
:10856000002000E0012002B010BD000008B5014667
:10857000074800F0C6FD48B910220649044806F035
:1085800029FE0028024818BF002008BD004808BD89
:10859000C8520020C417010838B50446E1B10123D0
:1085A00080221449B0F9C401FAF7E6FCA0B104F541
:1085B000E07528460121F9F739FDB4F8C63143F0DA
:1085C0000403A4F8C6314FF4E163A4F8CC31284683
:1085D000BDE83840F9F75ABDB4F8C631B4F9C40162
:1085E000044923F00403A4F8C631BDE83840FAF783
:1085F000EBBC00BF0418010808B510220449054867
:1086000006F0E8FD0028034808BF002008BD00BFB1
:10861000C4170108C85200202DE9F0470024054680
:1086200000F116074FF00109A2464FEAD40804F002
:10863000070617F8083009FA06F633420AD0E0B206
:10864000FEF778FB80F810A017F8083023EA06063A
:1086500007F808600134102CE7D10026AC695CB142
:108660002368AB616368A168B3F9C401FAF7ACFC95
:1086700026606660A660F1E710222146284606F0D3
:1086800075FE2C61BDE8F0872DE9F04F87B003F14E
:10869000080A02905046039117461E46FFF766FFF0
:1086A0000446002800F0B480F3885BBA9AB21AB985
:1086B00042F210738382ABE0DFF860918382103F57
:1086C0004FF00008002F70DD08F11003039AD51851
:1086D000D35C032B02D0222B4AD05EE00298FAF73B
:1086E0002DFC6B780190042B42D105F1100B082270
:1086F0004949584606F06EFD002839D02A7CFF2AE9
:1087000004D16A7C02F00F02022A31D0EA785106C5
:108710002ED413062CD46A6852B359460298FAF73D
:10872000C5FCAA7804905946D9F80800059200F0D3
:10873000FDFC059A824209D8D9F808305B7C9A4240
:1087400004D1D9F80430019A9A4207D0334B986883
:1087500020B11022324906F03DFD48B92F4B5A682E
:1087600032B9019A5A60049A9A60A2691A60A361A8
:10877000AB783F2B6B7801D8022B00E0032B0CD198
:10878000EA7804F11603C2F3C001012002F00702E7
:1087900000FA02F2585C02435A546B7808EBC308A3
:1087A0001FFA88F8A7EBC3078CE773885BBA9BB204
:1087B0002361B28852BA43EA02432361DAF8000027
:1087C000DAF80410234603C356F8100F716802222A
:1087D00003C3002104F1160006F0C8FD0023A361C5
:1087E000A58A104B04F11C0630465D43F8F778F972
:1087F00040F2232363860C4B6463B3F9003004F129
:1088000030022946304607B0BDE8F04F03F016BDF0
:1088100007B0BDE8F08F00BFB41701080053002077
:10882000C4170108008793032C2400202DE9F04190
:108830008846C108064614460831069A22201F467B
:10884000FBF751FA0546A0B18068002164BA0171B6
:108850004171C480867080F80380EA6800F10804E2
:10886000083A204606F082FD32463946204600F09E
:1088700083FC2846BDE8F08170B505460E461446D7
:1088800018211A462320FBF72EFA80B183686ABAB2
:108890002D0C6DBA76BA5A809D80DE8022689A606F
:1088A0006268DA6054F8082F1A6162685A6170BD14
:1088B000054BB3F90020904204D01AB90122188068
:1088C00059801A71704700BF0C530020034BB3F955
:1088D000002082420CBF1846002070470C53002035
:1088E00008B518B907490320F8F77EF9C31C1330FF
:1088F00013F8012F1AB98342FAD1012008BD0020D4
:1089000008BD00BF1D1201082DE9F0410C461546B7
:108910009846064618B926490320F8F765F911B1BB
:10892000CB8A002BF7D02DB1EB8A002BF3D00CB102
:10893000A28AB2BB06F1680718220021384606F069
:1089400015FD5CB12368042B03D06FF06900BDE80E
:10895000F08118222146384606F06EFC06F18007A9
:1089600018220021384606F001FD7DB12B68042B4A
:10897000EBD12846FFF7B4FF18B16FF01500BDE842
:10898000F08118222946384606F056FC24B1E28AC6
:108990000421304605F030FBA6F898800020BDE8A1
:1089A000F081AB8A002BC5D09A42C3D0E5E700BF67
:1089B0001D12010808B5014618B904490320F8F74B
:1089C00013F90420BDE80840FCF7A8B91D120108FE
:1089D0002DE9F04188B090460E461A460E9F044697
:1089E00018B111B1B8F1000F03D12E490320F8F7E7
:1089F000FBF8836E002B50D008AD01A945F8183D57
:108A00002B4605F011FB002849DB0198C368984507
:108A100005D20021FCF74EFC6FF068003FE0042116
:108A2000FCF7D3F90028E0D0D0F8088047B118222D
:108A30002946384606F000FCB8F800305BBAFB82E5
:108A4000D4F88030E3B1B8F80030B4F896205BBABF
:108A50009BB29A4206D001980021FCF72BFC6FF0E4
:108A600046001CE0843410220F49204606F0B2FB79
:108A700030B1102203A9204606F0ACFB0028EAD151
:108A8000019B30469968DA6806F0D6FB0198002110
:108A9000FCF710FC019BD86801E06FF07C0008B087
:108AA000BDE8F0811D120108C41701082DE9F0414D
:108AB0000F4686B090461D46044628B9002B7CD14F
:108AC00042490320F8F790F80AB10029F8D0ADB177
:108AD000EB8A13B96FF0150074E02846FFF700FF2A
:108AE0000028F7D12B68042B5ED16CB1B4F87C2040
:108AF00042B1AB8A33B19A4204D0EBE7D4F880306C
:108B0000002B54D0A36EF3B918220021684606F05A
:108B10002DFC2F4A138803EB03166FEA86466FEA93
:108B200096460133B6B21380ACB1A4F87E6015B995
:108B3000D4F8803000E02B68A3663246042120463A
:108B400005F05AFA07E0182204F168016846B4F803
:108B50007E6006F071FB25B904F18005B4F89640FB
:108B600000E0EC8A009A2B680AB9009301E09A426F
:108B7000B0D10023394642461846FCF7A9FA074609
:108B8000C0B13146224600F025F9014618B93846F1
:108B9000FCF790FB0EE011232A46694605F0A8FA7F
:108BA00000280FDD08380DE06FF069000AE06FF073
:108BB0007F0007E06FF00B0004E0002A88D0002956
:108BC00086D17DE706B0BDE8F08100BF1D12010827
:108BD000125300200021FCF76DBBF8B507468489CD
:108BE0000E46154600204DB900230822B96800F052
:108BF00061FA96F91030022B25D10DE0BD42F3D079
:108C0000B542F1D02346AA89A96800F053FAEB686F
:108C10006D681C44A4B2E6E702194FF6EE739A425F
:108C2000C4BF013080B2B168113420440023202237
:108C3000083180B200F03EFA4FF6FF73984203D03D
:108C4000C04380B2F8BD0020F8BD000070B510220E
:108C500098B000210DEB020006F088FB4D4B059308
:108C60004D4B1B88ADF81C3040F20523ADF80A309F
:108C700008216FF0850308A80393F9F7F3FB04A913
:108C80000420FCF729F86846F9F7E9FBBDF8023043
:108C90006FF400721344032BF5D8DFE803F0023BB6
:108CA0007575019D2846FCF713FB044608B9284654
:108CB00067E00221FCF789F8064618B93749032016
:108CC000F7F792FF606830B190F91030042B02D1B1
:108CD000C368082B06D0042208212046FCF712FAAC
:108CE00000284DD0002385682374EB885BBA9BB2C3
:108CF000002B45D022463146FFF76FFF4FF6FF733A
:108D000098423DD1698849BA234640F2012289B28E
:108D1000042031E0019E304696F91050FCF7D8FA55
:108D2000044608B930462CE0406826460028C5D0E5
:108D300090F91030042B07D0FCF7CAFA0346F8B1BB
:108D4000706040681E46F1E7FCF7C2FAC0B1826865
:108D500070600023C16840680B440028FAD15BBAF8
:108D600093806B1C08BF63680A4908BF93F91050D1
:108D700040F2022223462846FBF7FAFC002882D163
:108D80002046FFF727FF7EE702A96846F9F736FB82
:108D900079E700BF0000FFFFF40200201D12010868
:108DA00010B5044668B161B190F91030042B0BD1B5
:108DB0004268FFF712FF50B1A36840BAD880002084
:108DC00010BD6FF00D0010BD6FF04C0010BD6FF0C6
:108DD000010010BD38B50D461446042308220021B9
:108DE000FCF776F938B1836800226DBA64BA1D8049
:108DF0005C809A71DA7138BD1FB50A4CB4F9003045
:108E000063B9094A0193094B029200930522082392
:108E10004FF480610648F7F787FF2080B4F900001F
:108E200004B010BD14570020AE1701084D8C000887
:108E300014530020F8B504469DF8245025701E46B2
:108E400005F0070310250F46657006989DF8281059
:108E500015460AB1002F68D018B1002E69D13046EE
:108E6000F8BD23B1022B02D00DB9002873D0A17038
:108E700080B39DF82030E37002289DF821302371E3
:108E800004D0082816D0002851D120E002463249EB
:108E9000304606F09FF918B9237823F02003237099
:108EA000637843F008036370737863713378A37158
:108EB000072040E01C236370221D06F1080313F80D
:108EC000011D02F8011F9E42F9D10D2033E005205B
:108ED0001DB9F8BD0320002D3DD0431C9DF81C207A
:108EE00022549DF81D20E2540230022D03D0082D9B
:108EF0000CD0E5B9F8BD637863F07F0363707A78CE
:108F00002254431C3A78E2540230F8BD637863F08F
:108F10003F03637007F10803044413F8012D04F8BC
:108F2000012BBB42F9D10830F8BD3846F8BD00200E
:108F3000F8BD63B90DE075B1BDF81C20BDF8203057
:108F40009A42CAD1237843F040032370CDE7022B25
:108F50008AD1A1708DE7F8BDB2170108427802F0FE
:108F60000C03082B07D00C2B07D0CBB9017849068E
:108F700014D4032302E0072300E00D2312F0C00203
:108F80000CD00178490658BF0233802A01D1981CC1
:108F90007047C02A04D103F1080070471846704793
:108FA0000020704770B501B11AB926490320F7F7C0
:108FB0001BFE437803F00C03082B07D103785C06F3
:108FC00017D5C37813700379537012E00C2B07D1B7
:108FD00003785B060FD5C3781370037953700AE0EA
:108FE00013B16FF0150070BD03785E06F9D403234A
:108FF00002E0072300E00D23447814F0C00411D0F0
:1090000005786D0605D4C65C16705D1C0233455D9F
:109010005570802C08D1C25C4A70034402205B78F2
:109020000B7070BD204670BDC02CDAD1034401F135
:10903000080213F8010B02F8010D8A42F9D1082049
:1090400070BD00BF1D12010808B501B11AB9184959
:109050000320F7F7C9FD437803F00C03082B09D16F
:10906000C37813700379537043794B7083790B7015
:10907000022008BD0C2B0ED1C378137010F8043FEA
:10908000537001F1080310F8012F03F8012D8B42F2
:10909000F9D1082008BD3BB9037813F0400F14BF85
:1090A0006FF01500002008BD6FF0150008BD00BF6F
:1090B0001D120108F0B51AB3DC0705D511F8014BF4
:1090C000013A204492B20133570801EB47054C1C8A
:1090D00003350234AC4207D014F803EC14F8026CE8
:1090E00006EB0E263044F4E71A44D30703D511F8F3
:1090F000173000EB0320030C80B201D01844FAE7CC
:10910000F0BD30B54B68456804680A689D4208BFE9
:10911000944209D1C568CB6884688A689D4206BFBD
:1091200094420120002030BD002030BD30B510B386
:10913000E1B188421CD001380139002210F8015FEA
:1091400011F8014FA54202F1080303D1DAB2802AD7
:10915000F4D10FE085EA0401D8B20B060AD401323B
:10916000D2B249008242C9B2F7D130BD084630BD03
:10917000802030BD104630BD802A28BF8022F8B53F
:10918000D50814462A4606460F4606F055F86307EA
:109190000ED0A4EBC504725DFF23C4F1080403FAEA
:1091A00004F422EA040272557B5D1C40144374559A
:1091B000F8BD10F8013F43B18B42FAD10023037090
:1091C000437813B1013005F07FBC104670470000B2
:1091D0002DE9F04707468AB008B90020A8E0002929
:1091E000FBD000204FF0FF3406462346054631F8F9
:1091F00010E0BEF1000F07D1B3F1FF3F13BF0135FF
:1092000003B201252DB20BE0B3F1FF3F08D0B4F15A
:10921000FF3F01D0B54201DD2E461C464FF0FF3323
:1092200001300828E3D1581C04D0601C7DD0B54221
:1092300002DD7AE0601C03D0012ED8BF4FF0FF346E
:109240003D4800256B46E8464FF03A09AC4203D151
:1092500083F80090A5194EE015B183F80090013312
:1092600011F815E01EF0F00F4FEA450C17D04FEA49
:109270001E1A0EF00F0E10F80AA010F80EE083F878
:1092800001E001EB0C0E83F800A09EF801E04FEA2C
:109290001E1E033310F80EE003F801EC21E0BEF1CE
:1092A000000F10D010F80EA09E460EF802AB01EB96
:1092B0000C0A9AF801A04FEA1A1A10F80AA083F8CB
:1092C00001A073460DE001EB0C0E9EF801E01EF0CC
:1092D000F00F1FBF4FEA1E1E10F80EE083F800E0EB
:1092E00001338C4401359CF801E00EF00F0E10F8AC
:1092F0000EE083F800E0072D03F10103A6DD611CF9
:1093000005D03444082C02BF3A21197001330021E2
:1093100003F8011BC8EB030393423FF65EAF4146DF
:10932000384606F01BFC384602E02E461C4683E712
:109330000AB0BDE8F08700BF241801082DE9F04706
:109340000F46054610B90020BDE8F0870029FAD085
:109350001022002106F00AF83B783A2B04D00024B2
:10936000A1462646A04619E07A783A2A07F1010379
:10937000E9D11F46F3E751462B4806F00FFA98B99A
:1093800051462A4806F00AFA80B1284BC01A40EA32
:109390000616B6F5803FD6D24FF0010917F801AB9B
:1093A000BAF1000FE7D119E01F4BEFE7BAF13A0F1E
:1093B000C9D1B9F1000F05D1B8F1000FC3D105EB48
:1093C0000408EBE7A21C102ABDD8631CDBB2310AEB
:1093D00029558146EE54D4B20646DFE7B9F1000FB5
:1093E00008D0A21C102AAED8631CDBB2310A295562
:1093F000EE54D4B2B8F1000F10D02C44C8EB0408DE
:1094000005F1100201230021434504F1FF3407DC7C
:10941000207802F8010D01332170F5E7102C92D16C
:109420002846BDE8F08700BF241801083518010858
:1094300070B504460D461646F8F7D8F92946821944
:109440002046BDE87040F8F79DB90000014601488C
:1094500002F0F6BD18570020124BF0B593E8340027
:10946000D8681E691C6084EA050122F000424A4067
:1094700082EA420280EA500050405969D86040F3C5
:10948000000782EA802239404A4004EB12249A60A5
:109490009A693E40604044F30004754014405D60AA
:1094A0006040F0BD185700200C4B014618688268D8
:1094B0009368013B002B10B4936005DA9469A342D2
:1094C00008DBCBB20A2B05D01368581C106019704A
:1094D00010BC704710BC06F0B7BD00BF840200206E
:1094E00008B53E20FFF7E0FF2020FFF7DDFF034B2C
:1094F0001B689868BDE8084005F0BEBB84020020E8
:109500002DE9804885B0814600AF0E469246FFF7B0
:10951000E7FFB0460AF1FF340025C6EB0803A3427B
:10952000F5DA844B186841684B68013B002B4B60AF
:1095300004DA06F0B5F8002804DAE8E70B685A1CEC
:109540000A6018780D2801D00A280FD100240D20B8
:1095500088F80040FFF7A8FF0A20FFF7A5FF46455F
:10956000D5D033462246254620462BE0082801D098
:109570007F280DD14645D0D0082008F8015CFFF7C0
:1095800093FF2020FFF790FF08F1FF3B082003E046
:1095900008F1010B88F80000FFF786FFD846BCE70A
:1095A000222913D15C781CB35C2C25D001331C78A4
:1095B0008C42F7D1597820291AD80135197811B37E
:1095C00003F8010B19782029F8D9E9E7272906D1F2
:1095D000E8E74B1C497822290AD02029EDD91C78CC
:1095E0005C2C1946F5D1591C5B780132002BF0D167
:1095F000514806F04DF88AE79C1C9B780132002BFD
:10960000F6D02346D3E7002D81D0AB000E3323F0F4
:109610000703EB46ADEB030D6C464DF825103046C5
:1096200090F800E003460130BEF1000FF8D0BEF123
:10963000220F02D0BEF1270F00D1013344F82130B0
:109640001846013390F800E0BEF1000FF8D1013167
:109650008D42E5D1201FBAB150F8043FA3B119469D
:1096600013F801EBBEF1000FF5D0BEF15C0FF6D19F
:1096700091F800E0BEF1000F04D091F801E001F88C
:1096800001EBF5E7013AEAD12C4B2268FB60C7F801
:109690000890002307F1080151F82380B8F1000F6A
:1096A0000DD10133022B16D0F4E711463B607A60EE
:1096B00006F0EAF87A683B6830B108F10C08D8F88F
:1096C00000000028F1D1ECE7D8F808301BB12146A2
:1096D000284698472CE02168194806F0D5F8054639
:1096E00010BB184A1849194805F048FF184805F0FA
:1096F000CFFF124BC7F80890FB602C4607F1080318
:1097000053F824500DB10C3503E00134022CF5D18F
:109710000EE00C3555F8181C0029F6D055F8142C1D
:109720000A4805F02BFFF4E721680A4805F026FFF8
:10973000DD46ECE684020020461801085C1A0108A8
:109740005F180108641801087018010878180108EA
:10975000263201088218010808B503F011FD002027
:1097600008BD08B5F7F7A2FB002008BD012810B519
:1097700006D10020F8F73AF804460146074805E00C
:10978000486805F0A1F904460146054805F0F6FED3
:109790002046FFF75BFE002010BD00BFEC1A010859
:1097A000121B010808B5FFF757FE0146024805F0F5
:1097B000E5FE002008BD00BF8341010801460628E0
:1097C00014D8DFE800F004060B0D0F11090009485A
:1097D00000E0094805F0D2BE0848FBE70848F9E771
:1097E0000848F7E70848F5E70848F3E7084805F0B0
:1097F000C5BE00BF341B0108381B01083E1B010811
:10980000461B01084B1B01084E1B0108511B010898
:10981000571B0108102828D00BD803281BD003D8C9
:10982000E8B1022815D07047052816D006281AD0AE
:109830007047262815D004D8162818D0202818D00C
:1098400070472A2817D02B2817D0272818D10D4861
:1098500014E00D4812E00D4810E00D480EE00D48F0
:109860000CE00D480AE00D4808E00D4806E00D4800
:1098700004E00D4802E00D4800E00D4805F07EBE12
:10988000704700BFE31B01085C1B01086C1B01084B
:10989000791B01088F1B0108971B01089C1B0108FD
:1098A000AF1B0108C11B0108D61B0108FA1B0108E8
:1098B000051C010808B50146034805F05FFE034892
:1098C000BDE8084005F0E4BE141C0108391C01087D
:1098D00013B5044601A8FBF7B3F920B1BDF90400A4
:1098E000031B5842584102B010BD00001FB504AB25
:1098F000012403F8012D00940022FAF7B3FF002899
:1099000004DA094805F0C4FE20460BE09DF80F106C
:10991000064B074A0748002914BF1146194605F0AF
:109920002DFE002004B010BDC71F0108C41F010890
:10993000D43B0108E31F0108A0F13003DAB2092A81
:1099400004D9A0F16103DAB2052A01D8184670479C
:109950004138C3B2052B88BF4FF0FF30704700007D
:109960007FB50C46082105460DEB0100164604F0B4
:10997000C9FA08B911480FE0009002AB0022214655
:109980002846FAF76FFF00280ADA0D4805F0F6FDC1
:109990002046FFF73FFF0B4805F07AFE01200BE061
:1099A000094805F0EBFD2046FFF734FF3246294613
:1099B000064805F0E3FD002004B070BDFA1F010861
:1099C0006D200108D43B0108832001089120010883
:1099D0007FB5064610460D4605F076F804AB012427
:1099E00003F8010D0022009429463046FAF73AFFA9
:1099F00000280ADA0C4805F0C1FD2846FFF70AFFE7
:109A00000A4805F045FE20460CE0094805F0B6FD81
:109A10002846FFF7FFFE9DF80F200648314605F067
:109A2000ADFD002004B070BD6D200108D43B0108DD
:109A300083200108AA2001087FB506460D4610467E
:109A4000531E13F8014F1CB1303C092CF9D908E022
:109A50000A22214606F0ECFA0390013009D11C4895
:109A60001CE01022002106F0E3FA03900130F6D04A
:109A70000124039BB3F5803FF1D20223009300221F
:109A800003AB29463046FAF7EDFE00280ADA114802
:109A900005F074FD2846FFF7BDFE0F4805F0F8FD00
:109AA000012012E00D4805F069FD2846FFF7B2FEDF
:109AB00031460B4805F062FD039924B1094805F0D1
:109AC0005DFD002001E00848F9E704B070BD00BF6B
:109AD000C32001086D200108D43B01088320010840
:109AE00011210108272101083B220108022808D082
:109AF000FF2808D0054A064B01280CBF184610461F
:109B00007047044870470448704700BF402101086F
:109B10002F210108372101083C21010870B50129D6
:109B200088B00C46164609D104230093002207ABE7
:109B30002921FAF771FE051E0EDA09E0022905D186
:109B4000F9F754FC079008B1012505E06FF0850591
:109B5000154805F09DFD24E0E4B266B11C22002109
:109B6000079805F003FC2046FFF7C0FF01460F48A9
:109B700005F004FD15E02046FFF7B8FF079AD3680B
:109B800051680493936803931369029301911368D6
:109B90000B440093936952690146054805F0EEFCB9
:109BA0003546284608B070BD4821010882210108C9
:109BB000A32101082DE9F04790B002AF002604462A
:109BC000FE70F9F7BBF921460546CB4805F0D6FCF7
:109BD000082300933246FB1802212046FAF71CFEA8
:109BE000061E1CDB06EB460808F1070323F00703FB
:109BF000E946ADEB030D0DF1080AC04805F0BEFCC7
:109C0000334607F108024146504604F04FF9014639
:109C1000BB4805F0B3FCBB4805F0B0FCCD460223C1
:109C20000022009311463B1D2046FAF7F5FD00285F
:109C300003DBB988B44805F0A1FC0223009300229D
:109C40003B1D26212046FAF7E7FD002803DBB988F3
:109C5000AE4805F093FC0223009300223B1D062131
:109C60002046FAF7D9FD002803DBB988A84805F09B
:109C700085FCA84805F082FC082300930022FB180D
:109C800003212046FAF7C8FD061E1EDB06EB460838
:109C900008F1070323F00703E946ADEB030D0DF1CF
:109CA000080A9D4805F06AFC334607F10802414660
:109CB000504604F0FBF80146984805F05FFC9848D0
:109CC000CD4605F05BFC012600E000260223009350
:109CD0000022BB1D10212046FAF79EFD002804DB60
:109CE000B7F906108F4805F049FC012300930022C4
:109CF000BB1C18212046FAF78FFD002808DB8A4894
:109D000005F03CFCB878FFF759FD7E4805F036FCBD
:109D1000012300930022FB1816212046FAF77CFD50
:109D2000002803DB7978814805F028FC4FF0010812
:109D3000CDF8008007EB0803002220212046FAF727
:109D40006BFD002810DBCDF80080FB1C00221F21DA
:109D50002046FAF761FD002806DBFB78434503D176
:109D60007978734805F00AFC6A4805F007FC01237E
:109D700000930022FB1C13212046FAF74DFD00281A
:109D800008DB97F80380B8F1010F03D1694805F0AB
:109D9000F5FB4646012300930022FB1C14212046BC
:109DA000FAF73AFD002808DB97F80380B8F1010FB5
:109DB00003D1614805F0E2FB4646012300930022EF
:109DC000FB1C15212046FAF727FD002808DB97F831
:109DD0000380B8F1010F03D1584805F0CFFB464688
:109DE000012300930022FB1C12212046FAF714FDE8
:109DF000002808DB97F80380B8F1010F03D1504821
:109E000005F0BCFB4646012300930022FB1C1921F0
:109E10002046FAF701FD002808DB97F80380B8F127
:109E2000010F03D1474805F0A9FB464601230093E3
:109E30000022FB1C1F212046FAF7EEFC002808DB5D
:109E400097F80380B8F1010F03D13F4805F096FB66
:109E50004646012300930022FB1C1E212046FAF7F0
:109E6000DBFC002808DB97F80380B8F1010F03D171
:109E7000364805F083FB4646012300930022FB1C75
:109E800023212046FAF7C8FC002808DB97F8038056
:109E9000B8F1010F03D12E4805F070FB4646FDB125
:109EA000B5F8C8112B4805F069FB95F8CA112A4886
:109EB00005F064FBB5F8C631D80702D5274805F090
:109EC0005DFBB5F8C631990702D5254805F056FB6C
:109ED000B5F8C6315A0702D5224805F04FFB0126D6
:109EE0002046FEF7F3FC002840D00379002B3DD03C
:109EF0001D4805F043FB3AE04E2201088522010887
:109F0000952301089D2201085A22010869220108AF
:109F1000752201087D230108812201088F22010892
:109F2000932201089F220108B2220108BB220108E6
:109F3000CF220108E2220108EC220108F6220108E2
:109F4000002301080A230108142301081B23010828
:109F500025230108342301083E2301084623010874
:109F60004C230108522301085C23010816B139482B
:109F700005F004FB0223009300223B1D052120462F
:109F8000FAF74AFC002803DBB988334805F0F6FAF3
:109F9000002D58D0B5F8C6313049314813F0800F44
:109FA000304B08BF194605F0E9FA2A4805F0E6FAF1
:109FB00005F5E07610222C49284605F00BF900281B
:109FC00031D02A4805F0DAFA2822294607F1100094
:109FD000FFF7FEF808B36A7C254807F1100105F089
:109FE000CDFA08222349284605F0F4F838B12B7839
:109FF000FF2B06D16B7803F00F03022B01D11E4813
:10A0000000E01E4805F0BAFA2B7CDB0708D52B7858
:10A01000FF2B0CBF1A481B4800E01B4805F0AEFAA6
:10A020000C4805F0ABFA3835B542C3D1174805F0F6
:10A030002FFB002201212046FFF770FD00220221A4
:10A040002046FFF76BFD114805F022FB3837BD466F
:10A05000BDE8F0877D230108632301083F22010842
:10A060008A23010845220108C41701089823010822
:10A07000A5230108B4170108B4230108BA23010875
:10A08000C1230108CE230108D9230108D43B0108CC
:10A090002DE9F04F012889B0804602AF0E460BDC57
:10A0A00007F10800FAF7CCFD18B1B7F90800FFF77F
:10A0B00081FD002400F06EBC4868431E13F8014F78
:10A0C0003CB3303C092CF9D93168A94805F056FA5F
:10A0D0003068FFF7EFFB3168A64805F04FFA3168AA
:10A0E000A54805F04BFA3168A44805F047FA3168F5
:10A0F000A34805F043FA3168A24805F03FFA3168F9
:10A10000A14805F03BFAA14805F0C2FA012400F08D
:10A1100041BC04F0D9FC05B22846FFF7D9FB002862
:10A1200000F01984B8F1020F04D12846FFF742FD70
:10A1300000F030BC9649B06805F0A6FB002840F05E
:10A140002482B8F1040F01DC30681BE2D6F80C80E1
:10A150009048D6F800903669414605F095FB10B955
:10A16000324602210CE041468B4805F08DFB002869
:10A17000F6D04146894805F087FB28B932460321CD
:10A180002846FFF7EDFBACE34146854805F07CFB34
:10A1900010B93246002151E04146824805F074FB77
:10A1A0000028F6D04146804805F06EFB10B93246D3
:10A1B000262143E041467D4805F066FB10B9324652
:10A1C00006213BE041467A4805F05EFB0028F6D0C8
:10A1D0004146784805F058FB0028F0D041467648C3
:10A1E00005F052FB044610BB304604F06DFC07F14D
:10A1F0001803022223F8100D10210092284622464F
:10A20000FAF730FB002807DA6C4805F0B7F96C481C
:10A2100005F0B4F96B4877E76B4805F0AFF968488B
:10A2200005F0ACF9B7F908206848294607E341462C
:10A23000674805F029FB28B9324605212846FFF773
:10A24000FBFB4EE34146634805F01EFB0446002835
:10A2500063D13146604805F017FB08B9002332E0AE
:10A2600031465E4805F010FB0028F7D031465C48C7
:10A2700005F00AFB08B9012325E03146594805F0ED
:10A2800003FB0028F7D03146574805F0FDFA08B91E
:10A29000022318E03146554805F0F6FA0028F7D0B9
:10A2A0003146534805F0F0FA08B905230BE0314672
:10A2B000504805F0E9FA0028F7D031464E4805F03D
:10A2C000E3FAB8B9062301263B720022009607F193
:10A2D000080318212846FAF7C5FA002812DA474879
:10A2E00005F04CF9387AFFF769FA364805F0D0F9ED
:10A2F00034464FE33146424805F0C6FA0028E1D023
:10A30000404801E72946404805F038F9387AFFF718
:10A3100055FA2C4805F0BCF93CE341463B4805F0B2
:10A32000B3FA10B9324616210EE04146384805F01E
:10A33000ABFA10B93246202106E04146354805F017
:10A34000A3FA28B9324627212846FFF741FBC8E285
:10A350004146314805F098FA0446002840F09780BD
:10A3600031462E4805F090FA002859D1012363E0C8
:10A37000352B010815280108DA280108C82A010828
:10A38000C3260108C82701084A2B0108752B0108BC
:10A39000CA240108882401088D2401089824010892
:10A3A0008F1B0108A2240108971B0108A72401089C
:10A3B000AB240108AF240108B62401086D20010870
:10A3C000AF1B0108D43B010883200108AA20010823
:10A3D000BC240108E4120108C4240108341B01084C
:10A3E000A3290108381B0108AB120108461B01080C
:10A3F000C8240108511B0108CE24010817250108B3
:10A400003E1B0108D6240108362501085E250108F7
:10A41000662501087325010881250108EA23010842
:10A420003146B04805F030FA00289FD03146AE489A
:10A4300005F02AFAC8B900234FF001083B72002248
:10A44000CDF8008007F108032A212846FAF70AFA16
:10A45000002812DAA54805F091F8A54805F08EF815
:10A46000A44805F015F9444694E23146A24805F0A7
:10A470000BFA0028DFD0A14846E6A14805F07EF897
:10A480009B4805F07BF8324629469E48D7E1414675
:10A490009D4805F0F9F90446002872D1304605F0D0
:10A4A000CFFB4FEA500909F1070323F00703EA46FF
:10A4B0000E28ADEB030D83460DF1080801D193483A
:10A4C00006E0102801D1924802E0202804D19148EA
:10A4D00005F054F8002117E0302801D18E48F7E745
:10A4E000402801D18D48F3E7802801D18C48EFE75F
:10A4F0008C4805F043F817E0421C12D04A0800EBE4
:10A50000031008F8020002318B450FD9705CFFF789
:10A5100013FA721878605078FFF70EFA7B685A1CAD
:10A52000EAD1814805F0B4F8012428E0CDF8009084
:10A53000434600222B212846FAF794F9002807DA2F
:10A540006A4805F01BF8794805F018F86948E9E70A
:10A550006B4805F013F8754805F010F82946744863
:10A5600005F00CF84546C144A94505D015F8011B76
:10A57000704805F003F8F7E75E4805F089F8D5461E
:10A5800008E24846FFF796F9C0E56B49B06805F068
:10A590007BF9044600286AD1B8F1030F01D1316874
:10A5A00027E0A8F10308B8F1010FD6F80C9022D0EB
:10A5B0006249D6F800A0484605F066F920B9D6F8F9
:10A5C00010904FF0020A17E05D49F06805F05CF961
:10A5D00020B9D6F810904FF0010A0DE05949F06803
:10A5E00005F052F920B9D6F810904FF0000A03E0B8
:10A5F00051465548ABE182462F2140224846FEF79E
:10A60000D8FD431E802B0646494628BF402607F149
:10A6100008005FFA86FBFEF791FE00283AD0B8F1F9
:10A62000010F07D03B7AFF2B04D1BAF1010F07D0FD
:10A63000464869E5BAF1020F14BF4023412300E008
:10A6400040235A4607F108012846F8F795FC18B947
:10A650003F4804F093FF59E54FF0FF3343618361B6
:10A6600032462B4649463B4804F088FF92E13A497E
:10A67000B06805F009F90446B8B9B8F1030F02D182
:10A680003168364863E1F66807F108003146FEF7A5
:10A6900055FE08B9324837E507F108012846F8F7B2
:10A6A00093FC2A4631462F48C9E02F49B06805F08F
:10A6B000EBF80446002869D1B8F1030F02D13168E4
:10A6C0002A4844E1F06804F0FFF9A0F5A063B3F56F
:10A6D0007B4F06464ED34FF6FF724FF4A0612448DD
:10A6E0009FE000BF89250108C42401086D200108EE
:10A6F000FA1B0108D43B0108341B01088C25010812
:10A7000083200108912001089F260108BC2501082B
:10A71000D9250108F625010814260108322601086A
:10A72000502601086E26010888260108051C01082C
:10A73000A3260108BA260108BF2601080F27010831
:10A740001727010821270108C32601084E27010801
:10A750007A2701089D270108C4270108C827010896
:10A7600029270108EB2701081128010815280108ED
:10A77000302801082846F8F7E1FB08B98848C3E407
:10A78000A0F8C8612A463146864858E08649B06834
:10A7900005F07AF8044670BBB8F1030F17D083496F
:10A7A000F06805F071F8002800F0EA808049F06850
:10A7B00005F06AF8002800F0E6807E49F06805F0B0
:10A7C00063F8002800F0CA80F1687B48BAE04FF0D7
:10A7D000FF0919F0010F04D0224601212846FFF796
:10A7E0009DF919F0020F3FF491AC22460221284650
:10A7F000FFF794F98AE47149B06805F045F804461A
:10A8000000BBB8F1030F02D131686D489FE0F068DA
:10A8100004F05AF9FF28064606D96A484FF6FF7237
:10A82000002104F0ABFE71E42846F8F787FB08B975
:10A83000654869E480F8CA6164482A46314604F0F4
:10A840009DFEA7E0D6F80880614998F80030D6F858
:10A8500000902D2B08BF08F1010840460CBF0026D0
:10A86000012605F011F810B93246132136E0594996
:10A87000404605F009F810B9324612212EE056493B
:10A88000404605F001F810B93246142126E053493C
:10A89000404604F0F9FF10B9324615211EE0504938
:10A8A000404604F0F1FF10B93246192116E04D4937
:10A8B000404604F0E9FF10B932461F210EE04A4934
:10A8C000404604F0E1FF10B932461E2106E0474938
:10A8D000404604F0D9FF30B9324623212846FFF71D
:10A8E00005F8044656E04249404604F0CDFF0446D0
:10A8F00078B92846FDF7EAFF08B93E4804E426B1D6
:10A900000123037129463C481CE0067129463B4857
:10A9100018E03B49404604F0B7FF0446A8B9284672
:10A92000F8F70CFB10B93748FFF7EEBB2EB1012149
:10A93000F8F71BFB2946344804E03146F8F715FBCD
:10A940003248294604F01AFE24E03148494604F012
:10A9500015FEFFF7DBBB2F48FFF7D6BBB8F1040F9E
:10A960000AD04FF0020905222B49306905F0D6F9CB
:10A97000B0FA80F464092CE704464FF0020930E78E
:10A980004FF0FF0901E04FF00109B8F1040FEAD1DF
:10A99000002421E720461C37BD46BDE8F08F00BFEC
:10A9A0005828010872280108952801083C2101084F
:10A9B0009B2801085C1701089E280108D728010878
:10A9C000DA280108F428010822290108422901088F
:10A9D0006B290108732901087B29010883290108D3
:10A9E0008B2901088F290108942901089C29010855
:10A9F000A9290108AE290108CC290108F329010879
:10AA00001B2A0108232A0108572A01088F2A010856
:10AA1000C82A010816240108C82401082DE9F04FAE
:10AA200087B006AF0546884691469A4605F008F974
:10AA300028448542A0EB050413D010F801392F2BD0
:10AA400005D1601C284404F03FF806460BE03A2B81
:10AA500001D02E2BEDD1284605F0F2F80026044651
:10AA600001E00024264604F1080323F00703ADEBC0
:10AA7000030D0DF1180B621C0021584604F076FC02
:10AA800029462246584604F0D7FB404605F0D8F840
:10AA900059461648FEF752FCD0B1144D10244146D9
:10AAA0001348FEF74BFCD0B1114B102200213606A3
:10AAB000039102920193CDF810A0009623462A46F6
:10AAC00049460C4802F0B4FC0437BD46BDE8F08F9F
:10AAD00004F002F86A230360074D0424DFE703F063
:10AAE000FBFF6A2303600422044BDFE74457002086
:10AAF00034570020F82300205857002054570020D6
:10AB000001282DE9F34105460C4603D17A4802F0AD
:10AB100039FEBBE002281AD14968784804F0B4FE37
:10AB2000002800F0B1806168754804F0ADFE08B9F6
:10AB30007448B8E06168744804F0A6FE014620B984
:10AB40006D4802F064FD7148ADE07148ABE053DD43
:10AB500049686A4804F098FE58B16168684804F092
:10AB600093FE30B16168684804F08EFE08B1694810
:10AB700099E0032D25D16168634804F085FE054600
:10AB800090B9A06803F0A0FF04B22046FAF764F879
:10AB9000214628B1584802F03AFD21465E4800E0BF
:10ABA0005E4804F0EBFCA2E0A1685D48FEF7C6FB3E
:10ABB000054600286CD0102259494F4802F009FD83
:10ABC00064E0052D18D161684C4804F05DFE002852
:10ABD00068D1E168534804F057FE0546002861D16A
:10ABE00001A8FAF72DF8012831D14FF0FF33BDF954
:10ABF00004202169A0683DE0072D3ED161683F48EF
:10AC000004F042FEC8B9E168464804F03DFEA0B930
:10AC10006169454804F038FE054670B901A8FAF7A5
:10AC20000FF8012813D1A069BDF90480A66827692F
:10AC300003F04AFF424603461AE061682F4804F0D9
:10AC400023FE20B9E168374804F01EFE08B13748FA
:10AC500029E06169364804F017FE05460028F6D160
:10AC6000A069A668276903F02FFF4FF0FF3302B2F7
:10AC700039463046FFF7D2FE39E0092D12D161681E
:10AC80001E4804F001FE90B12A480CE000252EE099
:10AC900003F022FF6A23036004222749164802F0CA
:10ACA00098FC24E0254804F0F3FC01251FE0E1684E
:10ACB0001C4804F0E9FD0028E6D161691C4804F055
:10ACC000E3FD0028E0D1E169174804F0DDFD054609
:10ACD0000028D9D1A069A668276903F0F5FE80464F
:10ACE000206A03F0F1FE0FFA88F20346C0E7284617
:10ACF00002B0BDE8F08100BFF8230020BF260108A4
:10AD0000C42701088F2D0108232E0108292E0108D0
:10AD10004A2E0108C72E0108172F01084B2F0108E2
:10AD200044570020692F0108DF3001086D2F01080A
:10AD3000E8300108AF2B010858570020EC3001081B
:10AD400013B5044601A8F9F77BFF20B1BDF9040053
:10AD5000031B5842584102B010BD000000F007002C
:10AD6000072813D8DFE800F00406080A0C0E1210BA
:10AD700008480CE008480AE0084808E0084806E0EF
:10AD8000084804E0084802E0084800E0084804F0E9
:10AD9000F5BB00BF3C3101084931010856310108BB
:10ADA00063310108703101087D3101088A310108E1
:10ADB0009731010800F03000202805D0302805D058
:10ADC000102805D1044804E0044802E0044800E0EB
:10ADD000044804F0D3BB00BFA4310108A731010827
:10ADE000AC3101084C320108F0B5012893B0064699
:10ADF0000D4607D16B4804F04BFC6B4804F048FC4F
:10AE0000002005E04968694804F03EFD30BBF1E7E9
:10AE100002F0E0FF0446002800F0C180282221460D
:10AE200008A8FEF7D5F9237EB4F91A60054604F1A7
:10AE30001002182102A803F039F8324603462946C9
:10AE40005B4804F09BFB607EFFF788FF607EFFF7A6
:10AE5000B1FF584804F01CFC2046D9E7012E40F30E
:10AE60009680022E74D06968534804F00DFD0446A4
:10AE7000002857D1023E012E02D0022E0CD022E033
:10AE800008A8F9F7DDFE012898BFBDF92060AF687A
:10AE900088BF264600251CE0AF6808A83946FEF7A3
:10AEA0004DFA28B9A86803F00FFEEF6806B2F1E783
:10AEB00002A8F9F7C5FE012898BFBDF90860ED6842
:10AEC00088BF264605E0A86803F0FEFDEF682D69FF
:10AED00006B23046FFF734FF08B9384805E0394676
:10AEE00008A8FEF72BFA20B9354804F0D1FB01245D
:10AEF00055E04DB108212A460DEB010003F002F8A0
:10AF0000034610B92F48F0E72B460022009208A90B
:10AF100002AA304602F0BEFE08B92B48E5E73946E2
:10AF20002A4812E069682A4804F0AEFC044678B961
:10AF3000AD6808A82946FEF701FA0028D4D008A970
:10AF4000204602F03DFF2348294604F017FB26E087
:10AF50006968214804F098FC0446C0B902F03AFF41
:10AF60002146054655B119B1B1F91A0002F028FF82
:10AF7000284602F02FFF29460546F3E719B1B1F93B
:10AF80001A0002F01DFF154804F0F8FA07E02B68DC
:10AF900000931A461946124804F0F0FAA7E7204633
:10AFA00013B0F0BDB0310108FF310108EA19010802
:10AFB0004E320108D43B0108BF2601086332010864
:10AFC0002927010883320108AE320108DE32010868
:10AFD000C427010810330108C824010839330108C7
:10AFE0005833010870B501288AB00C460DDD486859
:10AFF00003F06AFD05B22846FFF7A2FE30B92168CA
:10B00000164804F0BBFA012025E00025144804F09E
:10B010003FFB144804F03CFB002002F0F3FE044622
:10B02000C8B1B4F91A600DB1AE4212D1282221463E
:10B030006846FEF7CDF8314602460B4804F09EFA0A
:10B04000607EFFF78BFE607EFFF7B4FE074804F0DA
:10B050001FFB2046E1E70AB070BD00BF04340108C1
:10B060001D3401081A32010851340108D43B01088B
:10B0700008B501460B4804F081FA0B4804F008FBC0
:10B080000A4804F005FB0A4804F002FB094804F0F2
:10B09000FFFA094804F0FCFA0848BDE8084004F04B
:10B0A000F7BA00BF5F340108BB340108C53401089A
:10B0B000D33401082D350108413501085235010806
:10B0C0000C4AF0B514880830260AE5B200238B42FA
:10B0D00009D2FF2C85BFC718C654C5547D708CBFDC
:10B0E00002330133F3E781BF138809181B0A01F803
:10B0F000013CF0BD800200202DE9F0430D4685B0F3
:10B1000002210446F9F761FE032107462046F9F7BC
:10B110005CFE07B108B9274845E08668264AB3882F
:10B12000F48812885BBA9BB264BA9A42A4B239D14D
:10B130002249234B0A881B889A4203D9944203D39D
:10B14000012307E0944204D39C428CBF00230123D7
:10B1500000E0002333B3BF68D0F80C901948944244
:10B1600098BF013207F1080898BF0A80282241469B
:10B17000FEF72EF84FF47A72B388B5FBF2F102FBBA
:10B18000115502910395FA7901925BBA02469BB27E
:10B19000494600940C4804F0F1F9404602F03AFEAA
:10B1A000012003E0094804F073FA002005B0BDE86F
:10B1B000F08300BF6D350108800200208457002015
:10B1C000865700205C570020A4350108E7350108A8
:10B1D0002DE9F04F99B081460C461022002114A8A9
:10B1E00004F0C4F881231593994BB9F1010F1B8822
:10B1F000ADF85C303BDDB9F1020F00F0C281606850
:10B2000003F062FC051ED4BF4FF000084FF00108A8
:10B2100008F101034FEA830754F82330089308F13B
:10B220000203D8BF0325994505DDE319586803F0EB
:10B230004BFC049001E00423049308F103039945B7
:10B2400005DDE319986803F03FFC064601E04FF482
:10B250007A7608F10408C14505DD2744F86803F053
:10B2600033FC099000E00995049B002B03DA206869
:10B27000FFF7FEFE3FE04FF0FF3225210898FDF773
:10B2800098FF04B2621C089910A808BF0024FEF7BA
:10B2900055F808B96F482CE008226F4910A803F050
:10B2A00099FF50B19DF84030FF2B05D19DF84130FA
:10B2B00003F00F03022B00D0A4B10EA8F9F7C0FCD5
:10B2C00044B1002800F05881BDF938309C4240F06C
:10B2D000538106E0012802D1BDF9383001E05F4812
:10B2E00007E01C4614A90320F9F7F6FC002804DA4D
:10B2F0005B4804F0CDF901204BE1F5F77BFB4FF4FF
:10B300007A7373430D9300220023CDE90A010027CD
:10B31000CDE906234FF0FF332E460593BA46BB46D0
:10B32000013E731C4F4A00F006814E4B19884E4B6C
:10B330001A88013292B21A80049B00938020002365
:10B3400002F0E6FB804698B104998068FFF7B8FEEA
:10B3500010AA0021404602F03BFC814640B1ACB14E
:10B360004FF0FF3308220021F9F7B2FE814618B9E9
:10B370003E4804F08DF9D3E7836800221A705A70B2
:10B380005A719A711A715A8083685C800020F6F7AE
:10B390002DFA4B46804640F2022235490220F9F749
:10B3A000E7F90C9038B9334804F072F90C99484623
:10B3B000F9F780FFB4E7304A00230EA800F058FFE9
:10B3C00000282DDBBDF83A2040F201239A4220D11B
:10B3D0000020F6F70BFADDF83C90C8EB0008414678
:10B3E0004846FFF789FE002183444846F9F762FF8B
:10B3F000059B474538BF4746434528BF434605930D
:10B40000DDE9062312EB080243F10003CDE9062330
:10B410001AE00F4B19880EA809B2F6F77BFF13E06C
:10B42000164804F035F90FE00EA8F7F715F80028D4
:10B4300028DDBDF83A304345F6D1114804F09EF8B6
:10B4400000210F98F9F736FF40F20128ECE700BF22
:10B45000F402002004360108B41701081D36010863
:10B460006B3601088002002086570020582401080E
:10B470000000FFFF8B36010840420F00B63601087E
:10B48000C33601081EB100210D9800F0ADFE099BE6
:10B490000AF1010A534502D0002E7FF441AFF5F7BF
:10B4A000A9FA089980463C4804F068F8BBF1000FFF
:10B4B000C6EB050A38DD5246DDE90601D31703F075
:10B4C00077F9DDE90A23B8EB02029046334AB8FB6C
:10B4D000F2F1642302FB11828DE806000C905A46BB
:10B4E000514603FB0BF32E4893FBFAF3C3F16403BD
:10B4F00004F044F84FF47A72B7FBF2F002FB107ECE
:10B5000001900C980C9BB3FBF2F302FB130000902C
:10B5100005980599CDF808E0B1FBF2F102FB1102A4
:10B52000204804F02BF803E051461F4804F026F8A9
:10B530004FF0000AF4E61D4B00211980138814A96E
:10B54000013303201380F9F7E9FB40F201240EA830
:10B55000F6F782FF00280BDDBDF83A30A342F6D1A2
:10B56000134804F00BF800210F98F9F7A3FEECE75D
:10B57000BBFA8BF040090CE021460E4803F0FEFFB9
:10B58000B9E66368089304274FF000080325049781
:10B5900053E619B0BDE8F08F0837010840420F00AC
:10B5A000243701086D370108A137010886570020AC
:10B5B000C3360108D83701089368013B002B10B44B
:10B5C000936008DA9469A34202DBCBB20A2B02D162
:10B5D00010BC04F039BD1368581C10601970C8B253
:10B5E00010BC704710B503F06FFA04B22046F7F7AD
:10B5F000A5FC20B9064804F04BF8012010BD2046F8
:10B60000F9F7B4FF2146034803F0B8FF002010BD4E
:10B61000FE3701081A38010830B58FB00D4603F027
:10B6200053FA2946C4B26846FDF788FE18B90E4899
:10B6300004F02EF810E000231A4669462046FAF777
:10B6400011F858B92822694604A8FDF7C1FD224621
:10B650000146064803F092FF012003E0044803F08E
:10B660008DFF00200FB030BD483801081C160108BE
:10B670004E16010810B503F027FAC4B22046FAF7B7
:10B68000E9FE10B92146084804E0FAF7E0FF214638
:10B6900020B9064803F072FF012010BD044803F0F2
:10B6A0006DFF002010BD00BF77380108A0380108E9
:10B6B000C738010830B58BB003F006FAC5B228468A
:10B6C000FAF7C8FE044620B90A4803F0E1FF01205A
:10B6D0000EE0383000F028FD282204F10801684609
:10B6E000FDF776FD2A460146034803F047FF002098
:10B6F0000BB030BDE73801080F39010830B58BB009
:10B7000003F0E2F9C5B22846FAF7A4FE044620B9D0
:10B710000A4803F0BDFF01200EE0383000F04AFD7A
:10B72000282204F108016846FDF752FD2A46014629
:10B73000034803F023FF00200BB030BDE7380108B9
:10B740004E39010870B58CB003F0BEF9C6B2304670
:10B75000FAF780FE0125044620B9134803F098FF4C
:10B7600028461EE0114A90F82730B2F9000094F8FC
:10B770002820019294F82620009205FA03F340F65F
:10B78000011204F1380100F0E5FC282204F108015F
:10B7900002A8FDF71DFD32460146054803F0EEFE06
:10B7A00000200CB070BD00BFE7380108084500203C
:10B7B0008F39010808B504490020FAF7EFF803486B
:10B7C00003F066FF002008BD8A170108D039010880
:10B7D00013B5234C234803F05BFFA3690093226950
:10B7E000A3682168204803F0C9FEE36900936269F9
:10B7F000E36861681D4803F0C1FEA36B0093226BF0
:10B80000A36A216A1A4803F0B9FEE36B0093626BE6
:10B81000E36A616A174803F0B1FEA36D0093226DDD
:10B82000A36C216C144803F0A9FEE36D0093626DD4
:10B83000E36C616C114803F0A1FEA36F0093226FCB
:10B84000A36E216E0E4803F099FEE36F0093626FC2
:10B85000E36E616E0B4803F091FE002002B010BD54
:10B86000784A0020E5390108283A01085A3A0108C7
:10B870008C3A0108BE3A0108F03A0108223B01085F
:10B88000543B0108863B01082DE9F041514C5248D8
:10B8900092B003F073FE63780BB9504800E0504853
:10B8A000504DDFF86C8103F069FE28680921826839
:10B8B000FFF782FE28680A218268FFF77DFE4A486A
:10B8C00003F05CFE002606EB08031B790BB9434826
:10B8D00000E04348434F03F051FE28680921826885
:10B8E0002436FFF769FE6C2EEDD13868394D826839
:10B8F0000A21FFF761FE38680A218268FFF75CFEC3
:10B90000F5F778F8637806460F46002B5DD0B5F85A
:10B910008A0095F880302978B5F92C200290B5F886
:10B9200088000190D5F88400008800902F4803F02B
:10B9300025FEE86E296F801B61EB0701002871F17D
:10B94000000305DB2A4A002302F032FF064600E02E
:10B950000026236A274993F98C50282208A8FDF76E
:10B9600037FC94F8363094F83270228E069613F035
:10B97000020F214B214918BF1946638F059394F894
:10B980003830049394F82630039394F82730012636
:10B990009E4025EAE5758DE86200194B1949022F92
:10B9A00008BF0B460146184803F0E8FDE46964B19E
:10B9B000611D282208A8FDF70BFCE369E28A014615
:10B9C000124803F0DBFD2468F1E7002012B0BDE867
:10B9D000F08100BFE8490020C43B0108D53B0108C5
:10B9E000D93B010884020020DD3B0108EC3B010843
:10B9F00040420F00F0490020EA230108C424010856
:10BA0000BD3B0108B83B0108303C0108873C0108F8
:10BA10005C45002038B50546084603F055F8C4B229
:10BA20002046FAF717FD28B921460B4803F0A6FD7A
:10BA3000012038BD083015B1FAF77CFF01E0FAF7B4
:10BA400080FF064B064A0748002D08BF1A462146CC
:10BA500003F094FD002038BD77380108BD3C010893
:10BA6000B83C0108C43C010838B50C4603F02CF87A
:10BA7000C5B22846FAF7EEFC28B929460B4803F070
:10BA80007DFD012038BD90F83630094923F00203CE
:10BA900043EA440380F83630064B0748002C08BFC1
:10BAA000194603F06BFD002038BD00BF7738010850
:10BAB000D43B0108B4180108ED3C0108012838B551
:10BAC00005460C4603DCBDE83840FFF7DDBE6349A0
:10BAD000606803F0D9FE0028F5D0032D09D1604934
:10BAE000606803F0D1FE88B9A068BDE83840FFF770
:10BAF00079BD042D0AD15B49606803F0C5FE28B901
:10BB0000E168A068BDE83840FFF786BD5649606827
:10BB100003F0BAFE30B9032D7AD1A068BDE83840F1
:10BB2000FFF7A8BD5149606803F0AEFE00BB042DCD
:10BB30006ED14F49A06803F0A7FE20B9E068BDE8C8
:10BB40003840FFF7B7BD4B49A06803F09DFE20B910
:10BB5000E068BDE83840FFF7D1BD4749A06803F071
:10BB600093FE002854D1E068BDE83840FFF7EABDF5
:10BB70004249606803F088FE58B9032D48D1404916
:10BB8000A06803F081FE002842D1BDE83840FFF7ED
:10BB900011BE3C49606803F077FE20B9032D37D110
:10BBA000A168012007E03849606803F06DFE30B9F4
:10BBB000032D2DD1A168BDE83840FFF72BBF3349D5
:10BBC000606803F061FED0B9022D21D03049A06831
:10BBD00003F05AFEE0B9052D1AD12E49E06803F0B2
:10BBE00053FE08B9012105E02B49E06803F04CFE43
:10BBF000014668B92069BDE83840FFF735BF2749DD
:10BC0000606803F041FE18B9BDE83840FFF7E0BDB9
:10BC1000234803F03DFD234803F03AFD224803F09A
:10BC200037FD224803F034FD214803F031FD21485F
:10BC300003F02EFD204803F02BFD204803F028FDE3
:10BC40001F4803F025FD1F4803F022FD1E4803F0A6
:10BC50001FFD1E4803F01CFD002038BD153D0108E6
:10BC6000011901081A3D01081F3D0108223D010884
:10BC7000C82401082A3D01082F3D010804140108C9
:10BC8000353D0108B83C0108BD3C0108CA24010843
:10BC9000393D0108EA230108C42401089528010858
:10BCA0003D3D0108553D01088F3D0108C83D010893
:10BCB000013E01083A3E0108713E0108B43E010808
:10BCC000FD3E01083A3F01085F3F0108AA3F010815
:10BCD0002DE9F04301288DB005460C4605DC0968C6
:10BCE0002D4803F04BFC2D481DE0182200210DEBE0
:10BCF000020003F03BFB0423069361687B2307A843
:10BD0000ADF82E30FDF71AFB022D04D0A06802F02A
:10BD1000DBFE014601E041F2883106A800F046F85A
:10BD2000002804DA1E4803F0B3FC01202DE000F0E7
:10BD3000A1F804460D46F4F75DFE15A3D3E90023F0
:10BD40008018594100196941164A002302F030FD5C
:10BD50000CAB43F81C0D184603F006F90269446960
:10BD6000C6688768D0F80480D0F80090551C00F0B1
:10BD700081F804F26C7403908DE8800333462A4600
:10BD80002146094803F0FAFB00200DB0BDE8F0831E
:10BD9000006043B7EF26F8FFD63F0108FB3F0108DC
:10BDA0001340010840420F002C40010800232DE9F8
:10BDB000F34102460E462A481946FCF7A5FD002825
:10BDC0004ADB284D30220021284603F0CFFA2B7899
:10BDD000234823F03F0343F023032B70302200233A
:10BDE0002946FCF763FE041E03DA1D48FCF7E2FD5A
:10BDF00031E0002433460094302229461848FCF7ED
:10BE0000E7FD061E164803DAFCF7D4FD304623E0B2
:10BE1000FCF7D0FD01211448F6F708F9D5F8288081
:10BE2000ED6AF4F7E7FD2DBA0646E8200F46002339
:10BE30000E4AA5FB000102F06BFC0C4B98FA88F847
:10BE4000E3FB0801801B0A4B61EB0701C3E900011A
:10BE50000548F6F71BF9204602B0BDE8F08100BFA7
:10BE600088570020345800203058002040420F00EE
:10BE700028580020D0B5074C01212046F6F7D6F807
:10BE8000054BD3E900672046F6F700F930463946FE
:10BE9000D0BD00BF30580020285800202DE9F74FB2
:10BEA000DFF8DC8001922C24444308EB04070546AC
:10BEB00097F829B0584689461E46F5F7C1F8012D76
:10BEC000824604D8019A02FB06F5A84203D82B4902
:10BED0000320F4F789FE58467968F5F7BDF858F85D
:10BEE0000440002323604FF001086360BB46636396
:10BEF000A363E363236457F838305A1C0FD0012141
:10BF000018460193F5F7F0FA019B9BF828101846A4
:10BF100008F10108F5F784FBB8F1050FEBD1BAFB86
:10BF2000F5F5731E013DB9F1010FA562E3620ED074
:10BF30000AD3B9F1020F0ED10023A361E361236894
:10BF400043F06003236006E046F2600301E047F23D
:10BF50007003A361E3614FF40043636441F2111382
:10BF60002362236843F001032360A06A00FB06609C
:10BF7000BAFBF0F003B0BDE8F08F00BF1D1201085E
:10BF800058400108012838B50AD8032908D82C23BD
:10BF9000013143430F4D03EBC1042C59013403D14C
:10BFA0000D490320F4F720FEEC58E36A9A424FF063
:10BFB0002C0303FB00F000EBC10005EB000188BF80
:10BFC000E26A0B7903F10C0304EB830488BF92B29D
:10BFD000626038BD584001081D12010830B5036881
:10BFE00045688468C168056085EA040223F000435F
:10BFF000534083EA430381EA510183EA010242F399
:10C00000000583EA8223C2600169426929402A400F
:10C010004C4053404460836030BD036823F00043CC
:10C0200063B9436853B9836843B9C36833B95421CA
:10C0300049224E234FF0590C80E80E107047000043
:10C0400038B50369436043698360836901600446CE
:10C05000C3600F4801256B1E03F0030305F00302C4
:10C0600054F8233054F8221083EA937300FB0353EF
:10C0700001354B40082D44F82230ECD12046FFF723
:10C08000CCFF2046FFF7AAFF013DFAD138BD00BF23
:10C090006589076C2DE9F341856804461DB9194986
:10C0A0000320F4F7A1FD427843689340C268C2EBD5
:10C0B00005086A0093424FF000072CBF826083603E
:10C0C000478038BF5D088668FDF7C6F9711BB0FB75
:10C0D000F1F202FB11000544B4F91030E5604FF4B1
:10C0E0007A7245446A43019304F11C030093A262EF
:10C0F000E7623B4604F1300000F0AAF802B0BDE868
:10C10000F08100BF1D12010810B5428803789A42E1
:10C11000044600D313B96369A06998472046BDE877
:10C120001040FFF7B7BF0000826843689A4210B51D
:10C13000044603D806490320F4F756FD3030F4F7DF
:10C14000CFFC6368A3602046BDE81040FFF7A2BFA4
:10C150001D120108F8B50C46174606469DF8181042
:10C160009DF81C201D461BB910490320F4F73CFD27
:10C1700003FA01F00E4B9842F6D800236380227038
:10C18000656026826170FDF767F9C5EB8503B0FB3A
:10C19000F3F202FB13000544E560A56026822462E9
:10C1A000E7832046BDE8F840FFF774BF1D12010881
:10C1B000FEFFFF7F3030F4F793BC438801334380A8
:10C1C0007047F5F763BFB0F90010F6F77FB838B5E0
:10C1D00004460020F5F70AFB05460020F5F706FBAC
:10C1E000401BA042F9D338BD30B587B004460D4698
:10C1F000F4F741F940B11DB10E490320F4F7F4FC06
:10C200002046FFF7E4FF13E00B4B009003900290F1
:10C21000012168460493CDF814D0F5F707FF2146B5
:10C2200001A82A46F4F78EFC01216846F5F7FEFEC8
:10C2300007B030BD1D120108C3C1000830B4034D62
:10C24000C560026130BC1380F4F75CBCC7C1000854
:10C2500070B41146039ABDF91050044EC6600261D5
:10C2600015801A4670BCF4F76DBC00BFC7C100084A
:10C2700070B58AB00021079106911049098803AC76
:10C2800009B2054643F23906019105A80094ADF8BC
:10C290000E600494FFF7DCFF2846F6F7E0F86B88A1
:10C2A000B34202D16B68A34204D005A8F4F718FC8E
:10C2B000012001E04FF0FF300AB070BDF402002011
:10C2C00010B5084B0446182240F83C3B02F0B4FF7E
:10C2D000082384F85630002384F8543084F857300B
:10C2E00010BD00BFE840010837B5044600F03CFB34
:10C2F00094F854301BB90321204600F060FA002561
:10C300000821684684F83650258701F071FF9DF8B2
:10C310000030019A23F0010343F002038DF800304E
:10C32000009B12BA1BBA204600F000F9BDF80010BD
:10C3300049BA204689B200F0E5F82046232100F0F2
:10C3400028F920461A2100F015F92946204600F068
:10C350003DF920460122202100F0B8F920460122B3
:10C360004FF4807100F0B2F92A4620464FF4005194
:10C3700000F0ACF9204601224FF4804100F0A6F90C
:10C38000204601224FF4805100F0A0F9012384F8E7
:10C390002830802220460C2100F057FA0421204644
:10C3A00000F065FA042100F0FD02204600F04DFA8D
:10C3B0000321204600F05BFA032100F0F002204642
:10C3C00000F043FA082220460E2100F03EFA0F2129
:10C3D000204600F04CFA1621204600F0F0F903B098
:10C3E00030BD10B590F857300133044680F857300F
:10C3F000204600F094FAA0F11103DBB2012BF7D92B
:10C40000192818BF84F856001921204600F0D7F9E2
:10C41000022384F8553010BD70B51D4690F8553094
:10C420006E1C1344144680F8553013460A46F1B288
:10C4300000F02FFA601970BD10B5012300F155020C
:10C440000021044600F025FA02221146204600F0A1
:10C45000FCF963683BB1228F120504D52046032105
:10C46000BDE81040184710BDF8B50821044600F09B
:10C47000A6F915210746204600F0F9F960F07F0281
:10C48000D2B215210646204600F0DFF906212046EB
:10C4900000F095F90821204600F0E9F960F07F02EC
:10C4A000D2B20821204600F0D0F90121204600F048
:10C4B000DEF903060546F8D532462046152100F080
:10C4C000C4F90821204600F07AF93946204600F0E8
:10C4D00076F9C5F38010F8BD38B50D460221044643
:10C4E00000F0B3F9162D07D0204600F018FA854267
:10C4F000FAD184F8545038BD204600F010FA1F28B5
:10C50000FAD0F6E710B50A0A044601F07F0180F878
:10C510002D2080F82C10202100F097F994F82C2081
:10C5200020462121BDE8104000F08FB92DE9F843E5
:10C53000054616461F4600F12D0800246FF0070936
:10C54000E2003046394602F0D7F809FB04F208F859
:10C55000010F38323046394602F0CEF804F124019A
:10C56000C2B2C9B22846013400F06FF9082CE7D1F5
:10C57000BDE8F883A1F10B020F2A07D890F8372005
:10C580008A4203D080F8371000F00ABA70470020C2
:10C59000704737B50D0A4185CAB22221044600F022
:10C5A00054F92A462321204603B0BDE8304000F06C
:10C5B0004CB9000008B5052100F059F9024B00F014
:10C5C0000F0033F9100008BDC6400108113109B24F
:10C5D0001429A8BF142121EAE171024B5A5C0521FC
:10C5E00000F033B9B040010808B52C2100F03FF944
:10C5F000C0F3071008BD38B50C462C21054600F0E5
:10C6000036F9072C28BF072400F00F0040EA041277
:10C61000D2B228462C21BDE8384000F016B908B542
:10C620002C2100F024F9C0F3420008BD0529A8BF61
:10C630000521002938B50C46A8BF0C464FF02C0147
:10C640000546B8BF072400F012F920F00E0040EABA
:10C650004402D2B228462C21BDE8384000F0F5B89B
:10C6600038B505460C4699B10A782D2100F0EDF851
:10C670002E21284600F0FBF8637800F0F80203F062
:10C6800007031A4328462E21BDE8384000F0DDB8E4
:10C6900038BD08B5092100F0EAF800F00F004000AD
:10C6A0005B3840B208BD0029C4BF494249B25B3182
:10C6B000C1F3430242F0C002092100F0C6B808B538
:10C6C000072100F0D4F85B3840B208BD10B5038FE5
:10C6D0000446B2B30B43B1F5807F03870AD002D87A
:10C6E000202925D010BDB1F5007F0ED0B1F5005F37
:10C6F00020D010BD00F12E01FFF7B2FF042120462B
:10C70000FFF794FF53222F2153E02E2100F0AFF8C2
:10C7100040F01002D2B22E21204600F096F81721E8
:10C72000204600F0A4F840F00202D2B2172140E007
:10C730002E212BE00E2100F09AF840F00402D2B234
:10C7400036E023EA0103B1F5807F03870AD002D8DF
:10C75000202921D010BDB1F5007F09D0B1F5005FCF
:10C7600021D010BD4FF0FF31BDE81040FFF75EBF94
:10C77000172100F07CF8172100F0FD02204600F0A0
:10C7800064F8238F9B0619D52E21204600F06FF800
:10C7900000F0EF022E210CE02E2100F068F840F0AE
:10C7A0001002D2B2F6E70E2100F061F800F0FB02B1
:10C7B0000E212046BDE8104000F047B810BD70B50E
:10C7C00004460D46204600F0AAF8A0F11103DBB2A2
:10C7D000012B0646F6D91F28F4D0032D02D12A4694
:10C7E000082126E0A84227D0162801D1192D02E001
:10C7F000192807D1162D0AD1092211462046FFF724
:10C800006BFE04E00F2802D1204600F094F80F2DB3
:10C810000DD103212046FFF7D2FF2946204600F024
:10C8200026F8E06CF4F736FF84F8545004E02A460A
:10C8300029462046FFF750FE304670BD90F8403044
:10C84000416CC06B0022F4F783BD70B504460D4601
:10C850001646FFF7F3FF334645F0C002616CE06B0C
:10C8600001F017FEE06BBDE87040F4F7B1BD38B5DC
:10C8700004460D46FFF7E2FF45F080020023616C9D
:10C88000E06B01F006FE0546E06BF4F7A1FD2846DB
:10C8900038BDF7B504460F4615461E46FFF7CEFFD6
:10C8A000616CE06B4023012201F0E2FD3B46616CCC
:10C8B000E06B012201F0DCFD0022E06B01960092AA
:10C8C0002B46616CF4F7A0FDE06B03B0BDE8F040CF
:10C8D000F4F77EBD10B50446FFF7B0FF616CE06B66
:10C8E00020230122BDE8104001F0C2BD07B58DE84C
:10C8F00006000023416CC06B0122F4F785FD03B0F4
:10C900005DF804FB10B50446416CC06B01230022A6
:10C9100001F0AEFDE06BBDE81040F4F759BD08B57D
:10C9200090F854300F2B04D00121FFF7A0FF00F046
:10C930001F03184608BD10B50446FFF7F0FF0F2887
:10C9400011D1E06CF4F7AFFE00214FF49970FFF7BE
:10C950004BFC01212046FFF78AFF00F01F0008284A
:10C9600084F85400F5D110BD10B50446006DF4F7FD
:10C970009AFE00213E20FFF737FC206DF4F78AFE77
:10C9800000213E20FFF730FC01212046FFF76FFF1A
:10C9900000F01F0310F0170F84F85430F4D110BDCD
:10C9A00038B508210446FFF70AFF0821054620464E
:10C9B000FFF75DFF94F8373000F0E00203F01F034B
:10C9C00020461A430821FFF740FF29462046BDE8CC
:10C9D0003840FFF7F4BE43680BB100211847704799
:10C9E0002DE9F0470446884616461F46FFF797FF95
:10C9F0008146002C00F0D3800F2840F0DF80B8F192
:10CA0000180F66D02046FFF796FFB8F1270F00F207
:10CA10002B81DFE818F042002901280033002901AA
:10CA200029013B00290129012901290129012901A5
:10CA3000290129012901550029018B008F007E0061
:10CA400029018400290129012901930097009B00F5
:10CA50009F002901A300AA00290129012901290118
:10CA600029014E00BA00022F03D98B490320F4F7A5
:10CA7000BBF831882046FFF745FD94E0082FF4D835
:10CA8000D6E900232046FFF751FD8CE0022FECD8B9
:10CA900031882046FFF77DFD85E0012FE5D0317814
:10CAA000A1F10B030F2B00F2EC802046FFF762FD93
:10CAB00079E0012FD9D03378002B40F0E2806CE090
:10CAC000022FD2D8B6F900102046FFF77FFD0225CD
:10CAD000D9E0012FC9D83378013B052B63D8DFE8B3
:10CAE00003F00507620C1403082102E00F2100E0A7
:10CAF00016212046FFF763FECBE0238F5A0540F155
:10CB0000C8802046FFF798FCC3E02046FFF7ECFB07
:10CB1000BFE0327820212046FFF7D8FD43E0012F07
:10CB2000A3D831782046FFF766FD36E032784FF41F
:10CB3000806116E032784FF4007112E032784FF4E1
:10CB400000510EE032784FF480410AE032784FF421
:10CB5000006106E032784FF4805102E032784FF401
:10CB600080712046FFF7B2FD17E0012F3FF67DAF41
:10CB7000238FDB0503D43378052B40F2828096F9AE
:10CB800000102046FFF752FD07E0012F3FF66DAF82
:10CB900096F900102046FFF786FD012573E06FF03F
:10CBA0001200BDE8F087B9F10F0F5DD03B46324669
:10CBB00041462046BDE8F04701F0DCBBB8F1270F45
:10CBC000F4D801A353F828F09BCA0008ADCB0008A5
:10CBD00067CA00087DCA0008ADCB0008ADCB0008CD
:10CBE0008DCA0008ADCB0008ADCB0008ADCB000866
:10CBF000ADCB0008ADCB0008ADCB0008ADCB000835
:10CC0000ADCB0008ADCB0008C1CA0008ADCB000811
:10CC10002DCB000835CB000813CB0008ADCB0008A6
:10CC20001FCB0008ADCB0008D3CA0008ADCB00086D
:10CC30003DCB000845CB00084DCB000855CB000884
:10CC4000ADCB00085DCB00086BCB0008ADCB000876
:10CC5000ADCB0008ADCB0008ADCB0008ADCB0008D4
:10CC6000B3CA00088BCB0008B8F1180F9ED06FF044
:10CC700085050F212046FFF7A2FD15F1860F05D18E
:10CC800094E76FF01505B9F10F0FF2D02846BDE813
:10CC9000F0870120BDE8F0871D1201082DE9F04161
:10CCA0000446FFF73CFE0F2806464CD00F212046D5
:10CCB000FFF7DDFD022107462046FFF7D8FD7B0781
:10CCC000054603D5636801212046984738073AD5C1
:10CCD000162E01D0112E05D1238F590433D5636848
:10CCE00002212CE0192E01D0122E2CD194F85730AD
:10CCF0001BB916490320F3F777FF013BDBB284F839
:10CD0000573023B994F856102046FFF758FD636852
:10CD1000CBB1228FD20416D505F0E000202809D02F
:10CD200002D838B1BDE8F081602807D0A02803D030
:10CD3000BDE8F081042102E0062100E00721204641
:10CD4000BDE8F0411847BDE8F08100BF1D120108A1
:10CD500013B50446416CC06BF4F7CCFA0121E06CCA
:10CD6000F4F7C2FBE06CF4F79EFC0121206DF4F7B0
:10CD7000BBFB206DF4F78EFC0D4B009401220021CB
:10CD8000A06CF4F7EBFB2046FFF7AEFA1C2120461F
:10CD9000FFF76DFD032807D11C22002104F10C00D0
:10CDA00002F0E4FA002001E04FF0FF3002B010BDC5
:10CDB000D7C900082DE9F34104460F4690461E46A8
:10CDC000FFF788FD01220DF103012046FFF78EFDDC
:10CDD0009DF8035005F07F05023D37B3454505D961
:10CDE0002046FFF78FFD6FF0680521E0236A0133CD
:10CDF0002362636A2B442A46394620466362FFF762
:10CE000075FD022201A92046FFF770FD6EB10122D7
:10CE1000B1182046FFF76AFD2046FFF773FD072192
:10CE20002046FFF724FD307002E02046FFF76AFD40
:10CE3000284602B0BDE8F0812DE9F04106460D46D6
:10CE40009046FFF7CEFA00273C46474512D06A6865
:10CE5000A31C13447F2B05F1080514D8F36955F87A
:10CE6000081C2344F36130462346FFF7D5FA013707
:10CE70000446EAE7338F5B0502D43046FFF7DCFA5D
:10CE80002046BDE8F0816FF08A00BDE8F081000027
:10CE900008B5FFF744FD0838C0B211289ABF024B0D
:10CEA000185C022008BD00BF004101082DE9F843CD
:10CEB0000F46164698460546002800F0B780A1F1B7
:10CEC0001103152B4DD8DFE803F01827344C4C4CD8
:10CED0004C204C383C40444C484C4C4C4C4C4C0B3B
:10CEE000B8F1010F03D857490320F3F77DFE002363
:10CEF0007370FFF74CFB307004E0B8F1010FF2D90A
:10CF0000662333800220BDE8F883B8F1000FEAD031
:10CF1000FFF7BEFF307009E0038F13F4806F03D07A
:10CF200001203070BDE8F883002333700120BDE894
:10CF3000F883038F13F4007FF1E7038FC3F34033CB
:10CF4000F3E7038FC3F38033EFE7038FC3F3C0230B
:10CF5000EBE7038FC3F30033E7E7038FC3F300234B
:10CF6000E3E74346324601F051F910F1860F0446DB
:10CF700060D12846FFF7D3FC0F28814611D12846FF
:10CF8000FFF7D9FC162F1CD004D8012F35D0102F55
:10CF90000ED046E0272F28D02F2F36D0202F1DD09F
:10CFA0003FE0162F0DD013D8012F26D0102F44D1DB
:10CFB000B8F1010F97D92846FFF7FCFA0224308018
:10CFC0002CE0B8F1000F8ED02846FFF70DFB23E0D0
:10CFD000272F0AD02F2F18D0202F2ED1B8F1000FD5
:10CFE00081D02846FFF71BFB16E0B8F1000F3FF495
:10CFF0007AAF2846FFF74DFB0EE0B8F1000F3FF483
:10D0000072AF2846FFF730FA06E0B8F1000F3FF4A0
:10D010006AAF2846FFF753FB30700124B9F10F0FB8
:10D0200008D10F212846FFF7CAFB03E06FF012007A
:10D03000BDE8F8832046BDE8F8836FF08500BDE8C1
:10D04000F88300BF1D120108094B70B51C68064625
:10D050000D4620460821F3F709F921463046F3F73B
:10D0600043FE2846F3F704FABDE87040F3F722BE0A
:10D07000F80200202DE9F04104460E461546F3F76C
:10D08000EFF927688046A7B13B68236096E8030064
:10D090007B6883E803000A21A7F10800F3F7E6F8AC
:10D0A00017F8034C4046F3F7E3F92046F3F71EF96F
:10D0B0001FE0A268E3689B1A2269934207DDDDB195
:10D0C0004146201DFFF7C0FFF3F7CAF980460D4B1C
:10D0D000E1681B8833804B1CE360236962690B4065
:10D0E00096E8030002EBC30383E803004046F3F72E
:10D0F000BFF90120BDE8F081F3F7BAF92846BDE891
:10D10000F08100BFF4020020F8B504460F46154632
:10D11000F3F7A6F9A168E3688B4206461CD04B1CC6
:10D12000A3602369626965680B4002EBC30393E85F
:10D13000030087E80300E5B128460A2150F80839C2
:10D140006360F3F793F815F8034C3046F3F790F962
:10D150002046F3F7CBF80FE03DB1084B1B680146C2
:10D16000DF602046FFF770FF06E0F3F781F92846FD
:10D17000F8BD3046F3F77CF90120F8BDF802002035
:10D18000BFF34F8F0549064BCA6802F4E0621343B0
:10D19000CB60BFF34F8F00BFFDE700BF00ED00E0A5
:10D1A0000400FA050121F4F741BF10B504464069B7
:10D1B00008B101F0EDF9E06908B101F0E9F90020EA
:10D1C0000022002360612061E061A0612080C4E949
:10D1D000022310BDF3F70EBC2DE9F04F89B08A464B
:10D1E00015469B460446FFF7F5FFCDE90401EB0029
:10D1F0000393079355445346AB4205D013F8012BD4
:10D20000002AF9D0002300E00123002702936FF0E9
:10D2100075030193B846B9463E46A268974270D25C
:10D2200022687D0102EB050EDEE90201002908BF3C
:10D23000B0F1FF3F23D0DDE90423994208BF9042BB
:10D240001DD200220023CEE9022322682A4416615F
:10D2500022682A4496612268565322682A445069FB
:10D2600020B101F095F922682A44566122682A44C7
:10D27000D06920B101F08CF922682A44D661039B61
:10D2800098453CD222682A445069002837D007AA22
:10D29000514601F0B3F938B923681D44129BCBF80D
:10D2A00000500120186034E0029B13B102282DD1F8
:10D2B000F2E7012814D122681544296911F07F4F43
:10D2C0001BD0079AB2EB116F17D3B8F1000F01D042
:10D2D000904512D20023CBF80050904601930AE00B
:10D2E00002280AD1B8F1000F07D12268CDF80480D6
:10D2F0001544CBF800504FF00109039B0793013709
:10D300008BE7129B0198C3F8009002E00128F4D14A
:10D31000D1E709B0BDE8F08F38B505460C46FFF7F8
:10D3200059FF4FF47A736B43C01841F10001C4E90F
:10D33000000138BD2DE9F04788B0972990461BBF02
:10D34000109A0792424605AA8A461CBFCDF814805F
:10D350008DF81830ADF806100292DF0000F11205CA
:10D3600000F1200600F11C046FF0010935F9023FBD
:10D37000DBB1BAF1970F03D000976A46414607E048
:10D38000D8F8183019684B78DB0000936A460231F0
:10D39000306801F033F9023007D0B5F9002003A955
:10D3A00001A8F4F7FDFF4FF00009A54206F10406BD
:10D3B000DCD1484608B0BDE8F087000030B587B042
:10D3C00006AA102302AD294642F8143D01F0F8F8F0
:10D3D000A842014620D1019B102B08D128220F48DA
:10D3E000FBF7F6FE01460E4802F0C8F814E00024F0
:10D3F000019BA34204D3295D0A4802F0BFF802E072
:10D40000094802F0BBF80134102CF1D10724074879
:10D4100002F0B4F8013CFAD107B030BD64580020E6
:10D4200012410108BA2601089C2201089D22010828
:10D430002DE9F04F00F10C0787B0044638469A46B4
:10D440008B469046149EFFF7ADFE01230493B8F17E
:10D45000000F01D0119B2BB93846F4F717FE6FF07F
:10D460000D006AE004AB0093524605AB41462046EE
:10D47000FFF7B2FE012802D04FF000091CE012991C
:10D480001198059C01F022F8054610B96FF00B04C5
:10D490004FE0E06901F07CF8139BE561721CA36129
:10D4A00002D004F1080139E04FF0FF320023C4E953
:10D4B00002233DE009F10109A2689145E6D2226804
:10D4C0004FEA49152A44D2E9020150EA0103F1D199
:10D4D00051464046039200F0F9FF039A50612268DA
:10D4E0002A44516971B1109B1361226812991198F5
:10D4F0002A44039200F0EAFF039A139BD06122684A
:10D500002A44936122682A44D1690029D2D0A2F822
:10D5100000B0731C216805D0294408313046FFF75C
:10D52000FBFE05E00D444FF0FF320023C5E9022366
:10D5300000243846F4F7AAFD204607B0BDE8F08F76
:10D540002DE9F04300F10C0585B0044628461F463E
:10D55000884691460E9EFFF725FE01230293B8F1FF
:10D56000000F00D02FB92846F4F790FD6FF00D00A2
:10D570002CE002AB00934A4603AB41462046FFF73E
:10D580002BFE012802D06FF00B041BE038460C99EB
:10D59000039C00F09BFF07460028F4D0E06900F0F0
:10D5A000F7FF0D9BA361731CE76105D004F108012F
:10D5B0003046FFF7B1FE04E04FF0FF320023C4E92C
:10D5C000022300242846F4F761FD204605B0BDE89B
:10D5D000F083F0B500F10C0485B0054620460E46F8
:10D5E0001746FFF7DFFD0123029302AB00933A4693
:10D5F00003AB31462846FFF7EFFD012802D103981F
:10D60000FFF7D3FD2046F4F741FD05B0F0BDF8B5B6
:10D6100000F10C06054630460F46FFF7C3FD002417
:10D62000AB689C420AD22868630117B1C25EBA4255
:10D6300002D11844FFF7B9FD0134F1E73046BDE8E7
:10D64000F840F4F723BD2DE9F04F00F10C0485B04C
:10D65000054620469B46894692460F9EFFF7A2FD4F
:10D6600001230293B9F1000F04D0BBF1000F01D0E8
:10D670000E9B2BB92046F4F709FD6FF0150049E029
:10D6800016B1BAF1000F05D12046F4F7FFFC6FF098
:10D690000D003FE002AF009703AB109A31462846D9
:10D6A000FFF79AFD0128804615D9119B0093324659
:10D6B000109B99212846FFF73DFE48B901230293AC
:10D6C000009703AB109A31462846FFF785FD804648
:10D6D000B8F1010F0CD8039B5A465146D86900F0A7
:10D6E0006FFF58B92046F4F7D1FC6FF0680011E0E5
:10D6F0002046F4F7CBFC6FF075000BE0039BB3F909
:10D700000020A9F800200E9A9B6913602046F4F7C8
:10D71000BDFC002005B0BDE8F08FF8B50646002539
:10D7200046F80C5F04463046FFF73CFD04F1120258
:10D7300004F11C0304F1300122F8025F43F8045F96
:10D740008B424FF00007F7D123792761022BA268A3
:10D750000BD1236852013946186801F007FE23688F
:10D760009A685868D200394602E02068520139466A
:10D7700001F0FCFD00F0A4FF3046BDE8F840F4F7EE
:10D7800085BC00002DE9F04F044600F10C0585B082
:10D790002846FFF707FDFFF71DFD2379012B804683
:10D7A00089466AD1674A684B684969488DE80C0028
:10D7B000684B01F0E3FE4FF0000BA3689B456BD272
:10D7C00021684FEA4B1A5144D1E90223134351D047
:10D7D0004869FFF7F3FD23685F485344196901F076
:10D7E000CDFE23685344196911F07F4F04D0090E10
:10D7F0005A4801F0C3FE02E0594801F0BFFE236819
:10D800005344D869FFF7DAFD2368534853449969B4
:10D8100001F0B4FE23685344D3E90267002F08BF28
:10D82000B6F1FF3F1CD0B6EB080667EB0907002EE8
:10D8300077F1000301DA4B4913E0304639464A4A92
:10D84000002300F0B5FF002303923046464A3946D4
:10D8500000F0AEFF039A0146444801F08FFE03E05A
:10D860004349444801F08AFE2368434833F90A10CB
:10D8700001F084FE0BF1010B9FE7022B0CD1324B20
:10D8800000933E4A3E4B3F493F4801F077FE4FF040
:10D89000000BA3689B4505D3284605B0BDE8F04FB3
:10D8A000F4F7F4BB236819684FEA4B1A5144D1E9E5
:10D8B0000223134343D08B691868FFF77FFD236869
:10D8C0001B6853445B691868FFF778FD23682F488D
:10D8D0001B685344196901F051FE23681B685344C7
:10D8E000D3E90267002F08BFB6F1FF3F1CD0B6EBAB
:10D8F000080667EB0907002E77F1000301DA1949E2
:10D9000013E030463946184A002300F051FF002347
:10D9100003923046144A394600F04AFF039A014602
:10D92000124801F02BFE03E01149124801F026FED7
:10D93000236811481B6833F90A1001F01FFE0BF130
:10D94000010BA6E755420108104201086B4201088D
:10D95000E7410108DE41010818420108224201089E
:10D960002B4201083342010840420F0042420108A5
:10D970004C4201083B420108DD1501085B420108E9
:10D9800052420108684201087742010899420108A1
:10D99000F8B5064684890F46154600206DB9002368
:10D9A000B289B168FBF786FB4FF6C57302199A423C
:10D9B00039680EDD013080B20BE0AE42EFD0234675
:10D9C000AA89A968FBF776FBEB686D681C44A4B2D2
:10D9D000E4E73A34204400232022083180B2FBF7E8
:10D9E00069FBC04380B2F8BD2DE9F3410C46804687
:10D9F00003212046F7F7E9F9054618B92E49032017
:10DA0000F3F7F2F80221F7F7E0F907460028F5D01E
:10DA1000EB68032B4CD900F1080122462846AE687A
:10DA2000FFF7B6FF002843D13378803B082B30D86E
:10DA3000DFE803F0052F2F2F2F0C151E2700AB89D1
:10DA4000B9683246404600F081F822E0EB68009366
:10DA5000BA68334621464046F5F79CFE19E0EB686C
:10DA60000093BA68334621464046F5F715FF10E0AB
:10DA7000EB680093BA68334621464046F5F7F4FC5C
:10DA800007E0EB680093BA68334621464046F5F755
:10DA9000B7FD3178234640F201220320F6F768FEF5
:10DAA000014628B9204602B0BDE8F041F7F702BCB4
:10DAB00002B0BDE8F08100BF1D12010838B50D4667
:10DAC000144600211A460323F7F702FB28B18368A6
:10DAD00000221D705C709A70DA7038BD10B5044673
:10DAE00068B190F91030032B0CD142680831FFF770
:10DAF0004FFF50B1A36840BA5880002010BD6FF0AE
:10DB00000D0010BD6FF04C0010BD6FF0010010BD96
:10DB10002DE9F041DDF81880154600220E461F461B
:10DB2000014608F108031046FFF7C8FF044650B14C
:10DB3000806876BA6DBA8680C58027B1424639467C
:10DB4000083001F079FB2046BDE8F081F7B50646C4
:10DB50000C46002A38D0072B36D99188D088083B4C
:10DB600040BA49BA009389B202F1080382B2812017
:10DB7000FFF7CEFF074638B3237EFF2B04F10802E0
:10DB80000CBF002104F1180100F022F8054610B97D
:10DB90000146384613E000231A4619461846F7F79F
:10DBA00065F8836809495E8004464560034640F293
:10DBB00002220220F6F7DCFD014628B9204603B018
:10DBC000BDE8F040F7F776BB03B0F0BD0000FFFF03
:10DBD000F8B50F461646022328220021F7F778FAF7
:10DBE000054600B38468102204F10800394617B1D5
:10DBF00001F022FB01E001F0B9FB04F11800102252
:10DC0000314616B101F018FB04E001F0AFFB01232F
:10DC100084F82730602200232270FF226370A370F3
:10DC2000E370A271E3712846F8BD38B505460C468D
:10DC300019B301F17000F2F753FF2846F5F77EF9AA
:10DC400038B1D0F810329C4203D100F5FC70F2F7E5
:10DC500047FF04F11C00F2F743FF04F13800F2F72C
:10DC60003FFF04F15400F2F73BFF10220021204651
:10DC700001F07CFB00236383637638BD08B5102276
:10DC8000034901F0A7FAB0FA80F0400908BD00BFCF
:10DC9000C41701082DE9F74F904600901E469DF8E5
:10DCA0003070894609B900205CE0082BFBD8084693
:10DCB000FFF7E4FF0028F6D1824604464FF0980BA8
:10DCC0002A4B0BFB0AF29D18494628460192FBF7A6
:10DCD00018FA019A78B1B8F1000F42D0002E40D066
:10DCE000224B02F1100041463246184401F0A4FADA
:10DCF0002E766F7635E02846FFF7C0FF10B1002C76
:10DD000008BF2C460AF1010ABAF1080FD8D1002C3D
:10DD1000C9D0BDF80030638310224946204601F087
:10DD20008BFAB8F1000F07D036B13246414604F104
:10DD3000100001F081FA2676677607F00707022FB8
:10DD400004BF032384F894304FF40973A4F8863099
:10DD50004FF40473C4F888406386646324652046E6
:10DD600000E0284603B0BDE8F08F00BF8C580020CB
:10DD70002DE9F04107460E4611B90020BDE8F081BB
:10DD80000846FFF77BFF0028F7D10C4D0446A84654
:10DD9000B5F91A3013B10FB1BB4209D1314628464B
:10DDA000FBF7AFF920B1982000FB0480BDE8F081BB
:10DDB0000134082C05F19805EAD1DEE78C580020E3
:10DDC00010B50446FFF7D4FF01462046BDE81040D9
:10DDD000FFF72BBF38B510B100F1980400E0074CF5
:10DDE000074DAC4205D22046FFF748FF18B19834E2
:10DDF000F7E7002038BD204638BD00BF8C58002012
:10DE00004C5D002008B5FFF7E5FF10B1437E1B070E
:10DE1000F9D508BDF8B501460020FFF7A9FF044673
:10DE200010B3437E13F0050F1ED0B0F91A00F5F7BA
:10DE300085F80E4BD0F8D461B3F9007004F13805C1
:10DE40002846F2F74DFE40F21723A4F84E3004F1B5
:10DE50004C023B4631462846FEF7F0F9637E23F03C
:10DE6000070343F0070363762046F8BD2C24002007
:10DE700010B5144600B119B90B490320F2F7B4FEEE
:10DE80002AB1537E03F00703013B012B01D8002088
:10DE900010BD137E0B70127E04F1100101F0CCF95D
:10DEA000B4F91A0010BD00BF1D120108F0B503EB54
:10DEB00043048C424FF0000122D8017005465E1EDB
:10DEC0000F464FF03A0E994219D014782409092CC4
:10DED00094BF3034573494462C709CF8004004F0C2
:10DEE0000F04092C94BF30345734B1426C700CBF0E
:10DEF0003C467446AC70013201310335E3E7F0BDB6
:10DF00000846F0BD2DE9F04112B90020BDE8F081CE
:10DF10001378002BF9D01446264601347378002B71
:10DF2000FAD107464FF0010C964217D33478A4F18A
:10DF300030055FFA85F8B8F1090F06F1FF3E23D9E5
:10DF4000A4F14105052D02D8A4F137051CE0A4F188
:10DF50006105052D11D8A4F1570515E0BCF1000F9E
:10DF6000D3D1013FB84205D23A780178397000F830
:10DF7000012BF6E71846BDE8F081BCF1000FC4D1D3
:10DF80004FF0010C7646CFE7724518D8A6F1020E85
:10DF900016F8016CA6F130045FFA84FCBCF1090F9D
:10DFA0000ED9A6F14104052C02D8A6F1370407E0EA
:10DFB000A6F16104052C02D8A6F1570400E0002464
:10DFC00001338B42A1D845EA04143C704FF0000C99
:10DFD0000137D7E713B5074A044692E80300002249
:10DFE0008DE80300694604F11000FFF743F802B022
:10DFF00010BD00BFA442010803460846002110B42A
:10E0000083E80600072401221C621A7203F1280427
:10E0100003F11002196159619961D9615C62DA609A
:10E02000194610BCF6F758BE70B51C46531E033394
:10E030000E4688B0114600F1100506D8294B07900E
:10E0400003A80693F2F75EFD00E02AB1012201A9C0
:10E050002846FFF759F805E001A92846FFF754F8CC
:10E06000002838D003A8F2F73BFDBDF8063040F297
:10E07000012293420CD048F2744293422ED1029A6C
:10E08000194B9A4214BF6FF003006FF0730027E042
:10E09000029D02212846F6F798FE10B1C368272B8F
:10E0A00003D812490320F2F79FFD8168102208313E
:10E0B000201D01F0C1F8042323604FF0FF312846F2
:10E0C000F6F783FE08B9A08202E083685B88A3822A
:10E0D0003560002004E06FF00A0001E06FF00300FB
:10E0E00008B070BDD5DF0008630B8AF31D1201086C
:10E0F0002DE9F0478946064690469A460146002497
:10E1000019B1CB6849681C44FAE7D9F80030D8F84F
:10E110000020934216D1042B14D108F1040209F116
:10E1200004013046FFF754FD0746C8B396F9105076
:10E130000DB902253574BB6883F806A0B9F81460E0
:10E1400056B906E03046F7F7B5F86FF06900BDE85C
:10E15000F087B8F8146086B1002319461A461846AD
:10E16000F6F784FD36B2014618B93846F7F7A2F83B
:10E1700016E08B685E804F600F460B493B4640F2CD
:10E1800002222846F6F7F4FA014630B93846F7F786
:10E1900091F86FF04C00BDE8F0872046BDE8F087AD
:10E1A0006FF00B00BDE8F0870000FFFF7FB50C4665
:10E1B000054600B119B90D490320F2F715FD0A46CD
:10E1C00001AE232101F0D2F8304600F04BF90023D4
:10E1D000B3FBF4F204FB1232F15CA85C0133414062
:10E1E0000C2BA954F4D104B070BD00BF1D1201085E
:10E1F00010B50446FFF7DAFF034B1A78511C19706B
:10E2000023785340237010BD82020020062938B5C0
:10E2100004460D46104636D006D8032922D029D808
:10E22000B1B3022911D09DE017294AD004D808299A
:10E2300051D0152932D095E0252948D0292900F060
:10E240008980192940F08E8035E0012B03D8484998
:10E250000320F2F7C9FC0A4604F12C0100F0ECFFA0
:10E26000284638BD072BF2D9082204F12E0100F010
:10E27000E3FF7AE0022BEAD1228F520701D5082270
:10E2800004E003806CE0022BE1D1628D028067E044
:10E29000022BDCD194F8373013800AE0012BD6D161
:10E2A000238F13F0200F02D00123037058E00023C6
:10E2B0000370012038BD012BC9D1238F13F0020F49
:10E2C000F1E7012BC3D194F92820027048E0022B1A
:10E2D000BDD10322DAE7072BB9D9238F5B074CBFE7
:10E2E0002B4602234FF000024CBF04F12E0104F133
:10E2F0002C01042B4270027018D0082B03D0022B83
:10E3000033D1134619E00A7882F0020202704A788B
:10E3100042708A788270CA78C2700A7902714A792A
:10E3200042718A798271CA79C27119E00B7883F0DF
:10E33000020303704B7843700223FF240022C47051
:10E34000FE24827004714271CA5C827119444B7858
:10E35000C3710AE0042B7FF47AAF04F10C01116061
:10E36000184638BD6FF0850038BD082038BD00BFA5
:10E370001D12010870B515461C4619296AD8DFE838
:10E3800001F00D691929393949696969696969694A
:10E39000696969696969694E69616958022C03D0C4
:10E3A0002F490320F2F720FC1388FF2BF8D880F8C0
:10E3B00037304DE0022CF3D800F12C060222002168
:10E3C000304600F0D3FF22462946304600F034FFA5
:10E3D000022070BD082CE3D800F12E06082200218F
:10E3E000304600F0C3FF22462946304600F024FFA5
:10E3F000082070BD022CD3D11388022B06D0082B25
:10E400002BD1038F43F00403038721E0038F23F014
:10E4100004030CE0022CC3D11388438518E0127862
:10E42000038F12B143F0200301E023F020030387A0
:10E43000CEE71278038F12B143F00203F7E723F01F
:10E440000203F4E7012CABD192F9003080F82830B8
:10E45000204670BD6FF0850070BD6FF0690070BD23
:10E460001D1201080C22014900F0E6BE107AFF1FC0
:10E4700010B586B006AC04F8093D012301930DF1F7
:10E48000170300932346F2F7BFFF9DF8170006B06D
:10E4900010BDF0B585B01F4604AB002403F8012D74
:10E4A000012205460E4601920094F2F7ADFF3B466D
:10E4B000224631462846FFF7DBFF05B0F0BD0000DD
:10E4C00001210148F3F7B2BD4C5D00202DE9F04772
:10E4D00080460E46FFF7F4FF294C002514F8013C56
:10E4E0009E420AD132464146204600F073FE20B9D2
:10E4F000244B122404FB053428E00135282D04F1B7
:10E500001204EBD1204B1B68272B33D81D4B002561
:10E51000122202FB05F91B4F19F803A0BAF1000FF4
:10E5200025D107EB090463789E4207D0102251469B
:10E53000A01C00F01BFF07F809A06670122000FB6A
:10E54000057032464146023000F076FE23780F48CF
:10E550000133DBB2012B08BF0B4A237002BF1368E3
:10E5600001331360F3F792FD2046BDE8F0870135D3
:10E57000282DCED10548F3F789FD0020BDE8F087AE
:10E58000565D0020545D0020505D00204C5D002051
:10E5900010B50446FFF794FF4CB123783BB1013B23
:10E5A000DBB223701BB9044A1368013B13600348B4
:10E5B000BDE81040F3F76ABD505D00204C5D0020BF
:10E5C00070B5154606460C46FFF77AFF72782B6841
:10E5D00093420AD3B11C204600F02EFE73782B60C4
:10E5E0000548F3F753FD204670BD2A600248F3F753
:10E5F0004DFD002070BD00BF4C5D00202DE9F041B5
:10E60000174606468846FFF75BFF72783B68B3EB18
:10E61000C20F05D1B01C002501244FF0FF3316E0D6
:10E620002648F3F733FD6FF00100BDE8F081591C77
:10E6300037D190F800E018F80510714537D02B4617
:10E64000C4B1BEFA8EF46409A4B10135013095421B
:10E65000EDD33CB100233B601848F3F717FD0220CF
:10E66000BDE8F0815D1C05D11448F3F70FFD20468D
:10E67000BDE8F0811E4418F80310B2784A40072123
:10E6800042FA01F4E40748B202D40139F8D108464D
:10E6900000EBC3033B600948F3F7F8FC0120BDE839
:10E6A000F081002CE6D00478B4FA84F4CBE7002C97
:10E6B000CBD0B1FA81F46409C7E700BF4C5D0020FC
:10E6C00070B5FFF7FDFE0A4C002504F5347604F81A
:10E6D000025C04F8015C204610220021123400F094
:10E6E00045FEB442F3D10348BDE87040F3F7CEBC19
:10E6F000565D00204C5D0020D0400B1CD1409C4654
:10E70000203AD3401843524263469340184370471F
:10E710007BB972B90029BEBF00204FF0004106E06E
:10E7200008BF00281CBF6FF000414FF0FF3000F021
:10E73000C9B9ADF1080C6DE904CE002909DB002B45
:10E740001ADB00F04DF8DDF804E0DDE9022304B047
:10E750007047404261EB4101002B1BDB00F040F8A9
:10E76000DDF804E0DDE9022304B0404261EB410141
:10E77000524263EB43037047524263EB430300F0A2
:10E780002FF8DDF804E0DDE9022304B0404261EB3C
:10E7900041017047524263EB430300F021F8DDF87A
:10E7A00004E0DDE9022304B0524263EB4303704707
:10E7B00053B94AB9002908BF00281CBF4FF0FF31E8
:10E7C0004FF0FF3000F07EB9ADF1080C6DE904CEDA
:10E7D00000F006F8DDF804E0DDE9022304B070473C
:10E7E0002DE9F0478C460E460446089D002B50D17B
:10E7F0008A4217466CD9B2FA82FEBEF1000F0BD0E6
:10E80000CEF1200420FA04F401FA0EF644EA060CD4
:10E8100002FA0EF700FA0EF44FEA1749220CBCFB7D
:10E82000F9F01FFA87F809FB10C642EA064600FB1A
:10E8300008F3B34209D9F61900F1FF3280F02281C2
:10E84000B34240F21F8102383E44F61AA2B2B6FB30
:10E85000F9F309FB136642EA064403FB08F8A045F6
:10E8600009D9E41903F1FF3280F00A81A04540F292
:10E870000781023B3C44C8EB040443EA004000210A
:10E88000002D62D024FA0EF400232C606B60BDE8EA
:10E89000F0878B4207D9002D55D0002185E8410033
:10E8A0000846BDE8F087B3FA83F1002940F0908074
:10E8B000B34202D3824200F2F880841A66EB030668
:10E8C0000120B446002D40D085E81010BDE8F08747
:10E8D00012B90127B7FBF2F7B7FA87FEBEF1000FB6
:10E8E00035D1F31B4FEA17481FFA87FC0121B3FB10
:10E8F000F8F0220C08FB103642EA06460CFB00F347
:10E90000B34207D9F61900F1FF3202D2B34200F246
:10E91000CE801046F61AA2B2B6FBF8F308FB1366D7
:10E9200042EA06440CFB03FCA44507D9E41903F1B1
:10E93000FF3202D2A44500F2B5801346CCEB0404AA
:10E9400043EA00409CE729462846BDE8F087CEF11F
:10E95000200106FA0EF307FA0EF720FA01F94FEA42
:10E960001748CE4049EA0309B6FBF8FA4FEA1944C2
:10E9700008FB1A661FFA87FC44EA06430AFB0CF2FE
:10E980009A4200FA0EF40AD9DB190AF1FF3180F03D
:10E9900087809A4240F28480AAF1020A3B449B1A83
:10E9A0001FFA89F9B3FBF8F108FB113349EA034375
:10E9B00001FB0CF69E4207D9DB1901F1FF326BD245
:10E9C0009E4269D902393B449B1B41EA0A418EE7CA
:10E9D000C1F1200E22FA0EF48B40234320FA0EF7E9
:10E9E00006FA01F44FEA134C26FA0EF63C43B6FB46
:10E9F000FCF9270C0CFB19661FFA83F847EA064658
:10EA000009FB08F7B74202FA01F200FA01FA08D945
:10EA1000F61809F1FF3041D2B7423FD9A9F10209F6
:10EA20001E44F61BA0B2B6FBFCF40CFB146640EAD5
:10EA3000064704FB08F8B84507D9FF1804F1FF3072
:10EA400028D2B84526D9023C1F4444EA0940C8EB05
:10EA50000707A0FB02894F4544464E4614D329D0F0
:10EA600065B3BAEB040367EB060707FA0EFECB406B
:10EA7000CF404EEA030385E888000021BDE8F08717
:10EA80001346F8E61046E0E6B8EB020469EB03062D
:10EA90000138E5E70446D8E7114695E78146C0E727
:10EAA0008A467CE7023B3C4448E708460AE70238CE
:10EAB0003E442FE7C245E7D33E46D1E72946BDE8AD
:10EAC000F08700BF704700BF0A22002101F00ABA98
:10EAD0000A23002201F072B9014B1868704700BF89
:10EAE000840200208B891A072DE9F0410D468046EB
:10EAF00035D44A68002A6BDDEC6A002C47D003F459
:10EB00008052002192B2D8F80060C8F80010002AA4
:10EB100062D06A6D5F0705D569686B6B521A0BB1DD
:10EB20002B6CD21A0023296A4046A047441C39D0D6
:10EB3000AB892A692A60DB044FF000026A6045D481
:10EB4000696BC8F8006011B305F14403994202D023
:10EB5000404600F059FC00206863BDE8F0810E6972
:10EB6000AEB10C680E6098070CBF4B690023A41B64
:10EB70008B600AE023463246AF6A296A4046B847AE
:10EB80000028A4EB0004064404DD002CF2DC002085
:10EB9000BDE8F081AB8943F04003AB814FF0FF301B
:10EBA000BDE8F081D8F800201D2AF3D8184BD340D7
:10EBB00003F0010383F00101002BEBD0AB892C693A
:10EBC0006960D9042C60BBD5002AB9D16865B7E764
:10EBD0000A6C002A90DCDAE70123296A4046A04744
:10EBE000431C024602D0AB89EC6A93E7D8F80030A8
:10EBF000002BF8D01D2B01D0162B02D1C8F80060D5
:10EC0000C5E7AB8943F04003AB81BDE8F08100BFAD
:10EC1000010040200B6933B310B5044682B008B13F
:10EC20008369ABB1114B994219D0114B994218D05D
:10EC3000104B994208BFE168B1F90C3013B90020BC
:10EC400002B010BD204602B0BDE81040FFF74ABF39
:10EC5000019100F019F90199044B9942E5D16168DD
:10EC6000EAE7A168E8E70020704700BFEC4201082E
:10EC7000CC420108AC42010820B1054B014618689E
:10EC8000FFF7C8BF034B0449186800F043B900BF41
:10EC9000840200200C43010815EC00080020704796
:10ECA000014900F037B900BF15EC0008002070479B
:10ECB00070B568234D1E03FB05F50E4605F1740182
:10ECC00000F0E8FB044640B100210C30666005F11D
:10ECD00068022160A06000F049FB204670BD00BFC3
:10ECE0001F4B70B51D68AB69064613B9284600F086
:10ECF00039F848356B68AC68013B05D521E0013B2C
:10ED00005A1C04F168041CD0B4F90C20002AF6D176
:10ED1000002501234FF6FF72E281A381656625601D
:10ED2000A560656025616561A5612946082204F139
:10ED30005C0000F01BFB6563A563A564E5642046E9
:10ED400070BD2B680BB11D46D4E704213046FFF798
:10ED5000AFFF286008B10546CCE70C23336070BDD7
:10ED60000C4301083D4B3E491A682DE9F04F904293
:10ED70004FF000038364C364036508BF012383B0BD
:10ED800008BF836181620746FFF7AAFF78603846B3
:10ED9000FFF7A6FFB8603846FFF7A2FF7D68F8606E
:10EDA00000240423AB812C606C60AC606C66EC8149
:10EDB0002C616C61AC61214605F15C00082200F019
:10EDC000D5FABE68DFF89CB0DFF89CA0DFF89C9015
:10EDD000DFF89C80C5F824B001230922C5F828A0DB
:10EDE000C5F82C90C5F830802D622146F381B281A0
:10EDF00034607460B460746634617461B46106F147
:10EE00005C000822019300F0B1FAFD68366212201E
:10EE10000222C6F824B0C6F828A0C6F82C90C6F87E
:10EE200030802146A881EA812C606C60AC606C6601
:10EE30002C616C61AC6105F15C00082200F096FA6F
:10EE4000019B2D62C5F824B0C5F828A0C5F82C9008
:10EE5000C5F83080BB6103B0BDE8F08F0C430108FA
:10EE6000A1EC000811F7000839F7000875F7000851
:10EE700095F70008024B0349186800F04BB800BF33
:10EE80000C43010815EC0008836903B96AE7704771
:10EE9000704700BF704700BF704700BF704700BF9A
:10EEA000024B0349186800F00FB800BF840200202D
:10EEB000ADEC0008024B0349186800F005B800BF2C
:10EEC000840200209DEC00082DE9F04110F1480774
:10EED0001BD0884600267D68BC68013D0FD4A389FD
:10EEE000012B05F1FF3506D9B4F90E300133204668
:10EEF00001D0C04706436B1C04F16804EFD13F68A2
:10EF0000002FE8D13046BDE8F0813E463046BDE8EE
:10EF1000F08100BF2DE9F84310F148071FD0884663
:10EF200006464FF000097D68BC68013D11D4A389F5
:10EF3000012B05F1FF3508D9B4F90E300133214614
:10EF4000304602D0C04749EA00096B1C04F168044E
:10EF5000EDD13F68002FE6D14846BDE8F883B946B9
:10EF60004846BDE8F88300BF38B50A4B1C68E16B22
:10EF7000054621B12846BDE8384000F00DB82420F0
:10EF800000F018F9E06301462846BDE8384000F07B
:10EF900003B800BF840200200268634B63482DE978
:10EFA000F04383FB02431344D417C4EB234400FB18
:10EFB00014200028C0F2AE8004F52F2404F66C243F
:10EFC0005B4E5C4D5C4ADFF884E1DFF884C15B4F47
:10EFD00086FB0436E317C3EBE63605FB0645AB08B4
:10EFE000A2FB038205EBD222AEFB0383A2EBD3127A
:10EFF0002B09ACFB03C3A2EB1313DFF858C1504A33
:10F00000ACFB038CA2FB038205EBDC3C9D1A9B0846
:10F0100002EB5505AEFB03232D0A4A4AACEBD31392
:10F0200040F26D1E0EFB1533DFF82CC182FB002E63
:10F0300003EB830202328644ACFB02C24FEAE07C5F
:10F04000CCEBEE2C4FF4616E0EFB1C000334DFF8AA
:10F050000CE1C1F808C084FB078904EB090C8EFBA6
:10F06000007EE717C7EBAC07C7EBC707D209092A31
:10F07000A4EB07044FEAE078864402EBC20C8CBF95
:10F080006FF009070227C8EB6E1E0CEB0C1CDFF8B3
:10F09000D0808C614FF4C87404FB06563A440CF1DE
:10F0A000020CCEEB0E17A8FB0C4CA0EB87005C1CEF
:10F0B000012A98BF0136B3F5997FA4EB9C0481E83F
:10F0C000014024D2A80717D01F48A0FB0570C00933
:10F0D0004FF4C87707FB1055B5FA85F56D093B333A
:10F0E0002B44A6F26C76002008624E61CB610A6167
:10F0F000CC600846BDE8F0831348A0FB05704009CA
:10F10000642707FB10500028DED00125E7E7A3F5B0
:10F110009973E6E700F5A83004F52F2400F5C070D8
:10F1200004F66B244CE700BF07452EC28051010056
:10F13000BD066B394FC5FDFF7F206B399324499283
:10F1400061F31967C5B3A2911F85EB51D97CC659EC
:10F1500041D672001F2BD3E5D7802BD689888888AB
:10F16000CDCCCCCC70B50F4E0F4D761BB61018BF62
:10F17000002405D0013455F8043B9847A642F9D144
:10F180000A4E0B4D761BF1F701F8B61018BF00249C
:10F1900006D0013455F8043B9847A642F9D170BD1A
:10F1A00070BD00BF54440108544401085444010890
:10F1B00054440108024B0146186800F06BB900BFC7
:10F1C00084020020024B0146186800F01DB900BF00
:10F1D00084020020032A70B426D940EA01039B0769
:10F1E00011D004780D78AC4222D10244431C05E0D2
:10F1F00013F8014B11F8015FAC4219D19342F7D1DA
:10F20000002070BC70470C4603461E682568AE425D
:10F210001846214603F1040304F10404E1D1043A41
:10F22000032A18462146F0D8002ADAD11046E8E72A
:10F23000601B70BC704700BF844641EA000313F0B6
:10F2400003036DD1403A41D351F8043B40F8043BED
:10F2500051F8043B40F8043B51F8043B40F8043BB0
:10F2600051F8043B40F8043B51F8043B40F8043BA0
:10F2700051F8043B40F8043B51F8043B40F8043B90
:10F2800051F8043B40F8043B51F8043B40F8043B80
:10F2900051F8043B40F8043B51F8043B40F8043B70
:10F2A00051F8043B40F8043B51F8043B40F8043B60
:10F2B00051F8043B40F8043B51F8043B40F8043B50
:10F2C00051F8043B40F8043B403ABDD2303211D3F0
:10F2D00051F8043B40F8043B51F8043B40F8043B30
:10F2E00051F8043B40F8043B51F8043B40F8043B20
:10F2F000103AEDD20C3205D351F8043B40F8043BF0
:10F30000043AF9D2043208D0D2071CBF11F8013BED
:10F3100000F8013B01D30B8803806046704700BFB3
:10F32000082A13D38B078DD010F003038AD0C3F1C2
:10F330000403D21ADB071CBF11F8013B00F8013BA4
:10F3400080D331F8023B20F8023B7BE7043AD9D363
:10F35000013A11F8013B00F8013BF9D20B78037038
:10F360004B7843708B7883706046704770B4840725
:10F3700046D0541E002A41D0CDB2034602E0621EA0
:10F38000E4B3144603F8015B9A07F8D1032C2ED995
:10F39000CDB245EA05250F2C45EA054519D903F1FB
:10F3A00010022646103E0F2E42F8105C42F80C5C0C
:10F3B00042F8085C42F8045C02F11002F2D8A4F1B1
:10F3C000100222F00F0204F00F041032032C134439
:10F3D0000DD91E462246043A032A46F8045BFAD8A1
:10F3E000221F22F003020432134404F003042CB160
:10F3F000C9B21C4403F8011BA342FBD170BC704787
:10F4000014460346C2E700BF30B481B151F8043C52
:10F410000439002BB8BFC9181D4B1A682AB18A429B
:10F420000AD908680C18A24225D04A60196030BC7D
:10F4300070478B4203D81A465368002BF9D11468E1
:10F4400015198D420CD007D808680C189C4218D0AA
:10F450004B6030BC516070470C23036030BC704778
:10F4600009680C44111999421460E0D10ACB0C448C
:10F4700053601460DBE7146852684A6020440860F7
:10F48000D4E71C685B684B60204408605160CEE79D
:10F490002460002070B5CD1C25F0030508350C2D27
:10F4A00038BF0C25002D06463BDBA94239D8274939
:10F4B0000A6852B113685B1B04D436E023685B1BF7
:10F4C0001AD522465468002CF8D149681F4C0029EF
:10F4D00036D029463046F0F75DFE431C21D0C41CCF
:10F4E00024F00304A04205D0211A3046F0F752FE62
:10F4F000013016D0256004E00B2B0DD923601C448D
:10F50000256004F10B0020F00700231DC31A02D070
:10F510005A42E25070BD70BD94420ED06368536091
:10F52000EFE70C233360002070BD0B2B03D853682A
:10F5300014460B60E5E71446E0E713461446F8E787
:10F540003046F0F727FE6060C3E700BF246000206C
:10F550000EB410B5044683B018B183690BB9FFF738
:10F5600093FC06A803460190059AA168204600F086
:10F57000F5FE03B0BDE8104003B070470FB410B5FE
:10F580000A4B1C6882B024B1A36913B92046FFF767
:10F590007BFC05A803460190049AA168204600F070
:10F5A000DDFE02B0BDE8104004B0704784020020C8
:10F5B0002DE9F0410E46804600283ED08369002B9D
:10F5C00039D084682F4B9C4243D02F4B9C4256D05D
:10F5D0002E4B9C4208BFD8F80C40A3891B073DD591
:10F5E0002369002B3AD0013EA36816F8015F013B66
:10F5F000A360B5B1002B04DB23685A1C22601D7088
:10F60000F2E7A769BB4222462946404601DB0A2DA4
:10F61000F2D100F019FD0130E6D14FF0FF30BDE826
:10F62000F081002B21DB23680A22591C21601A700B
:10F630001046BDE8F081FFF727FCD8F81830D8F85D
:10F640000840002BBED14046FFF71EFC0D4B9C42EC
:10F65000BBD1D8F80440A3891B07C1D4214640463A
:10F6600000F054FD0028BED0D7E7224640460A21CC
:10F6700000F0EAFC0130D0D00A20BDE8F081D8F8D3
:10F680000840AAE7EC420108CC420108AC4201085C
:10F69000024B01461868FFF78BBF00BF84020020B1
:10F6A00038B50C46054608B18369B3B1114B9C428D
:10F6B00018D0114B9C4217D0104B9C4208BFEC68ED
:10F6C0002846214601F080F980B994E80C00013BFE
:10F6D000511C84E80A00107838BDFFF7D5FB054BB4
:10F6E0009C42E6D16C68EBE7AC68E9E74FF0FF308D
:10F6F00038BD00BFEC420108CC420108AC42010811
:10F70000024B01461868FFF7CBBF00BF8402002000
:10F7100010B50C46B1F90E10F0F75AFD002803DBC6
:10F72000636D0344636510BDA38923F48053A381F3
:10F7300010BD00BF002070472DE9F0411646B1F919
:10F740000C201F46D3050C46054607D50022022390
:10F75000B1F90E10F0F749FDB4F90C20B4F90E1010
:10F7600022F48052A2813B4632462846BDE8F04151
:10F77000F0F732BD10B50C46B1F90E10F0F735FDBB
:10F78000A389421C0EBF23F4805343F48053606569
:10F79000A38110BDB1F90E10F0F722BD70B411F0C5
:10F7A000FF0434D085070FD00378002B5AD09C4239
:10F7B0002BD0431C05E013F8012B002A4FD09442B4
:10F7C00023D09A071846F6D10E0206F47F46264348
:10F7D000036846EA064601E050F8043F86EA03055E
:10F7E000A5F10132A3F1013122EA050221EA030366
:10F7F000134313F0803FEFD0037823B932E010F8C1
:10F80000013F002B2ED09C42F9D170BC7047840779
:10F810000BD00378002BF8D0431C03E002780133AF
:10F82000002AF2D099071846F8D10268A2F10133F4
:10F8300023EA020313F0803F08D150F8042FA2F10D
:10F84000013323EA020313F0803FF6D00378002B44
:10F85000DBD010F8013F002BFBD170BC7047104685
:10F8600070BC7047184670BC704700BF00000000B5
:10F870000000000000000000000000000000000088
:10F88000A2EB0300704700BF02780B78012A28BF63
:10F890009A42F5D16DE9044540EA0104CDE90267D9
:10F8A0006FF0000C4FEA447212B380EA010414F0C6
:10F8B000070F6AD100F0070420F0070004F00305E9
:10F8C00021F007014FEAC505F0E8042314F0040F06
:10F8D000F1E804670CFA05F462EA040266EA040639
:10F8E0000AD063EA0403624667EA0407664603E057
:10F8F000F0E80423F1E8046782FA4CF582EA060492
:10F90000A4FA8CF46CBB83FA4CF583EA0705A5FADC
:10F910008CF595B950E9022351E9026782FA4CF55A
:10F9200082EA0604A4FA8CF483FA4CF583EA07050C
:10F93000A5FA8CF52543DBD09CB92DBAB5FA85F430
:10F9400024F0070427FA04F1DDE9026723FA04F33F
:10F9500003F0FF0001F0FF01FDE80445A0EB01000A
:10F96000704724BAB4FA84F424F0070426FA04F1A8
:10F97000DDE9026722FA04F202F0FF0001F0FF0164
:10F98000FDE80445A0EB0100704714F0030F3CD1E3
:10F9900010F0030428D150F8082B51F8083B82FAE4
:10F9A0004CF582EA0305A5FA8CF55DB950F8042CF4
:10F9B00051F8043C82FA4CF582EA0305A5FA8CF56D
:10F9C000002DE8D02DBAB5FA85F424F0070423FA07
:10F9D00004F122FA04F202F0FF0001F0FF01FDE859
:10F9E0000445A0EB010070474FEAC40420F0030077
:10F9F00050F8082B21F0030151F8083B0CFA04F4ED
:10FA000062EA040263EA0403C9E710F003041AD0AF
:10FA1000A1EB040120F00300E40750F8042B06D00A
:10FA20000FD28B785FFAA2F4E41A06D12BB1CB780F
:10FA30005FFAB2F4E41A00D11BB920465DF8104B0E
:10FA4000704701F1040150F8042BCC0721F00301A9
:10FA500051F8043B48D824D222F07F4482FA4CF576
:10FA600094EA1325A5FA8CF50AD165B951F8043B3F
:10FA700084EA0204B4EB036F0ED150F8042BEBE7D9
:10FA80004FEA132355E035F07F454DD10878FDE866
:10FA90000445C0F1000070474FEA126203F0FF0313
:10FAA00047E002EA1C4482FA4CF594EA1345A5FAB1
:10FAB0008CF50AD165B951F8043B84EA0204B4EB31
:10FAC000034F0CD150F8042BEBE74FEA134330E01F
:10FAD00015EA1C4528D10B884FEA124229E04FEA6B
:10FAE000124203EA1C4324E002F0FF0482FA4CF5C0
:10FAF00094EA1365A5FA8CF50AD165B951F8043B6F
:10FB000084EA0204B4EB032F09D150F8042BEBE78D
:10FB10004FEA13630DE015F0FF0F05D10B684FEAB4
:10FB2000122223F07F4304E04FF00000FDE804457B
:10FB3000704712BA1BBA82FA4CF482EA0304A4FAA0
:10FB40008CF5B5FA85F402FA04F203FA04F34FEAED
:10FB50001260FDE80445A0EB1360704780EA0102E3
:10FB6000844612F0030F4FD111F0030F32D14DF83C
:10FB7000044D11F0040F51F8043B0BD0A3F10132F6
:10FB80009A4312F0803F04BF4CF8043B51F8043B09
:10FB900016D100BF51F8044BA3F101329A4312F081
:10FBA000803FA4F101320BD14CF8043BA24312F088
:10FBB000803F04BF51F8043B4CF8044BEAD0234685
:10FBC0000CF8013B13F0FF0F4FEA3323F8D15DF837
:10FBD000044B704711F0010F06D011F8012B0CF8FF
:10FBE000012B002A08BF704711F0020FBFD031F877
:10FBF000022B12F0FF0F16BF2CF8022B8CF80020FE
:10FC000012F47F4FB3D1704711F8012B0CF8012B80
:10FC1000002AF9D1704700BF00000000000000007A
:10FC200000000000000000000000000000000000D4
:10FC300000000000000000000000000000000000C4
:10FC400090F800F06DE9024520F007016FF0000C1C
:10FC500010F0070491F820F040F049804FF00004C4
:10FC60006FF00700D1E9002391F840F000F108009F
:10FC700082FA4CF2A4FA8CF283FA4CF3A2FA8CF3D7
:10FC80004BBBD1E9022382FA4CF200F10800A4FA3E
:10FC90008CF283FA4CF3A2FA8CF3E3B9D1E9042392
:10FCA00082FA4CF200F10800A4FA8CF283FA4CF3C9
:10FCB000A2FA8CF37BB9D1E9062301F1200182FA83
:10FCC0004CF200F10800A4FA8CF283FA4CF3A2FA89
:10FCD0008CF3002BC6D0002A04BF04301A4612BA97
:10FCE000B2FA82F2FDE8024500EBD2007047D1E99A
:10FCF000002304F00305C4F100004FEAC50514F029
:10FD0000040F91F840F00CFA05F562EA05021CBFF9
:10FD100063EA050362464FF00004A9E7002A41D0D8
:10FD200040EA010313F00303F0B425D1032A23D9D9
:10FD300004680D68AC421FD1043A35D0A4F10135F6
:10FD400025EA040414F0803F31D1071D0D1D0DE09C
:10FD500057F8043B0E68A3F10134B34224EA0304CC
:10FD60000AD1043A20D014F0803F23D1032A294637
:10FD7000384605F10405EBD803780C789C4202F173
:10FD8000FF320CD182B114B916E06AB17BB110F820
:10FD9000013F11F8014FA34202F1FF32F5D0181BC9
:10FDA000F0BC7047104670471046F0BC70471846CC
:10FDB000F0BC70470020F3E72046F1E72DE9F04F53
:10FDC000474C83460E46D4F800E000E02646344611
:10FDD00014F8015B0EEB0500407800F0080000F01D
:10FDE000FF080028F2D12D2D5CD02B2D04BF757893
:10FDF000B41C002B3ED0102B60D09A46B8F1000FF7
:10FE00000CBF6FF000404FF000400027B0FBFAF944
:10FE1000BC460AFB19000CE0303DAB4219DD7E1CEC
:10FE200005D0CC4523D820D00AFB0C5C012714F860
:10FE3000015B0EEB0506767816F0040FECD116F098
:10FE4000030606D0012E14BF57263726AD1BAB4242
:10FE5000E5DC7B1C16D0B8F1000F10D16046002AFB
:10FE600039D0DFB91160BDE8F08F8542DCDD4FF09D
:10FE7000FF37DCE7302D1AD00A239A46BEE7CCF1D3
:10FE8000000CEBE7B8F1000F4FF022030CBF6FF04E
:10FE900000404FF00040CBF80030F2B1611E11601D
:10FEA000BDE8F08FB41C75784FF00108A1E7237806
:10FEB00003F0DF03582B08D008239EE7302D9CD198
:10FEC000207800F0DF00582897D14FF0100A6578AD
:10FED0005346023492E7BDE8F08FBDE8F08F00BFD3
:10FEE000E802002010B4044C13460A46014620687C
:10FEF00010BCFFF763BF00BF840200202DE9F04F64
:10FF0000494C82460E46D4F800E000E026463446CE
:10FF100014F8015B0EEB0500407800F0080000F0DB
:10FF2000FF0C0028F2D12D2D54D02B2D04BF757855
:10FF3000B41C5BB1102B5ED04FF0FF38B8FBF3F868
:10FF400003FB08FB6FEA0B0B994607E0302D46D008
:10FF50000A23DFF8D88099464FF0050B0027384672
:10FF60000CE0303DAB4219DD7E1C05D0404522D867
:10FF70001FD009FB0050012714F8015B0EEB0506AA
:10FF8000767816F0040FECD116F0030606D0012E99
:10FF900014BF57263726AD1BAB42E5DC002F0FDB25
:10FFA000BCF1000F00D0404242B17FB91160BDE802
:10FFB000F08F5D45DDDD4FF0FF37DDE7BDE8F08F09
:10FFC0002223CAF800304FF0FF305AB3611E11608F
:10FFD000BDE8F08FB41C75784FF0010CA9E72378C9
:10FFE00003F0DF03582B0DD0082399464FF0070B81
:10FFF0006FF06048B2E7302D0ED1207800F0DF00BE
:020000040801F1
:10000000582809D14FF0100965784B464FF00F0B77
:1000100002346FF07048A1E74FF00F0B6FF070489B
:1000200099469BE7BDE8F08FE8020020999999195D
:1000300010B4044C13460A460146206810BCFFF772
:100040005DBF00BF84020020F8B50E461446054689
:1000500010B18369002B41D0254B9C4243D0254BE6
:100060009C4242D0244B9C4208BFEC68A389A26901
:10007000A2601A0721D52369FBB122686169D31AEE
:100080008B42F7B221DA0133A168501C0139A1601B
:100090002060167062699A4206D0A389DB0701D5F9
:1000A0000A2F01D03846F8BD21462846FEF7B2FD9A
:1000B0000028F7D04FF0FF37F4E72146284600F03C
:1000C00025F80028F6D12369D7E721462846FEF710
:1000D000A1FD0028EED122680123D5E7FEF7D4FE6A
:1000E000034B9C42BBD16C68C0E7AC68BEE700BF65
:1000F000EC420108CC420108AC420108024B0A461E
:1001000001461868FFF7A0BF84020020384B70B585
:100110001D6806460C4615B1AB69002B42D0354B25
:100120009C4245D0344B9C4258D0344B9C4208BF33
:10013000EC68B4F90C2093B219070CD52069A8B16A
:1001400013F001021ED0636900225B42A361A2602A
:10015000F0B1002070BDDD0642D558072AD42069D1
:1001600042F00803A3819BB20028E9D103F4207276
:10017000B2F5007FE4D03046214600F06FF8A38945
:100180002069DDE7990758BF6269A2600028E0D1C5
:10019000B4F90C301A06DDD543F04003A3814FF0CB
:1001A000FF3070BD2846FEF76FFE124B9C42B9D15E
:1001B0006C68BEE7616B51B104F14403994204D00D
:1001C0003046FFF721F9B4F90C20002363630023C4
:1001D0002069636022F024022060C1E7AC68A8E7D0
:1001E00042F04002092333604FF0FF30A28170BD1E
:1001F00084020020EC420108CC420108AC42010814
:1002000070B50C46B1F90E10002990B015461E4687
:1002100013DB01AAEFF7EEFF00280EDB029A02F4CF
:100220007042A2F50052B2FA82F252094FF4806392
:10023000002032602B6010B070BDA38900221B0625
:10024000326004D5402300202B6010B070BD4FF405
:10025000806300202B6010B070BD00BF8A899207B8
:100260000B4606D501F1470201211A601A61596156
:100270007047F0B583B001AB6A460C460546FFF700
:10028000BFFF009906462846FFF704F9B4F90C3081
:10029000D0B1019A124F0099AF6243F08003A3815D
:1002A0002060206161611AB93343A38103B0F0BDBE
:1002B0002846B4F90E10EFF7A2FFB4F90C3000286D
:1002C000F2D043F00103EFE79A05EFD404F14702BF
:1002D00043F002030121A381226022616161E5E70D
:1002E000A1EC00089368013B002B10B4936007DB7E
:1002F000CCB21368581C10601970204610BC7047AF
:100300009469A34202DBCCB20A2CF2D110BCFFF7F5
:100310009BBE00BF93B1F8B514460F460646D518EC
:1003200001E0AC4208D03A4614F8011B3046FFF712
:10033000D9FF431CF5D1F8BD0020F8BD002070475F
:10034000936810B5144613B95360184610BD00F0F9
:10035000D1FB0023A360636010BD00BF2DE9F04F07
:100360009DB0884614460393814618B18369002BDB
:1003700000F00B818B4B984500F00D818A4B98451E
:1003800000F00C81894B984508BFD9F80C80B8F86B
:100390000C301D0740F1EF80D8F81030002B00F032
:1003A000EA8030238DF82A302378814DDFF804A2CB
:1003B0000021202209918DF82920002B00F0858052
:1003C000252B264603D117E0252B00F0868016F852
:1003D000013F002BF8D1B6EB040B76D022465B46EA
:1003E00041464846FFF796FF01306ED0099B3278B0
:1003F0005B440993002A68D000234FF0FF31721C40
:100400000493079306938DF853301A9305910126B0
:1004100004E0049906FA03F30B430493144664487A
:100420002178052200F0ECFC621C431B0028F0D16F
:10043000049BD80644BF20228DF853201907217849
:1004400044BF2B228DF853202A2968D0A1F1300215
:10045000092A0BD8079B14F8011F03EB830302EB57
:100460004303A1F13002092AF5D907932E293FD081
:100470000322504800F0C4FC48B10499CAEB0000C4
:10048000402202FA00F041EA00030134049321788B
:1004900049488DF828100622013400F0B1FC0028EC
:1004A0005FD0464BEBB103AB00934246444B04A9EB
:1004B0004846AFF3008007467A1C06D0099B3B44B0
:1004C00009932378002B7FF47BAFB8F80C305B06E0
:1004D00058D409981DB0BDE8F08FB6EB040B8BD053
:1004E0007CE7039B073323F0070308330393E5E717
:1004F00061782A291DD0A1F130020023092A04F1D4
:1005000001040593B4D814F8011F03EB830302EB35
:100510004303A1F13002092AF5D90593A8E7039A0C
:10052000116804320029039215DB079161780134C8
:100530009CE7039B1A680592002A03F104030393C6
:10054000B8BF4FF0FF3204F10203AEBFA178A1782B
:1005500005921C468CE7494243F00203079104933D
:10056000E4E703AB00934246154B04A9484600F06C
:10057000CDF80746A0E741464846FFF7C7FD0028EB
:100580003FF40FAF4FF0FF30A4E7FEF77DFC054BC3
:1005900098457FF4F3AED9F80480F8E6D9F80880DE
:1005A000F5E600BFEC420108CC420108AC4201086C
:1005B00018440108204401082444010800000000F8
:1005C0001503010810B4044C13460A46014620687E
:1005D00010BCFFF7C3BE00BF840200202DE9F04726
:1005E0000C4691460969A268DDF820808A42B8BFAE
:1005F0000A46C9F8002094F8431006461F4611B178
:100600000132C9F80020236899065DD5D9F8002089
:100610000232C9F80020236813F0060F19461DD1D5
:10062000E1688A1A002AD8BF194617DD04F1190AB1
:10063000002505E0E368D9F800209B1AAB420CDDE9
:100640000123524639463046C047013005F10105C5
:10065000F0D14FF0FF30BDE8F087216894F84330C7
:10066000003318BF01238A060AD5E1185A1C30202E
:1006700081F84300224494F8451082F84310023375
:1006800004F1430239463046C0470130E1D02368C7
:1006900003F00603042B29D0A36822699342C8BF44
:1006A0004FF000092FDD9B1A99441A34002501E010
:1006B0004D4528D00123224639463046C0470130F7
:1006C00005F10105F4D1C4E713F0060F08D1E16884
:1006D000D9F800208A1A002AD8BF1946A6DCBDE73F
:1006E00094F84330003318BF0123C9E7D9F800005C
:1006F000E168A3682269091A934221EAE179D2DC10
:10070000B9F1000FD1D10020BDE8F0872DE9F04309
:100710000C46097E85B06E29064617460C98984609
:1007200004F1430C5AD01AD8632900F0128100F268
:10073000D68000295CD0582940F0F58084F8451017
:1007400022680368DFF864E2150603F104011ED491
:10075000550653BF1B6801601B88016019E07329AF
:1007600000F0CF807ED86F2900F0E480702940F03F
:10077000DA80226842F020022260782384F8453033
:100780000368DFF82CE2150603F10401E0D51B68CD
:100790000160D00744BF42F020022260002B40F0ED
:1007A0009080226822F0200222601021002284F82A
:1007B00043206068A0600028C0F28880226822F090
:1007C00004022260002B62D1002840F0818065463F
:1007D00008296AD0C5EB0C0323610CE023681A06D4
:1007E00040F1D58003686269191D01601B681A60B9
:1007F000002365462361CDF800803B4603AA2146CD
:100800003046FFF7EBFE013021D02A4623693946F6
:100810003046C04701301AD02368039813F0020F06
:10082000E36819D01A1A002A16DD04F11909002507
:1008300004E0E36803981A1AAA420DDD01234A4630
:1008400039463046C047013005F10105F1D14FF07E
:10085000FF3005B0BDE8F0839842B8BF184605B038
:10086000BDE8F083752965D078295CD1226884E7DA
:100870006168A1602D200029C3F1000384F84300C2
:1008800021DB22F00402DFF824E122600A21654620
:10089000B3FBF1F201FB123013461EF8002005F8FD
:1008A000012D002BF4D1082994D12368D90791D5C3
:1008B000626823699A428DDC302305F8013C013DD2
:1008C00088E7102172E7DFF8E4E00A21002BDED18F
:1008D0009EF8003084F8423004F1420578E764293C
:1008E00001D069291FD122680368150603F10401AC
:1008F0003AD51B680160002BBADBDFF8B0E00A21B3
:1009000057E703686268191D01601D6800212846C9
:1009100000F076FA002846D0401B6060206100237A
:1009200084F8433067E7012384F84210236104F11F
:100930004205F4E723681A061ED503681A1D1B68D2
:100940000260227EDFF864E06F2A14BF0A210821CA
:100950002CE703681A68191D0123016004F14205A0
:1009600084F842202361DAE7550653BF1B68016013
:10097000B3F900300160BEE713F0400F036803F1E4
:10098000040215BF02601B681B880260D9E713F0E0
:10099000400F0368626903F1040101601B6814BF22
:1009A0001A801A6024E76068B8E700BF2C44010889
:1009B00040440108838903F00903092B01D000207A
:1009C0007047FEF759B900BFF8B50C46054610B19F
:1009D0008369002B45D0424B9C4247D0414B9C42FF
:1009E0006FD0414B9C4208BFEC68B4F90C2093B225
:1009F00000219F06616031D45E0722D5616B61B131
:100A000004F14403994202D02846FEF7FDFC236C12
:100A1000636000206063002B43D12369002B52D018
:100A2000B4F90C70BEB2B30722D122692260284605
:100A30006369656A216AA8470028606009DD0020B3
:100A4000F8BDD80644D519072ED442F00402A2817D
:100A5000E3E7A3891DD143F02003A3814FF0FF30CA
:100A6000F8BDFEF711FA1E4B9C42B7D16C68BCE78B
:100A70001E4B1F4918680123A38106F00906FEF7E3
:100A800023FA092EA781D0D121462846FEF72AF85D
:100A9000CBE7002243F04003A38162604FF0FF30B8
:100AA000F8BDE36B2360F8BD21462846FEF7B2F897
:100AB0000028D3D1B4F90C20A060A06122F0080274
:100AC000C3E7AC6891E721462846FFF7C7FBA7E7D5
:100AD00042F0400209232B604FF0FF30A281F8BDA5
:100AE000EC420108CC420108AC4201080C43010869
:100AF000B50901089368002B76D02DE9F04F8B895A
:100B000085B00C4619070190164629D522693AB3DB
:100B100003F002081FFA88F0356800282FD04FF044
:100B20000009B44FC846B246B84543464A4628BFB6
:100B30003B460198B8F1000F50D0216AA66AB04731
:100B4000002871DDDAF808301B1A8144C0EB080870
:100B5000CAF80830002BE7D1002005B0BDE8F08FBF
:100B600021460198FFF7D2FA002840F03A81A38984
:100B7000356803F002081FFA88F00028CFD113F07F
:100B800001095BD14F4602961FB39A05D4F808803D
:100B90002CD54745C246C0F0A48013F4906F40F0B6
:100BA000B18020685246494600F07AF9A06823686F
:100BB000C8EB00005344A06023603846029A936853
:100BC0001B1A81443F1A9360002BC5D0A389002FC4
:100BD000DBD1D5F800906F680835D5E7D5F80090DF
:100BE000D5F8048008359FE7002070472068236906
:100BF000984203D861698F4280F0B780B84528BF1A
:100C0000B8464246494600F04BF9A3682268C8EB53
:100C100003034244A3602260002B49D1214601987E
:100C2000FDF7F8FF002843D0B4F90C3043F040033F
:100C30004FF0FF30A38105B0BDE8F08F80460290F1
:100C400082468146B9F1000F2AD0029B002B4CD07E
:100C5000206823696269C845C34628BFCB469842CD
:100C60005F4604D9A36813449B4500F390809345E5
:100C700020DB1346A76A216A01985246B847071E2F
:100C8000D2DDB8EB070823D0B368DB1BBA44C7EB4F
:100C90000909B360002B3FF45FAFB9F1000FD4D165
:100CA0000023D5F800A0D5F8049002930835C9E7D1
:100CB000404683E75A46514600F0F2F8A26823689E
:100CC000CBEB02025B44B8EB0708A2602360DBD1E8
:100CD00021460198FDF79EFF0028A5D1CDF8088098
:100CE000D2E72068B846BA465CE74A460A21504631
:100CF00000F086F800286FD001300123CAEB00080D
:100D00000293A5E762692068216902EB4208C1EB02
:100D1000000A08EBD8780AF101004FEA6808384465
:100D20004045424684BF804642465B0542D5114657
:100D30000198FEF7AFFB8346002855D05246216943
:100D4000FEF77AFAA38923F4906343F08003A3812A
:100D5000CAEB08030BEB0A00C4F81480C4F810B007
:100D60002060A360B846BA461CE76FF00043BB4260
:100D700028BF3B464A4693FBF1F30198A66A01FB64
:100D800003F3216AB04700283FF718AF4CE71A4633
:100D90005146039300F084F82268039B01981A449B
:100DA00022602146FDF736FF039B00287FF43CAF0D
:100DB0001F4666E7019800F0D7F883460028C7D1A0
:100DC000019D21692846FEF71FFBB4F90C300C2267
:100DD00023F080032A6029E7012309F10108029327
:100DE00036E74FF0FF30B8E6019A0C231360B4F9F0
:100DF0000C301BE700FCFF7F00000000000000003B
:100E000001F0FF01102A2BDB10F0070F08D010F8BB
:100E1000013B013A8B422DD010F0070F42B3F6D1BF
:100E2000F0B441EA012141EA014122F007047FF0D8
:100E300000070023F0E80256083C85EA010586EA2F
:100E4000010685FA47F5A3FA87F586FA47F6A5FA6B
:100E500087F68EB9EED1F0BC01F0FF0102F0070277
:100E600032B110F8013B013A83EA010313B1F8D122
:100E70000020704701387047002D06BF3546033803
:100E8000073815F0010F07D1013015F4807F02BF3C
:100E9000013015F4C03F0130F0BC0138704700BF8D
:100EA0008842F0B50DD98B1898420AD28118002AD1
:100EB00051D09A1A13F8014D01F8014D9342F9D11E
:100EC000F0BD0F2A48D941EA00039B0746D100F143
:100ED000100401F11003154653F8106C44F8106C1F
:100EE00053F80C6C44F80C6C53F8086C44F8086C1C
:100EF000103D53F8046C44F8046C0F2D03F11003FB
:100F000004F11004E8D8A2F1100323F00F0302F05B
:100F10000F0E1033BEF1030F1944034421D91E1FD5
:100F20000D467446043C55F8047B46F8047F032CB8
:100F3000F8D8AEF1040424F003040434234421441B
:100F400002F0030262B1013B0A4411F8014B03F8BD
:100F5000014F8A42F9D1F0BD0346F3E70346F2E7B9
:100F6000F0BD7246EEE700BFF9B1F8B5064615468A
:100F7000B2B10C4600F01CF8854201D82046F8BDFD
:100F800029463046FEF786FA074668B12A462146CA
:100F9000FEF752F930462146FEF736FA3846F8BDDC
:100FA000FEF732FA2846F8BDF8BD1146FEF772BAD0
:100FB00051F8040C0028BEBF091851F8043CC018B1
:100FC000043870474E4D492048414E444C4552002C
:100FD0004D454D204D414E4147452048414E444CE2
:100FE000455200425553204641554C542048414EED
:100FF000444C4552005553414745204641554C54B9
:101000002048414E444C4552004445425547204DEE
:101010004F4E2048414E444C45520044554D4D5989
:101020002048414E444C4552000A495352207374A3
:1010300061636B206F766572666C6F7765640053D1
:101040007461636B20706F696E74657220636F7278
:101050007275707465642C20726573657420746F8A
:1010600020746F70206F6620737461636B000A4395
:101070006F6E74657874206265666F726520686152
:1010800072646661756C743A0020202072303A20D8
:1010900030782530386C780A20202072313A2030A0
:1010A000782530386C780A20202072323A20307847
:1010B0002530386C780A20202072333A2030782589
:1010C00030386C780A0020207231323A203078258E
:1010D00030386C780A2020206C723A203078253025
:1010E000386C780A20202070633A20307825303818
:1010F0006C780A20207073723A2030782530386C72
:10110000780A0A004653522F4641523A002043467D
:1011100053523A2030782530386C780A00204846FF
:1011200053523A2030782530386C780A00204446F3
:1011300053523A2030782530386C780A00204146E6
:1011400053523A2030782530386C780A00204246D5
:1011500041523A2030782530386C780A004D4D469F
:1011600041523A2030782530386C780A004D697346
:1011700063004558435F5245543A20307825303853
:101180006C780A00417474656D7074696E672074C0
:101190006F207265636F6E737472756374207374FD
:1011A00061746520666F7220646562756767696E39
:1011B000672E2E2E00496E204744423A0A202073A3
:1011C0006574202470633D3078256C780A20206691
:1011D00072616D6520300A202062740A000A49534A
:1011E0005220737461636B206F766572666C6F77E3
:1011F0006564206279206174206C656173742025B8
:10120000642062797465732E0A0048415244204676
:1012100041554C542048414E444C455200464149AA
:101220004C454420415353455254494F4E2E0025BE
:10123000700A002A2A2A2052494F54206B65726E88
:10124000656C2070616E69633A0A25730A0A002A88
:101250002A2A2068616C7465642E0A0A006D61692F
:101260006E28293A20546869732069732052494FC7
:101270005421202856657273696F6E3A20554E4B83
:101280004E4F574E20286275696C646469723A202B
:101290002F686F6D652F656C6F7065732F504645B5
:1012A00031352F52494F5429290A0069646C650071
:1012B0006D61696E005F5100E1130108E9130108D7
:1012C000F2130108FB1301080114010809140108B5
:1012D000121401081B140108241401082C1401081D
:1012E000341401087374617465006E616D650009E2
:1012F000706964207C20252D3231737C20252D39A6
:101300007351207C20707269207C20737461636B40
:10131000202028207573656429207C206261736514
:10132000206164647220207C2063757272656E7423
:1013300020202020200A000920202D207C206973F5
:10134000725F737461636B20202020202020202096
:101350002020207C202D20202020202020202D2017
:101360007C2020202D207C202536692028253569E9
:1013700029207C2025313070207C20253130700AD6
:10138000000925336869207C20252D323073207CAC
:1013900020252D387320252E3173207C202533699C
:1013A000207C20253669202825356929207C2025A8
:1013B000313070207C2025313070200A007C0053B1
:1013C000554D000925357320252D3231737C25318B
:1013D0003373253673202536692028253569290A77
:1013E0000073746F7070656400736C656570696E0E
:1013F0006700626C206D7574657800626C2072788D
:1014000000626C2073656E6400626C207265706CA3
:101410007900626C20616E79666C00626C20616C90
:101420006C666C00626C206D626F780072756E6E17
:10143000696E670070656E64696E67000044004005
:1014400000000200030002400200024007070026DD
:101450000048004000000400090C0240080C024053
:10146000070700270706040201070705030200001B
:101470000030014007000240060002400500024023
:101480000400024005000000001000000100000000
:10149000003800400F0402400E0402400D040240D8
:1014A0000C040240050000000040000000000000A5
:1014B00000000040FFFFFFFF01000000001C0000D3
:1014C000000C0040FFFFFFFF08000000003200009A
:1014D0000202000000000000000000000000000008
:1014E0004172726574206427757267656E6365006A
:1014F000626161643A613535353A3A3137303200EC
:101500004572726F72206372656174696E672055EF
:10151000445020736F636B00747073206465207493
:1015200072616E736D697373696F6E203A202569FD
:101530000A004572726575722064616E73206C6179
:101540002073796E6368726F6E69736174696F6E10
:10155000202D204E6F7576656C6C652074656E74F9
:101560006174697665203A006F6666736574203A27
:101570002025690A007265707269736520646520B0
:101580006C6120636F6D6D756E69636174696F6EF8
:10159000202D2074656E7461746976652064652001
:1015A00073796E6368726F6E69736174696F6E20B0
:1015B0003A004572726F722073656E64696E6720BF
:1015C0007265706C79004465677261646174696FFB
:1015D0006E00636F6D7074657572203A2025640A21
:1015E000006D7367206E6F6E2072656375004572C3
:1015F000726F722073656E64696E67206D657373B8
:10160000616765004572726F722072656365697605
:10161000696E67206D657373616765006572726FCF
:10162000723A20636F756C64206E6F74206164641D
:1016300020444F444147202825732920746F206996
:101640006E7374616E636520282564290A007375C2
:10165000636365737366756C6C792061646465643B
:101660002061206E65772052504C20444F44414702
:101670000A0052494F54206E6574776F726B207365
:101680007461636B206578616D706C65206170704A
:101690006C69636174696F6E00736F636B5F636C19
:1016A00069656E745F74687265616400736F636B03
:1016B0005F74696D655F7365727665725F74687279
:1016C00065616400736F636B5F7365727665725FEB
:1016D000746872656164006E6577206E6F64652062
:1016E0003F00416C6C2075702C2072756E6E696EB7
:1016F0006720746865207368656C6C206E6F770076
:101700000100000003000000060C0240021002402D
:10171000070C02400A0C02405B6175746F5F696ED2
:1017200069745F6E657469665D206572726F7220A0
:10173000696E697469616C697A696E672061743871
:1017400036726632787820726164696F202325755D
:101750000A006174383672663278780069707636BD
:1017600000293A11676E72635F6E65746465763A3C
:1017700020706F737369626C79206C6F7374206969
:101780006E746572727570742E00FF0200000000A6
:101790000000000000000000001A52504C0001023E
:1017A0000000366C6F00FF7F3F1F0F070301756459
:1017B0007000FFFFFE80000000000000000000003D
:1017C0000000000000000000000000000000000019
:1017D00000000000FF010000000000000000000009
:1017E00000000001FF0200000000000000000000F7
:1017F00000000001FF0200000000000000000001E6
:10180000FF000000FF0200000000000000000000D8
:1018100000000002000000000000000000000000C6
:1018200000000001303132333435363738396162E7
:1018300063646566003031323334353637383941C8
:101840004243444546007368656C6C3A20696E6398
:101850006F72726563742071756F74696E6700686A
:10186000656C70004465736372697074696F6E00B3
:10187000436F6D6D616E6400252D323073202573CA
:101880000A007368656C6C3A20636F6D6D616E64FD
:10189000206E6F7420666F756E643A2025730A009F
:1018A0007265626F6F74005265626F6F7420746846
:1018B00065206E6F6465007073005072696E74739A
:1018C00020696E666F726D6174696F6E2061626F00
:1018D00075742072756E6E696E67207468726561CA
:1018E00064732E0070696E67360050696E672076EB
:1018F00069612049434D5076360072616E646F6DA8
:101900005F696E697400696E697469616C697A6592
:1019100073207468652050524E470072616E646F88
:101920006D5F6765740072657475726E7320333213
:1019300020626974206F662070736575646F207211
:10194000616E646F6D6E657373006966636F6E665A
:10195000696700436F6E666967757265206E6574AE
:10196000776F726B20696E74657266616365730070
:10197000666962726F757465004D616E6970756C31
:1019800061746520746865204649422028696E6646
:101990006F3A2027666962726F757465205B6164B7
:1019A000647C64656C5D2729006E63616368650013
:1019B0006D616E616765206E65696768626F722030
:1019C00063616368652062792068616E6400726F8C
:1019D000757465727300495076362064656661756A
:1019E0006C7420726F75746572206C697374007208
:1019F000706C0072706C20636F6E666967757261DF
:101A000074696F6E20746F6F6C20282772706C2061
:101A100068656C702720666F72206D6F7265206933
:101A20006E666F726D6174696F6E29006E7470649A
:101A30006174650073796E6368726F6E697A65733D
:101A4000207769746820612072656D6F74652074F9
:101A5000696D65207365727665720000A0180108D3
:101A6000A718010859970008B7180108BA18010803
:101A700063970008E4180108EA180108D1B10008CA
:101A8000FA180108061901086D9700081B190108CA
:101A900026190108A59700084A19010853190108D9
:101AA00091A00008701901087919010801AB00081C
:101AB000A9190108B0190108E9AD0008CE190108FB
:101AC000D6190108E5AF0008EF190108F31901085C
:101AD000BDBA00082C1A0108341A0108D1BC00084C
:101AE00000000000000000000000000050524E47BF
:101AF00020696E697469616C697A656420746F200D
:101B000063757272656E742074696D653A20256420
:101B10000A0050524E4720696E697469616C697A97
:101B2000656420676976656E2076616C75653A201C
:101B300025640A004F464600534C45455000535417
:101B4000414E4442590049444C45005258005458B3
:101B50000052455345540025303878002873686F8B
:101B60007274292061646472657373006C6F6E67B0
:101B7000206164647265737300736F7572636520AE
:101B800061646472657373206C656E67746800636A
:101B900068616E6E656C0070616765006E65747774
:101BA0006F726B206964656E746966696572005452
:101BB0005820706F776572205B696E2064426D5D9E
:101BC000006D61782E2072657472616E736D697339
:101BD00073696F6E730043534D412072657472696F
:101BE000657300434341207468726573686F6C6469
:101BF000205B696E2064426D5D00656E6372797072
